:100000000C94121C0C94521C0C94521C0C94521CF8
:100010000C94521C0C94521C0C94521C0C94521CA8
:100020000C94521C0C94521C0C94521C0C94521C98
:100030000C94521C0C94521C0C94521C0C94521C88
:100040000C94521C0C94E99E0C94521C0C94521C5F
:100050000C94521C0C94F28C0C94521C0C94F07A5C
:100060000C94521C0C94AA3B0C94A03B0C94521C74
:100070000C94521C0C94521C0C94521C0C94521C48
:100080000C94521C0C94521C0C94521C0C94521C38
:100090000C94521C0C94521C0C94521C0C94521C28
:1000A0000C94521C0C94521C0C94521C0C94521C18
:1000B0000C94521C0C94521C0C94521C0C94521C08
:1000C0000C94521C0C94521C0C94521C0C94422DF7
:1000D0000C940C2D0C94521C0C94521C0C94521C1D
:1000E0000C94521C084AD73B3BCE016E84BCBFFD2A
:1000F000C12F3D6C74319ABD56833DDA3D00C77FF8
:1001000011BED9E4BB4C3E916BAAAABE0000008090
:100110003F05A84CCDB2D44EB93836A9020C50B91F
:10012000918688083CA6AAAA2ABE000000803F004B
:100130000C9461CF0C94D82D0C94A9F20C94543CDF
:100140000C943D2C0D94521D0C94B8F20C944C3C24
:100150000C94F32D0C94E42D0C94BBE40D945B1DD6
:100160000C94AFE40C942C770C94632C0C94C1F297
:100170000C940F790C943C700C94A9E40C94A8791D
:100180000D946E200C94B8E40C9458770C9468CEBF
:100190000C9432770C94F72B0C94A4F20C942A79DB
:1001A0000D94651D0C9444770D94761D0C94A4E673
:1001B0000C94ACF20C94BA790C94C7F20C943C7782
:1001C0000C945C770D94AD200C9482780C94B2E47E
:1001D0000C94062E0C94663C0C94503C0D94691DB6
:1001E0000D94AE1C0C94192C0D94371D0C941B2CE3
:1001F0000C940B770C94C4F20C9440770C94A3E409
:100200000C943B700D944E1C0D94FE2C0C94C1E488
:100210000D94E11C0C94BBF20C9423780D94771C84
:100220000C94CD2D0D946B1D0D942E1D0D947A20E4
:100230000C94EBE60C94FE2D0C94AFF20C94E83B7E
:100240000C94B5F20C94BEE40C9423E50C94367730
:100250000C94E82D0C943CCF0C94612C0C94F52B51
:100260000C943B2C0D94E01B0D94B9200D94811A35
:100270000C9425770C94D5E40D94231D0C945B3CD1
:100280000D94491D0C94BE2D0C946E3C0C94263C90
:100290000C94173C0C9452770C94BEF20C94483C8E
:1002A0000C940A7A0C9474E40C941ECE0C94A6E47C
:1002B0000C94DC2D0C94802D0C9421770C94F2CEB0
:1002C0000C9443CE0C944A770C941D770C94B9E6A9
:1002D0000C94E7790C943F2C0C94DCCD0C947AE6CA
:1002E0000C9406770C94353C0D949E200C944E771C
:1002F0000D94D4200D94C21C0C945F2C0D94321BD1
:100300000C941FE50C94EC2D0D941C2D0C94E02DF9
:100310000C9417CF0D94401D0C94CDCE0C94D42D7D
:100320000C94B5E40C94B2F20C94ACE40C94CB2B8A
:100330000D94B61B0C94172C0C94B96F0C94297760
:100340000D948B1C0C94443C0D94421A0C94A8CE32
:100350000C94403C0D94C5200C9406780C943C3CC5
:100360000C94AF2D0C94D72B0C94CB784E414E4966
:100370004E495459494E46CDCCCC3D0AD7233C1763
:10038000B7D13877CC2B329595E6241FB14F0A00B0
:100390000020410000C84200401C4620BCBE4CCAA0
:1003A0001B0E5AAEC59D7400407A10F35A00A0721D
:1003B0004E18090010A5D4E80000E87648170000A0
:1003C000E40B54020000CA9A3B000000E1F505006E
:1003D0000080969800000040420F000000A08601B7
:1003E000000000102700000000E803000000006487
:1003F00000000000000A00000000000100000000F2
:10040000002C76D888DC674F0823DFC1DFAE59E1C6
:10041000B1B796E5E3E453C63AE651997696E8E635
:10042000C28426EB898C9B62ED407C6FFCEFBC9C08
:100430009F40F2BAA56FA5F490055A2AF75C936B1A
:100440006CF9676DC11BFCE0E40D47FEF520E6B5D5
:1004500000D0ED902E0300943577050080841E08AF
:100460000000204E0A000000C80C333333330F98CD
:100470006E12831141EF8D2114893BE65516CFFE94
:10048000E6DB18D1844B381BF77C1D901DA4BBE420
:1004900024203284725E228100C9F124ECA1E53D62
:1004A00027434F4D4D554E49434154494F4E00440B
:1004B000525952554E004552524F525300494E46E2
:1004C0004F004543484F004572726F722077726942
:1004D00074696E6720746F20454550524F4D210A54
:1004E0000053544F505045442E20005072696E7492
:1004F00065722073746F7070656420647565207414
:100500006F206572726F72732E204669782074684E
:1005100065206572726F7220616E6420757365204C
:100520004D39393920746F20726573746172742E7D
:10053000202854656D7065726174757265206973E9
:100540002072657365742E20536574206974206170
:10055000667465722072657374617274696E67295E
:100560000A004E6F20436865636B73756D20776971
:100570007468206C696E65206E756D6265722C20E2
:100580004C617374204C696E653A20004E6F2043B5
:100590006865636B73756D2077697468206C696E2C
:1005A00065206E756D6265722C204C617374204CF1
:1005B000696E653A2000636865636B73756D206DC5
:1005C00069736D617463682C204C617374204C698D
:1005D0006E653A20004C696E65204E756D626572DD
:1005E000206973206E6F74204C617374204C696EA7
:1005F00065204E756D6265722B312C204C617374D1
:10060000204C696E653A20004D31313000536572DF
:1006100069616C20737461747573206D69736D61A9
:100620007463680A00776169740A00534420726534
:100630006164206572726F720A002121204B494C5F
:100640004C2063617573656420627920746F6F203C
:100650006D75636820696E6163746976652074697D
:100660006D65202D2063757272656E7420636F6DE9
:100670006D616E643A2000486F74656E6420496451
:100680006C652054696D656F757400486F74656E94
:10069000642049646C652054696D656F75740A0047
:1006A0003D3D6F6E46696C616D656E7452756E6F1F
:1006B00075743D3D007061757365004D36303000D6
:1006C0002066696C616D656E745F72756E6F7574AE
:1006D000200066696C616D656E745F72756E6F7512
:1006E0007420540046696C616D656E7452756E6F4E
:1006F00075742054004D3130303053006275737979
:100700003A2070617573656420666F7220696E703F
:1007100075740A00627573793A2070617573656447
:1007200020666F7220757365720A00627573793A7C
:100730002070726F63657373696E670A0025533AA0
:10074000202553002A2A2A6B696C6C2A2A2A0070F9
:100750006F7765726F6666004B494C4C45442E209E
:10076000005072696E7465722068616C7465642EE5
:10077000206B696C6C28292063616C6C6564210AAC
:10078000006563686F3A004572726F723A004269A1
:100790006C696E656172204C6576656C696E672068
:1007A000477269643A0A002F2F616374696F6E3A69
:1007B0000070726F6D70745F00627574746F6E009C
:1007C000626567696E00486F74656E6420746F6F50
:1007D00020636F6C640A0053656E64204D313038BD
:1007E00020746F20726573756D650A00496E7365BC
:1007F00072742066696C616D656E7420616E642030
:1008000073656E64204D3130380A00526568656149
:100810007420446F6E6500526568656174696E6727
:100820002E2E2E00526568656174004865617465FE
:10083000722054696D656F75740053656E64204D48
:1008400031303820746F2068656174206E6F7A7A59
:100850006C650A004E6F7A7A6C65205061726B6528
:10086000640070617573656400506175736500574D
:10087000616974696E6720666F722068656174755E
:10088000702E0A004C656176696E6720473236002B
:100890003F53706563696669656420582C5920630D
:1008A0006F6F7264696E617465206F7574206F6616
:1008B00020626F756E64732E0A003F28522965709E
:1008C0006561742076616C7565206E6F7420706C44
:1008D00061757369626C653B206D75737420626528
:1008E000206174206C6561737420312E0A003F28EA
:1008F00052296570656174206D757374206265207E
:10090000737065636966696564207768656E206EDB
:100910006F74207573696E6720616E204C43442E9E
:100920000A003F537065636966696564206E6F7A7B
:100930007A6C652074656D7065726174757265207E
:100940006E6F7420706C61757369626C652E0A003D
:100950003F5370656369666965642066696C616DA3
:10096000656E742073697A65206E6F7420706C6197
:10097000757369626C652E0A003F53706563696622
:10098000696564207072696D65206C656E67746856
:10099000206E6F7420706C61757369626C652E0ACD
:1009A000003F5072696D65206C656E677468206DDC
:1009B0007573742062652073706563696669656428
:1009C000207768656E206E6F74207573696E67207E
:1009D000616E204C43442E0A003F53706563696684
:1009E000696564206E6F7A7A6C652073697A652018
:1009F0006E6F7420706C61757369626C652E0A008D
:100A00003F52657472616374696F6E204D756C74CA
:100A100069706C696572206D7573742062652073EE
:100A200070656369666965642E0A003F537065638B
:100A300069666965642052657472616374696F6E7A
:100A4000204D756C7469706C696572206E6F7420CE
:100A5000706C61757369626C652E0A003F53706536
:100A6000636966696564206C61796572206865698F
:100A7000676874206E6F7420706C61757369626C46
:100A8000652E0A0043292E0A003F5370656369668C
:100A9000696564206265642074656D706572617457
:100AA000757265206E6F7420706C61757369626C0D
:100AB00065202834302D00473236207374617274FB
:100AC000696E672E2E2E0A004F46460A0046616464
:100AD00065204865696768742000426564204C653C
:100AE00076656C696E6720004661696C6564207488
:100AF0006F20656E61626C6520426564204C65768E
:100B0000656C696E670A00496E76616C6964206D78
:100B10006573682E0A0050726F62696E6720506FAD
:100B2000696E740025532025692F2569002E0A005F
:100B30002F0050726F62696E67206D657368207058
:100B40006F696E742000202844525952554E290076
:100B5000473239204175746F20426564204C6576B8
:100B6000656C696E67003F20284C2C522C462C4245
:100B700029206F7574206F6620626F756E64732E06
:100B80000A003F2856296572626F7365206C65768E
:100B9000656C20696D706C61757369626C65202885
:100BA000302D34292E0A00426164205A2076616C6F
:100BB00075650A004E6F2062696C696E656172200E
:100BC000677269640A00446576696174696F6E00D2
:100BD00025533A2025730046696E69736865642160
:100BE0000A003A207A3A2000206F662000476F6999
:100BF0006E6720746F3A20580043570A00206469DA
:100C0000723A0020616E676C653A005374617274C9
:100C1000207261646975733A004D343820506F69F1
:100C20006E740025533A2025642F256400506F739D
:100C30006974696F6E696E67207468652070726F81
:100C400062652E2E2E0A003F4C656773206F66206A
:100C50006D6F76656D656E7420696D706C6175730E
:100C600069626C652028302D3135292E0A003F201D
:100C700028582C5929206F7574206F6620626F7573
:100C80006E64732E0A0050726F6265206F75742057
:100C90006F6620626F756E6473003F53616D706C98
:100CA000652073697A65206E6F7420706C6175734E
:100CB00069626C652028342D3530292E0A004D34A8
:100CC00038205A2D50726F626520526570656174CC
:100CD0006162696C69747920546573740A003F28F5
:100CE00056296572626F7365206C6576656C206944
:100CF0006D706C61757369626C652028302D3429C4
:100D00002E0A005374616E646172642044657669D2
:100D10006174696F6E3A20002052616E67653A20F7
:100D200000204D61783A2000204D696E3A20002065
:100D30005369676D613A20004D65616E3A2000206D
:100D4000440020204D323030205300202844697365
:100D500061626C6564293A0046696C616D656E7408
:100D60002073657474696E67730020204D323031D2
:100D70002058004D617820416363656C6572617431
:100D8000696F6E2028756E6974732F733229002085
:100D9000204D3230332058004D61782066656564FF
:100DA00072617465732028756E6974732F732900DE
:100DB00020520020204D32303420500041636365C2
:100DC0006C65726174696F6E2028756E6974732F1B
:100DD0007332292028503C7072696E742D616363F0
:100DE000656C3E20523C726574726163742D616360
:100DF00063656C3E20543C74726176656C2D616352
:100E000063656C3E29005741524E494E4721204CA4
:100E10006F77205A204A65726B206D6179206C656E
:100E2000616420746F20756E77616E7465642070E4
:100E300061757365732E0A00205400205300202032
:100E40004D323035204200416476616E6365642026
:100E500028423C6D696E5F7365676D656E745F7483
:100E6000696D655F75733E20533C6D696E5F6665A5
:100E70006564726174653E20543C6D696E5F747286
:100E80006176656C5F66656564726174653E205865
:100E90003C6D61785F6A65726B3E20593C6D61788C
:100EA0005F6A65726B3E205A3C6D61785F6A65725D
:100EB0006B3E20453C6D61785F6A65726B3E290030
:100EC00020440020490020204D333031205000487C
:100ED0006F74656E6420504944002044002049002E
:100EE00020204D3330342050004265642050494466
:100EF0000020580020204D61783A2000200020205A
:100F00004D696E3A2000203B200020204D323131C7
:100F1000205300203B0020550020204D3630332048
:100F20004C0046696C616D656E74206C6F61642F56
:100F3000756E6C6F6164004D323453256C645425BA
:100F40006C64004739322E394525730047314625F8
:100F5000640047315A2573463630300047315825F2
:100F6000735925734633303030004D3130365025BB
:100F700069532569004D313039532569004D3230B0
:100F800030442573004739322E395A2573004D34C9
:100F900032305325635A257300473238523058593E
:100FA0000047315A257346363030004739322E39E2
:100FB0005A2573004739322E394530004D313039CA
:100FC000532569004D313930532569004D34323095
:100FD000205330205A30003D3D4F6E506F77657280
:100FE0004C6F7373526573756D653D3D00203B20FA
:100FF0000020204D343133205300506F7765722D1F
:101000006C6F7373207265636F76657279003B2035
:101010000020496E76616C6964206578747275642D
:101020006572200047322F4733206261642070616F
:1010300072616D65746572730A00536C6565702E1C
:101040002E2E005A2050726F6265205061737420FA
:101050004265640A005A2050726F626520506173C5
:101060007420426564004732384C3000205A3A20E0
:101070000020593A200042656420583A20004D650E
:10108000736820706F696E74206F7574206F6620AE
:1010900072616E67650A004D302053746F70004DA9
:1010A000312053746F7000436C69636B20746F2040
:1010B000526573756D652E2E2E004E6F204D6F7626
:1010C000652E00456E642066696C65206C697374DA
:1010D0000A00426567696E2066696C65206C6973F9
:1010E000740A004E6F206D656469610A0052657371
:1010F000756D696E6720534400286E6F2066696CB9
:1011000065290043757272656E742066696C653A74
:1011100020005072696E742074696D653A20000A6F
:1011200053746174733A2046696C616D656E742006
:10113000757365643A20002C204C6F6E676573747C
:10114000206A6F623A2000546F74616C2074696D7C
:10115000653A200053746174733A20002C20466174
:10116000696C65643A20002C2046696E6973686575
:10117000643A20005072696E74733A2000537461AF
:1011800074733A20006F6B006F666600C204BD0482
:10119000B604AF04A10444454255473A004D3131ED
:1011A00033205300544D3344203130532050726F5C
:1011B000204F46462E002F2F0046523A0020466C04
:1011C0006F773A200050726F6265204F66667365D4
:1011D00074205A0050726F6265204F6666736574A2
:1011E000205A0064697300656E0043290A00616239
:1011F0006C656420286D696E2074656D70200043F5
:101200006F6C6420657874727564657320617265B3
:101210002000504944204175746F74756E6500500C
:101220004944204175746F74756E65206661696C00
:10123000656421204261642068656174657220697B
:10124000640A004F4646004F4E00203B20486F7313
:10125000742068616E646C696E6720006D6D00209B
:101260003B2044697374616E6365200046696C615C
:101270006D656E742072756E6F757420004D34321A
:101280003120696E636F7272656374207061726180
:101290006D657465722075736167650A004D6573CD
:1012A0006820706F696E74206F7574206F6620728D
:1012B000616E67650A004F666673657473204170DE
:1012C000706C696564004572723A20546F6F2066D5
:1012D00061722100546F6F206661722066726F6DBB
:1012E000207265666572656E636520706F696E74E5
:1012F0000A00454550524F4D204F4B0A00290A0025
:1013000020746F20003F5A206F7574206F66207222
:10131000616E6765202800290A0020746F20003F55
:1013200059206F7574206F662072616E6765202882
:101330002D00290A0020746F20003F58206F75741B
:10134000206F662072616E676520282D004D38344D
:1013500000446F6E65207072696E74696E672066F6
:10136000696C650A004D3737004D333100454550F3
:10137000524F4D206461746173697A6520657272A1
:101380006F722E0A0053657474696E6720566F6C15
:10139000756D65204F6E203A200053657474696E38
:1013A00067205374616E646279204F6E203A20008A
:1013B00053657474696E6720566F6C756D65203A5D
:1013C000200053657474696E6720526F746174698C
:1013D0006F6E203A200053657474696E67205374F1
:1013E000616E6462792054696D65203A200053650E
:1013F0007474696E67205374616E646279203A2058
:101400000053657474696E67204272696768746E10
:10141000657373203A20004C6F6164696E672044E5
:1014200057494E204C43442073657474696E67209D
:1014300066726F6D20454550524F4D0A00446973E6
:1014400063617264696E67204457494E204C43447F
:101450002073657474696E672066726F6D204545F0
:1014600050524F4D202D2073657474696E67732040
:1014700076657273696F6E20696E636F72726563F1
:10148000740A0044697363617264696E672044572B
:10149000494E204C43442073657474696E6720661E
:1014A000726F6D20454550524F4D202D2073697A43
:1014B0006520696E636F72726563740A00290A00A1
:1014C0002062797465733B2063726320002073741B
:1014D0006F7265642073657474696E6773207265DA
:1014E00074726965766564202800202863616C63E6
:1014F000756C6174656429210A0020213D20004536
:101500004550524F4D20435243206D69736D6174B5
:101510006368202D202873746F7265642920002071
:1015200053697A653A2000496E6465783A20000074
:1015300000FA430000FA430000204100008C420002
:1015400000A0420000A0420000C8430080CF43EE4C
:10155000020000EE020000640000003C00000020D9
:101560004D61726C696E3D563836290A004545500A
:10157000524F4D2076657273696F6E206D69736D81
:10158000617463682028454550524F4D3D0024F456
:10159000D43050C38E20C2A24017828B7011127AB1
:1015A000910D816CD90AA861E108C758660761519D
:1015B00043061E4B5D05C145A7041A411104093DB0
:1015C0009803713931034036DB0265339102D43020
:1015D0005402802E1D02632CEE01752AC501B0282D
:1015E000A001102781018F2564012B244B01E022EB
:1015F0003401AC211F018D200D01801FFC00841ED1
:10160000ED00971DDF00B81CD200E61BC600201BB2
:10161000BC00641AB200B219A8000A19A0006A1826
:101620009900D117910040178B00B5168400311630
:101630007E00B31579003A157300C7146F00581473
:101640006A00EE1366008813630025135E00C7125C
:101650005B006C12570015125400C111510070113B
:101660004F0021114B00D61049008D104700461045
:10167000440002104200C00F4000800F3E00420FA5
:101680003C00060F3B00CB0E3800930E37005C0E7B
:101690003500270E3400F30D3200C10D3100900DDE
:1016A0003000600D2E00320D2D00050D2C00D90CE0
:1016B0002B00AE0C2900850C29005C0C2700350C92
:1016C00027000E0C2600E80B2400C40B2400A00BFE
:1016D00023007D0B23005A0B2100390B2100180B2E
:1016E0002000F80A1F00D90A1E00BB0A1E009D0A2E
:1016F0001D00800A1D00630A1C00470A1B002C0AFB
:101700001B00110A1A00F7091A00DD091900C409A3
:101710001900AB091900920917007B091800630929
:1017200017004C09160036091600200916000A0990
:101730001500F5081500E0081400CC081400B808DE
:101740001400A4081400900813007D0812006B0810
:10175000130058081200460812003408110023082C
:1017600011001208110001081100F0071000E00735
:101770001000D0071000C0071000B0070F00A1072D
:10178000100091070E0083070F0074070F00650714
:101790000E0057070E0049070E003B070D002E07ED
:1017A0000E0020070D0013070D0006070D00F906B7
:1017B0000C00ED060D00E0060C00D4060C00C80677
:1017C0000C00BC060C00B0060C00A4060B00990629
:1017D0000C008D060B0082060B0077060B006C06D2
:1017E0000B0061060A0057060B004C060A00420671
:1017F0000A0038060A002E060A0024060A001A0605
:101800000A001006090007060A00FD050900F40594
:101810000900EB050900E2050900D9050900D0051A
:101820000900C7050900BE050900B5050800AD059A
:101830000800A50509009C050800940508008C0512
:101840000800840508007C050800740508006C0584
:101850000700650508005D050700560508004E05F0
:101860000700470507004005080038050700310557
:1018700007002A050700230507001C0506001605BA
:1018800007000F0507000805060002050700FB0416
:101890000600F5040700EE040600E8040600E20472
:1018A0000700DB040600D5040600CF040600C904C7
:1018B0000600C3040600BD040600B7040600B10418
:1018C0000500AC040600A6040600A00405009B0465
:1018D000060095040500900406008A0405008504AE
:1018E0000500800406007A040500750405007004F4
:1018F00005006B04050066040500610405005C0436
:10190000050057040500520405004D040500480475
:101910000500430405003E0404003A0405003504B4
:101920000500300404002C040500270404002304EF
:1019300005001E0404001A04040016040500110426
:1019400004000D040400090405000404040000045C
:101950000400FC030400F8030400F4030400F00393
:101960000400EC030400E8030400E4030400E003C3
:101970000400DC030400D8030400D4030400D003F3
:101980000400CC030400C8030300C503030024F4CF
:1019900004D9201BC40C5C0E9804C4095F026507BF
:1019A0007101F405F900FB04B30048048700C1038A
:1019B00069005803550003034500BE023A00840243
:1019C000310053022A002902250004022000E4010C
:1019D0001C00C8011900AF01170098011400840110
:1019E0001300710110006101100051010E0043014C
:1019F0000D0036010B002B010B0020010B0015011F
:101A000009000C01090003010800FB000800F300B5
:101A10000800EB000700E4000600DE000600D80026
:101A20000600D2000600CC000500C7000500C20079
:101A30000500BD000400B9000400B5000400B100B9
:101A40000400AD000400A9000400A5000300A200EA
:101A500003009F0004009B00030098000300950012
:101A6000020093000300900003008D0002008B0031
:101A70000300880002008600020084000300810049
:101A800002007F0002007D0002007B00020079005E
:101A9000020077000100760002007400020072006C
:101AA0000100710002006F0002006D0001006C0077
:101AB00002006A0001006900020067000100660080
:101AC0000100650001006400020062000100610085
:101AD0000100600001005F0002005D0001005C0089
:101AE00001005B0001005A0001005900010058008C
:101AF000010057000100560001005500010054008C
:101B00000100530000005300010052000100510089
:101B10000100500001004F0001004E0000004E0087
:101B200001004D0001004C0001004B0000004B0083
:101B300001004A000100490001004800000048007F
:101B4000010047000100460000004600010045007A
:101B50000000450001004400010043000000430074
:101B6000010042000000420001004100000041006D
:101B70000100400001003F0000003F0001003E0066
:101B800000003E0001003D0000003D0001003C005F
:101B900000003C0000003C0001003B0000003B0056
:101BA00001003A0000003A0001003900000039004D
:101BB0000100380000003800000038000100370044
:101BC000000037000100360000003600000036003B
:101BD0000100350000003500000035000100340030
:101BE0000000340000003400010033000000330026
:101BF000000033000100320000003200000032001B
:101C0000010031000000310000003100010030000F
:101C1000000030000000300001002F0000002F0005
:101C200000002F0000002F0001002E0000002E00F9
:101C300000002E0001002D0000002D0000002D00EE
:101C400000002D0001002C0000002C0000002C00E2
:101C500000002C0001002B0000002B0000002B00D6
:101C600000002B0001002A0000002A0000002A00CA
:101C700000002A00010029000000290000002900BE
:101C800000002900000029000100280000002800B1
:101C900000002800000028000000280001002700A4
:101CA0000000270000002700000027000000270098
:101CB000010026000000260000002600000026008B
:101CC000000026000100250000002500000025007E
:101CD0000000250000002500000025000100240070
:101CE0000000240000002400000024000000240064
:101CF0000100230000002300000023000000230057
:101D00000000230000002300000023000100220047
:101D1000000022000000220000002200000022003B
:101D2000000022000100210000002100000021002D
:101D3000000021000000210000002100000021001F
:101D40000100200000002000000020000000200012
:101D50000000200000002000000020000000200003
:101D600001001F0000001F0000001F0000001F00F6
:101D700000001F0000001F0000001F0001001E00E7
:101D800000001E0000001E0000001E000000393090
:101D900000003325000087190000B00F0000DB08A9
:101DA0000000BD040000740200003F010000204359
:101DB0006F756E7420583A0023646566696E6520FD
:101DC00044454641554C545F0000626564004B64D5
:101DD00020004B6920004B70200050494420417581
:101DE000746F74756E652066696E697368656421C9
:101DF0002050757420746865206C617374204B707A
:101E00002C204B6920616E64204B6420636F6E73DD
:101E100074616E74732066726F6D2062656C6F778B
:101E200020696E746F20436F6E66696775726174A6
:101E3000696F6E2E680A00504944204175746F74B2
:101E4000756E65206661696C6564212074696D65D5
:101E50006F75740A00504944204175746F74756E33
:101E600065206661696C6564212054656D706572DA
:101E7000617475726520746F6F20686967680A0005
:101E8000504944204379636C6573002553202569CC
:101E90002F256900204B643A2000204B693A20002E
:101EA000204B703A200020436C61737369632050AB
:101EB0004944200A00204E6F206F76657273686F68
:101EC0006F740A002054753A2000204B753A2000A8
:101ED000206D61783A2000206D696E3A2000206400
:101EE0003A200020626961733A20005761697420CA
:101EF000666F7220686561742075702E2E2E0050FA
:101F00004944204175746F74756E652073746172F5
:101F1000740A00504944204175746F74756E6520D1
:101F20006661696C6564212054656D7065726174C9
:101F300075726520746F6F20686967680A00426572
:101F400064004531004500626564002C207379739C
:101F500074656D2073746F707065642120486561CD
:101F60007465725F49443A200048656174696E6720
:101F7000204661696C65640048656174696E67201C
:101F80006661696C6564004D313132205368757447
:101F9000646F776E001000C90210012C014001220D
:101FA0000170011801B0010E01F00104015002FAA4
:101FB00000B002F0003003E600D003DC009004D251
:101FC000007005C800A006BE000008B400B009AA51
:101FD00000D00BA000600E960060118C00001582EE
:101FE0000020197800C01D6E00A0226400B0275A9E
:101FF00000902C500000314600E0343C0010383294
:1020000000903A2800603C1E00A03D1400803E0A6B
:1020100000203F00004572723A204D415854454D12
:1020200050004D415854454D5020747269676765A2
:10203000726564004572723A204D494E54454D50C8
:10204000004D494E54454D50207472696767657262
:10205000656400544845524D414C2052554E4157FD
:10206000415900546865726D616C2052756E6177DC
:10207000617900202F002042403A0020403A0020A1
:10208000573A0020573A00496E76616C69642065C2
:10209000787472756465720A0000002100240027BC
:1020A000002A002D00300033000101000004010768
:1020B000010A017C3C3E5E2B3D3F2F5B5D3B2C2AA1
:1020C000225C0043616E6E6F74206F70656E2073CA
:1020D000756264697220004D6564696120496E69AA
:1020E00074204661696C0053442063617264206F00
:1020F0006B0A006F70656E526F6F74206661696C59
:1021000065640A00766F6C756D652E696E69742062
:102110006661696C65640A004E6F205344206361F8
:1021200072640A000A4D3234004D323320257300A8
:102130002E0A006F70656E206661696C65642C20E4
:1021400046696C653A200046696C652073656C656C
:10215000637465640A002053697A653A2000466911
:102160006C65206F70656E65643A2000454E4420B2
:10217000535542524F5554494E450A002220706F24
:1021800073002220706172656E743A2200535542CA
:10219000524F5554494E452043414C4C2074617276
:1021A0006765743A220053756263616C6C204F76E8
:1021B0006572666C6F770045786365656465642059
:1021C0006D617820535542524F5554494E45206415
:1021D000657074683A002E0A0044656C6574696F16
:1021E0006E206661696C65642C2046696C653A20D6
:1021F0000046696C652064656C657465643A0053DB
:1022000044207072696E74696E672062797465200B
:10221000004E6F74205344207072696E74696E674B
:102220000A002F6175746F25632E670057726974F9
:10223000696E6720746F2066696C653A200066726B
:1022400065736800646F696E67002066696C653A43
:1022500020004E6F7720002020506C616E6E6572FA
:1022600042756666657242797465733A200020464D
:10227000726565204D656D6F72793A200020436F5D
:102280006D70696C65643A20466562203230203298
:102290003032320A00204C617374205570646174CE
:1022A00065643A20323032322D30322D3035207C88
:1022B00020417574686F723A20426F6E6474656372
:1022C00068202F20496E73616E6974794175746F4F
:1022D0006D6174696F6E0A004D61726C696E2032B7
:1022E0002E302E395F4457372E342E350A002053B6
:1022F0006F6674776172652052657365740A002099
:102300005761746368646F672052657365740A006F
:102310002042726F776E206F7574205265736574FA
:102320000A002045787465726E616C205265736591
:10233000740A00506F77657255700A007374617289
:10234000740A004739310A47315A350A4739300A89
:102350004D38340A4D31303453300A4D3134305316
:1023600030004D31303031006572726F72207772FB
:102370006974696E6720746F2066696C650A004431
:102380006F6E6520736176696E672066696C652E75
:102390000A004D323900456E6473746F7073002506
:1023A0005320256320256320256320256300205AC0
:1023B0003A0020593A0020583A00656E6473746FF1
:1023C0007073206869743A200000002200250028FC
:1023D000002B002E0031003400020100000501082E
:1023E000010B01050505050705080808080202029A
:1023F000020A0A08080404040401010101010101A0
:10240000010303030303030303040707070C0C0C76
:102410000C0C0C0C0C02020202060606060606064E
:10242000060B0B0B0B0B0B0B0B01021020200808EB
:102430001020401020408002010201080402010126
:10244000020408102040808040201008040201800F
:102450000402018040201008040201080402010166
:10246000020408102040800102040810204080006F
:10247000000A0B02090C0D0E0807030401000000FE
:10248000000000000000000000000000000000004C
:102490000000000000000000000000121110000009
:1024A000000000000000000000000000000000002C
:1024B0000000000000FFFFFF50726F62696E67202E
:1024C0004661696C65640A0050726F62696E6720CC
:1024D0004661696C656400205A3A200020593A2010
:1024E0000042656420583A2000726573756D65641A
:1024F000004469736D69737300526573756D696E1D
:10250000670073686F770044697361626C65527528
:102510006E6F75740050757267654D6F726500500F
:10252000617573656400656E6400436F6E74696EF7
:102530007565004C6F61642046696C616D656E74F1
:102540002054004C6F61642046696C616D656E7447
:1025500000496E736572742066696C616D656E7496
:1025600020616E642073656E64204D3130380A003E
:1025700020204D323036205800486F6D65206F6640
:1025800066736574004361703A00434F4E46494795
:102590005F4558504F5254004D4541545041434BB4
:1025A00000434F4F4C45525F54454D5045524154A6
:1025B000555245004348414D4245525F54454D50A8
:1025C0004552415455524500424142595354455099
:1025D00050494E470041524353004D4F54494F4ECE
:1025E0005F4D4F44455300544845524D414C5F5058
:1025F000524F54454354494F4E00455854454E445C
:1026000045445F4D323000435553544F4D5F46496A
:10261000524D574152455F55504C4F4144004C4636
:102620004E5F5752495445004C4F4E475F46494C08
:10263000454E414D45004155544F5245504F52541F
:102640005F53445F5354415455530053445F5752B2
:10265000495445005245504541540053444341526A
:10266000440050524F4D50545F535550504F5254A8
:1026700000484F53545F414354494F4E5F434F4DC1
:102680004D414E445300454D455247454E43595FD9
:1026900050415253455200434153455F4C494748CE
:1026A000545F4252494748544E45535300544F4794
:1026B000474C455F4C494748545300534F46545785
:1026C0004152455F504F574552004255494C445F77
:1026D00050455243454E54004C4556454C494E4793
:1026E0005F44415441005A5F50524F424500525599
:1026F0004E4F5554004155544F4C4556454C005093
:1027000052494E545F4A4F420050524F4752455330
:1027100053004155544F5245504F52545F54454D0C
:1027200050004155544F5245504F52545F504F53F3
:1027300000564F4C554D4554524943004545505263
:102740004F4D0042494E4152595F46494C455F54F6
:1027500052414E534645520053455249414C5F58F1
:102760004F4E5F584F4646004649524D57415245DD
:102770005F4E414D453A4D61726C696E20322E308C
:102780002E395F4457372E342E3520544D33442094
:1027900053534D444E422028466562203230203249
:1027A0003032322031333A33383A31322920534FE4
:1027B000555243455F434F44455F55524C3A687408
:1027C0007470733A2F2F6769746875622E636F6D2A
:1027D0002F496E73616E6974794175746F6D6174A0
:1027E000696F6E2F4D61726C696E2F747265652F03
:1027F000437265616C6974794477696E5F322E301B
:102800002050524F544F434F4C5F56455253494FFF
:102810004E3A312E30204D414348494E455F545980
:1028200050453A544D3344203130532050726F207C
:1028300045585452554445525F434F554E543A31D2
:1028400020555549443A63656465326132662D34DA
:102850003161322D343734382D396231322D6335C0
:10286000356336326633363766660A00203B002011
:10287000204D3835312058005A2D50726F62652036
:102880004F66667365740043616E6E6F74206F707F
:10289000656E207375626469722000256973002576
:1028A000696D20256973002569682025696D2025DB
:1028B000697300256964202569682025696D2025D4
:1028C00069730025697920256964202569682025B8
:1028D000696D2025697300436F6F6C696E672E2EDA
:1028E0002E0048656174696E672E2E2E00453120DA
:1028F00025530042656420436F6F6C696E672E2E0E
:102900002E004265642048656174696E672E2E2E24
:10291000003D3D4477696E20496E697420436F6DB8
:10292000706C6574653D3D00202D2064342000648A
:10293000333A2000202D206432200064313A2000F8
:10294000202D206C656E20005650207265636569ED
:102950007665643A200077616974776179203D3D3E
:102960000020202A2A2A2A2A2A2A5254535F486100
:102970006E646C65446174612A2A2A2A2A2A2A2AEA
:1029800020002A2A2A4E6F7A7A6C6554656D70533E
:1029900074617475735B325D203D003D3D48656137
:1029A00074696E6720446F6E65204368616E676569
:1029B0002046696C616D656E743D3D002020737426
:1029C00061727470726F677265737320004D32327A
:1029D0000A4D3231003D3D77616974776179203568
:1029E0003D3D003D3D7761697477617920343D3D1F
:1029F000003D3D7761697477617920333D3D003D4D
:102A00003D7761697477617920313D3D00436F6E98
:102A10006669726D20436F6E74696E7565005061F2
:102A200075736553746174757300524553554D4504
:102A3000204F5054494F4E533A0048656174696EB7
:102A4000672E2E2E000000436C69636B20746F208C
:102A500068656174000000526573756D696E672E5C
:102A60002E2E00000050757267696E672E2E2E00A4
:102A70000000496E7365727420616E6420436C6956
:102A8000636B000000436C69636B20746F20636F9D
:102A90006E74696E7565000000456A656374696EE1
:102AA000672E2E2E000000506C65617365207761E3
:102AB00069742E2E2E0000005061726B696E672EB5
:102AC0002E2E0000002A2A2A496E6974696E67203A
:102AD00063617264206973204F4B2A2A2A003D3DAE
:102AE0006F6E5072696E7454696D657253746F7055
:102AF0007065643D3D003D3D6F6E55736572436F7B
:102B00006E6669726D52657175697265643D3D00EE
:102B10005061757365204D6F6465205374617475E1
:102B200073004C6F6164696E672E2E2E0000003DAD
:102B30003D6F6E466163746F727952657365743D63
:102B40003D00270A0A0000272027002027002D002B
:102B50006E6F74696669636174696F6E200063618A
:102B60006E63656C005072696E742041626F72749E
:102B700065640055492041626F7274656400726536
:102B800073756D65004D3234002A2A2A43506C61FA
:102B90007920546F6E652A2A2A003D3D6F6E50726F
:102BA000696E7454696D65725061757365643D3DFD
:102BB00000486F6D696E67204661696C6564006FDF
:102BC00070656E00545249474745524544003A20CB
:102BD0000066696C616D656E74007A5F6D696E0088
:102BE000795F6D696E00785F6D696E005265706F18
:102BF0007274696E6720656E6473746F702073748D
:102C0000617475730A0020746F6F206C6F6E67209B
:102C1000657874727573696F6E2070726576656E13
:102C20007465640A0020636F6C6420657874727543
:102C300073696F6E2070726576656E7465640A00E4
:102C4000486F6D652025732573257320466972735F
:102C500074005761726E696E673A20486F6D696ED5
:102C6000672042756D702044697669736F72203CED
:102C700020310A00020204000000000000000000F1
:102C800000000000809D4300009B430000C84300FB
:102C90000000410000004100000040000000010071
:102CA0000000010000800055555500000040003331
:102CB000333300AAAA2A004992240000002000C74A
:102CC000711C0099991900D1451700555515003B05
:102CD000B113002449120011111100000010000F5F
:102CE0000F0F00E3380E0043790D00CCCC0C00C36D
:102CF000300C00E8A20B0064210B00AAAA0A0070A5
:102D00003D0A009DD80900427B090092240900DC9D
:102D1000D30800888808001042080000000800F06E
:102D2000C107008787070075500700711C07003E28
:102D3000EB0600A1BC0600699006006666060070FE
:102D40003E06006118060017F4050074D105005B0B
:102D5000B00500B290050062720500555505007877
:102D6000390500B81E0500050505004EEC04008776
:102D7000D40400A1BD040090A7040049920400C13E
:102D80007D0400EE690400C7560400444404005C5E
:102D90003204000821040041100400000004003F38
:102DA000F00300F8E0030026D20300C3C30300CC05
:102DB000B503003AA803000A9B0300388E0300C045
:102DC0008103009F750300D0690300505E03001D5E
:102DD00053030034480300913D03003333030016CE
:102DE000290300381F030097150300300C0300036C
:102DF0000303000BFA020049F10200BAE802005C8A
:102E0000E002002DD802002DD0020059C80200B007
:102E1000C0020031B90200DAB10200AAAA0200A081
:102E2000A30200BC9C0200FA9502005C8F0200DF46
:102E300088020082820200457C0200277602002779
:102E4000700200436A02007C640200D05E02003F10
:102E5000590200C8530200FFFDFCFAF8F6F4F2F044
:102E6000EEECEAE9E7E5E3E1E0DEDCDAD9D7D5D458
:102E7000D2D0CFCDCBCAC8C7C5C3C2C0BFBDBCBAF4
:102E8000B9B7B6B4B3B2B0AFADACAAA9A8A6A5A461
:102E9000A2A1A09E9D9C9A99989795949392908FA9
:102EA0008E8D8B8A8988878684838281807F7E7DD0
:102EB0007B7A797877767574737271706F6E6D6CDA
:102EC0006B6A696867666564636261605F5E5D5CCA
:102ED0005B5A5958585756555453525150504F4EAB
:102EE0004D4C4B4A4A494847464645444342424175
:102EF000403F3E3E3D3C3B3B3A393838373635352E
:102F0000343332323130302F2E2E2D2C2B2B2A29D8
:102F10002928272726252524232322212120201F75
:102F20001E1E1D1C1C1B1B1A191918181716161506
:102F30001514131312121111100F0F0E0E0D0D0C8C
:102F40000C0B0A0A09090808070706060505040408
:102F5000030302020100003D3D6F6E5072696E7402
:102F600054696D6572537461727465643D3D00000F
:102F7000809D4300009B430000C843000000000008
:102F800000000000000000536176696E672044571E
:102F9000494E204C43442073657474696E67206603
:102FA000726F6D20454550524F4D0A003D3D6F6E8A
:102FB000436F6E66696775726174696F6E53746F83
:102FC00072655772697474656E3D3D005365747423
:102FD000696E67732053746F72656400290A00205C
:102FE00062797465733B2063726320005365747467
:102FF000696E67732053746F7265642028000A201D
:10300000696E6974207A70726F62655F7A6F666646
:10301000736574203D20003D3D6F6E436F6E6669A1
:103020006775726174696F6E53746F726552656112
:10303000643D3D00454550524F4D20496E697469CD
:10304000616C697A65640A0048617264636F6465E3
:10305000642044656661756C742053657474696E90
:103060006773204C6F616465640A0020286D6D29C8
:1030700000203B204C6576656C696E67200020203F
:103080004D3432302053004175746F204265642006
:103090004C6576656C696E6700203B2053656E73E6
:1030A0006F72200020440020204D34313220530024
:1030B00046696C616D656E742072756E6F757420F3
:1030C00073656E736F7200204A00202047323920EA
:1030D0005720490020204D3134392043203B2055D2
:1030E0006E69747320696E2043656C736975730A29
:1030F0000054656D706572617475726520556E69F6
:103100007473002020473231203B004C696E6561AA
:103110007220556E6974730070012C0190012701B3
:10312000B0012201C0011D01F001180110021301BC
:1031300030020E016002090190020401C002FF008A
:103140000003FA004003F5008003F000D003EB0019
:103150002004E6007004E100E004DC004005D70034
:10316000C005D2004006CD00D006C8008007C300CD
:103170003008BE00F008B900C009B400B00AAF00C2
:10318000B00BAA00D00CA500000EA000500F9B00B1
:10319000C01096005012910000148C00C0158700DA
:1031A000B0178200B0197D00D01B7800001E73009C
:1031B00040206E0090226900F024640040275F00E8
:1031C00090295A00E02B5500102E500020304B0063
:1031D00010324600E033410090353C001037370094
:1031E00070383200A0392D00B03A2800A03B2300EF
:1031F000603C1E00103D1900903D1400103E0F0071
:10320000703E0A00C03E0500003F0000403FFBFF4B
:10321000803FF6FFC03FF1FF220A00556E6B6E6FD4
:10322000776E20636F6D6D616E643A2022002042DC
:10323000002050006F6B00204500205A00205900EC
:1032400020204D393220580053746570732070650A
:103250007220756E69740020746F6F206C6F6E67DA
:1032600020657874727573696F6E2070726576650B
:103270006E7465640A0020636F6C642065787472F4
:103280007573696F6E2070726576656E7465640A19
:10329000004D323520500A4D323400526573756D41
:1032A000650055492050617573650043616E6E6F0E
:1032B0007420656E746572207375626469723A2059
:1032C000004E6F204D61746368203A00436F6E7347
:1032D000747261696E206D65736856616C20006D53
:1032E00065736856616C200079506E7420007850C8
:1032F0006E7420006D657368506F696E74200044B1
:103300006973706C61794272696768746E65737312
:10331000205365743A2000446973706C617942727D
:10332000696768746E657373204C43443A20004D9E
:1033300032320A4D32310052656672657368005050
:10334000675570005067446F776E00497320466977
:103350006C6520004973204469722000476F5570E6
:1033600044697200486173204D6564696100466973
:103370006C656E616D652053656C65637465640092
:103380004D3130303043004D31303030002046690F
:103390006C616D656E7420526573706F6E7365201D
:1033A0004E6F00526573756D6520596573206475A5
:1033B00072696E67207072696E74000A204E6F2009
:1033C00046696C616D656E7400496E76616C696406
:1033D000204F7074696F6E004D3530300053746F3C
:1033E00072652053657474696E6773004D3939399D
:1033F0000A4D32383050305331363000424C546F21
:10340000756368205265736574004D3530320A4D1E
:1034100035303000496E697420454550524F4D009B
:103420004D3530300053746F726520536574746984
:103430006E677300496E4C616E6743686F696365C0
:10344000000A202A2A2A7265636461742E646174FA
:10345000615B305D203D004732380A4731204631FC
:10346000303030205A313000556E737570706F7285
:10347000746564204F7074696F6E2053656C65636A
:10348000746564004D32313153300A4739310A478F
:10349000315A302E3032350A4739300A4D32313107
:1034A0005331004D32313153300A4739310A4731F7
:1034B0005A2D302E3032350A4739300A4D323131EB
:1034C00053310047323953320047323953310047C4
:1034D000323652323535004D3139305335350A47A1
:1034E00032380A4732390A4D3430300A4D313034DF
:1034F000533231350A4732380A4D3130395332317F
:10350000350A4D34323053310A4731583130305951
:1035100031303046353030300A47315A300A4D3577
:1035200030300A4D31313720536574205A204F66B0
:1035300066736574004731204631303030205A3090
:103540002E30004732380A473120463130303020A3
:103550005A302E30005A204F6666736574203A2028
:103560002573005A204F6666736574203A202573D0
:10357000004732385A0A473146313530305A302EFA
:1035800030004732380A473146313530305A302E14
:103590003000426564204C6576656C204F7074691C
:1035A0006F6E200052657475726E203A20004D389F
:1035B0003400473146313030305A302E30004732F7
:1035C000380A473146313030305A302E30004D61A4
:1035D0006E75616C53657454656D70005A204F664A
:1035E00066736574203A20257300526F756E6469A6
:1035F0006E6720746F207374657000526571756515
:1036000073746564204F6666736574200053746F2D
:1036100070205472696767657265640053746F70D7
:10362000204E6F0053746F705072696E7400486161
:103630006E646C6520446174612041646A757374C2
:1036400020322053657474696E6720536372656518
:103650006E200048616E646C652044617461205086
:1036600072696E7446696C652033205365747469A1
:103670006E672053637265656E200048616E646CEE
:10368000652044617461205072696E7446696C658E
:1036900020322053657474696E67205363726565C8
:1036A0006E20004D38340048616E646C65204461C2
:1036B0007461205072696E7446696C6520506F7336
:1036C000740048616E646C652044617461205072BE
:1036D000696E7446696C6520507265004265676961
:1036E0006E537769746368003D3D20436865636B82
:1036F0006B65793D3D007265636461742E6164643D
:1037000072203D3D007265636461742E6461746172
:103710005B305D203D3D0020453A00205A3A0020B4
:10372000593A00583A006F6B0A00526573656E642F
:103730003A2000544D3344203130532050726F20D2
:1037400052656164792E005072696E74696E672EDD
:103750002E2E005072696E7420506175736564007E
:103760006E6F74696669636174696F6E200052459B
:1037700053554D45204F5054494F4E533A004865DC
:103780006174696E672E2E2E000000436C69636BB6
:1037900020746F2068656174000000526573756D58
:1037A000696E672E2E2E00000050757267696E6775
:1037B0002E2E2E0000004C6F6164696E672E2E2E37
:1037C000000000496E7365727420616E6420436C62
:1037D00069636B000000436C69636B20746F206346
:1037E0006F6E74696E7565000000456A6563746983
:1037F0006E672E2E2E000000506C65617365207779
:103800006169742E2E2E0000005061726B696E6724
:103810002E2E2E00000050617573654D73673D00BC
:103820008401040111241FBECFEFD1E2DEBFCDBF62
:1038300000E00CBF84B780936A1814BE0FB6F894EA
:10384000A89580916000886180936000109260006C
:103850000FBE16E0A0E0B2E0ECEEFBE702E00BBF2B
:1038600002C007900D92A032B107D9F728E1A0E27B
:10387000B6E001C01D92AA36B207E1F71CE1C1E132
:10388000DCE100E006C021970109802FFE010F94C2
:10389000233AC031D10780E00807A9F70F94E1254A
:1038A0000D94E43D0C94000020912507833021F411
:1038B00025FD0CC024FD0CC030E0A90102C05595C7
:1038C00047958A95E2F7CA018170089581E00895CD
:1038D00080E008958091E00984FD0BC08091E209A9
:1038E00087FD07C09091E309937081E019F480E0AF
:1038F000089581E00895CF92DF92EF92FF92CF93E7
:10390000DF93EC01CC80DD80EE80FF8027E137EB98
:1039100041ED58EBC701B6010F948C3C87FD23C0E5
:1039200023E030E04BE953E4C701B6010F945C3368
:103930001816CCF0C880D980EA80FB8027E137EBED
:1039400041ED58EBC701B6010F948C3C87FD0BC0CD
:10395000C1E023E030E84DE953E4C701B6010F941C
:103960005C3318160CF4C0E08C2FDF91CF91FF90E0
:10397000EF90DF90CF900895269A2E9A08952F9277
:103980003F924F925F926F927F928F929F92AF92EF
:10399000BF92CF92DF92EF92FF920F931F93CF933C
:1039A000DF93CDB7DEB760970FB6F894DEBF0FBEDA
:1039B000CDBF8B876C87042F122F282F30E03E87D6
:1039C0002D87462F50E05A87498785E0982E929E92
:1039D000C001939E900D1124988B8F87FA01E80FF8
:1039E000F91FEE0FFF1FEE0FFF1FE15EF14F608129
:1039F0007181828193819B01AC010F941E3D8823CC
:103A000009F445C14B85400F6C85610F949EC00140
:103A10001124E985FA85E80FF91FEE0FFF1FEE0F5D
:103A2000FF1FE15EF14FC080D180E280F380040F80
:103A3000909EA0011124E985FA85E40FF51FEE0F91
:103A4000FF1FEE0FFF1FE15EF14F0081918082802A
:103A50007380262F30E0EF85F889E20FF31FEE0F19
:103A6000FF1FEE0FFF1FE15EF14F20807181798310
:103A700072817A8373817B83610F70E0EF85F889AF
:103A8000E60FF71FEE0FFF1FEE0FFF1FE15EF14F76
:103A9000F88BEF87F081FC83EF85F889F181FD8356
:103AA000EF85F889F281FE83EF85F889F381FF8342
:103AB000FC01E20FF31FEE0FFF1FEE0FFF1FE15E91
:103AC000F14F20812887A180B2806380FA01E60F40
:103AD000F71FEE0FFF1FEE0FFF1FE15EF14F40805B
:103AE000518032801381202F392D482D572D602F82
:103AF000792D882D972D0F941E3D882321F000E00D
:103B0000912C812C712C9601A701B601C7010F944D
:103B10001E3D882321F0C02ED92CE82CF72C2C81B7
:103B20003D814E815F816C817D818E819F810F946B
:103B30001E3D882321F01C821D821E821F82222DA1
:103B400039814A815B81622D79818A819B810F94C1
:103B50001E3D882339F02C803D8139834E814A8374
:103B60005F815B839201432D512FB201832D912FF1
:103B70000F941E3D882321F0412C512C312C10E054
:103B800028853A2D4B2D562D68857A2D8B2D962D17
:103B90000F941E3D882321F04886A52CB32C612E5E
:103BA00085E02D853E85829FF001839FF00D1124D5
:103BB00049855A85E40FF51FEE0FFF1FEE0FFF1F1B
:103BC000E15EF14FFA87E9879601A701B601C701C7
:103BD0000F942C3A202F392D482D572D0F942B3A26
:103BE0006B017C01222D39814A815B81622D7981B3
:103BF0008A819B810F942C3A2C813D814E815F817B
:103C00000F942B3A9B01AC01C701B6010F942C3ADB
:103C10006B017C0128853A2D4B2D562D68857A2D18
:103C20008B2D962D0F942C3A9201432D512F0F94EA
:103C30002B3A9B01AC01C701B6010F942C3A20E04E
:103C400030E040E450E40F94263BE985FA85608338
:103C50007183828393836C858B8560960FB6F8940D
:103C6000DEBF0FBECDBFDF91CF911F910F91FF90AF
:103C7000EF90DF90CF90BF90AF909F908F907F900C
:103C80006F905F904F903F902F900D94D207609669
:103C90000FB6F894DEBF0FBECDBFDF91CF911F915D
:103CA0000F91FF90EF90DF90CF90BF90AF909F90DB
:103CB0008F907F906F905F904F903F902F900895DE
:103CC0000F931F93CF93DF9300D01F92CDB7DEB732
:103CD0009C0103E119E090E1E8EAFEE0D8010190DF
:103CE0000D929A95E1F7F90120813181428153814A
:103CF000F80160857185828593850F942C3AF801CF
:103D0000608771878287938780E090E0A0EAB0E4C3
:103D100089839A83AB83BC83CE0101960E9441BF05
:103D20000F900F900F900F90DF91CF911F910F91F7
:103D300008952F923F924F925F926F927F928F924F
:103D40009F92AF92BF92CF92DF92EF92FF921F931A
:103D5000CF93DF93CDB7DEB72C970FB6F894DEBFC5
:103D60000FBECDBF7A011901DC012D913D914D911E
:103D70005C912D833E834F835887FB0140805180A7
:103D8000628073808090A80E9090A90EA090AA0ED9
:103D9000B090AB0EA50194016D817E818F819885D5
:103DA0000F945C3381110EC011E0A3019201609168
:103DB000AC0E7091AD0E8091AE0E9091AF0E0F943F
:103DC0005C33811110E0D1012D913D914D915C91B9
:103DD00029873A874B875C87F701C080D180E280D2
:103DE000F38020910C0230910D0240910E0250910F
:103DF0000F02C701B6010F945C33882309F44EC04B
:103E0000C0920C02D0920D02E0920E02F0920F02CC
:103E10008091B40E9091B50EA091B60EB091B70EF0
:103E20004091AC0E5091AD0E6091AE0E7091AF0E00
:103E30008092130990921409A0921509B092160964
:103E400040931709509318096093190970931A0940
:103E5000C0921B09D0921C09E0921D09F0921E0924
:103E600080931F0990932009A0932109B093220900
:103E700020E030E040E05FE36091BE0D7091BF0D47
:103E80008091C00D9091C10D0F94C23369837A83E4
:103E90008B839C83CE0101960E9441BF2D813E8180
:103EA0004F815885209313093093140940931509C5
:103EB00050931609409217095092180960921909F7
:103EC00070921A09D1012D913D914D915C916091B3
:103ED0001F097091200980912109909122090F9466
:103EE0002C3A60931F0970932009809321099093C5
:103EF000220911112FC020E030E0A90169857A85DF
:103F00008B859C850F945C33811133C060E070E039
:103F100088EC92E469837A838B839C83CE0101963B
:103F20000E9441BF2C960FB6F894DEBF0FBECDBFE6
:103F3000DF91CF911F91FF90EF90DF90CF90BF90D6
:103F4000AF909F908F907F906F905F904F903F9039
:103F50002F9008952AEF3EE74AE25FE36091C20D99
:103F60007091C30D8091C40D9091C50D0F94C23313
:103F7000D1CF60E070E080EA91E4CCCFCF93DF93C3
:103F800000D01F92CDB7DEB780E090E0A0EAB0E4A9
:103F900089839A83AB83BC8361E0CE0101960E9442
:103FA000ACC00F900F900F900F90DF91CF910895BC
:103FB0008091140790911507009731F04AE050E086
:103FC00070E060E00D94773160E070E0CB0108951F
:103FD0000F931F93CF93DF9300D000D01F921F92B7
:103FE000CDB7DEB78B01FC0123A5211102C00E94D1
:103FF000B6761D821E821F82188620E030E040E0E7
:104000005FE36091B00E7091B10E8091B20E90910D
:10401000B30E0F942C3A69837A838B839C839E0121
:104020002B5F3F4FAE014F5F5F4F6CEA7EE088EA47
:104030009EE00E94991E1D821E821F82188620E02B
:1040400030E040E05FE3F80160857185828593850B
:104050000F942C3A69837A838B839C83B8016C5FBD
:104060007F4F9E012B5F3F4FAE014F5F5F4FC801F7
:104070000E94991E28960FB6F894DEBF0FBECDBFE2
:10408000DF91CF911F910F91089580911407909126
:104090001507009731F04AE050E070E060E00D94C1
:1040A000493060E070E0CB0108950E94452097FD03
:1040B0000CC00E9445206F3F71058105910509F0F4
:1040C00034F40E944520862F089580E008958FEFF4
:1040D00008958091140790911507892B41F00E9453
:1040E000552091E0811101C090E0892F089591E061
:1040F000FCCFFC0165917591859194910895809113
:104100005E08882319F080E00E9436C380E008959D
:104110008F929F92AF92BF92CF92DF92EF92FF92D7
:10412000CF93DF93EC018090870A9090880AA0904B
:10413000890AB0908A0A20E030E0A901C501B401E3
:104140000F945C33882309F454C0C880D980EA8076
:10415000FB80A7019601C501B4010F945C331816CA
:104160000CF04CC020917F0A3091800A4091810A66
:104170005091820AC701B6010F945C33882331F154
:10418000C0927F0AD092800AE092810AF092820A5D
:104190002091830A3091840A4091850A5091860AC1
:1041A000688179818A819B810F94C2339B01AC0124
:1041B00060E070E080E89FE30F942B3A6093100278
:1041C0007093110280931202909313026091100277
:1041D000709111028091120290911302DF91CF91A0
:1041E000FF90EF90DF90CF90BF90AF909F908F9017
:1041F000089560E070E080E89FE3F0CF60E070E059
:10420000CB01ECCF682F70E090E080E00C94F7F0E9
:104210009B01AC01485F5F4FBC016C5F7F4F0C940A
:10422000991E2F923F924F925F926F927F928F9240
:104230009F92AF92BF92CF92DF92EF92FF920F9335
:104240001F93CF93DF93CDB7DEB7A6970FB6F89441
:10425000DEBF0FBECDBF8C011B015A87498740903E
:10426000A80E5090A90E6090AA0E7090AB0E809090
:10427000AC0E9090AD0EA090AE0EB090AF0EDB01E4
:104280008D919D910D90BC91A02D8B8B9C8BAD8BB6
:10429000BE8B9C01AD01C301B2010F942B3A6B019F
:1042A0007C01D10114968D919D910D90BC91A02D12
:1042B0008F8B988FA98FBA8F9C01AD01C501B40176
:1042C0000F942B3A6B8F7C8F8D8F9E8FA985BA852B
:1042D0008D919D910D90BC91A02D8B879C87AD8772
:1042E000BE879C01AD01C301B2010F942B3A6F8FC1
:1042F00078A389A39AA3A985BA8514968D919D91D7
:104300000D90BC91A02D8F87988BA98BBA8B9C01A7
:10431000AD01C501B4010F942B3A6BA37CA38DA30F
:104320009EA3A7019601C701B6010F94C2336B018A
:104330007C012B8D3C8D4D8D5E8DCA01B9010F9492
:10434000C2339B01AC01C701B6010F942C3A4B015B
:104350005C012B893C894D895E896B857C858D85C7
:104360009E850F942B3A2B013C012F89388D498D66
:104370005A8D6F85788989899A890F942B3A6B01B8
:104380007C01A3019201C301B2010F94C2332B013E
:104390003C01A7019601C701B6010F94C2339B01EE
:1043A000AC01C301B2010F942C3A0F94DA3C6B01BB
:1043B0007C012F8D38A149A15AA1CA01B9010F94DE
:1043C000C2332B013C012BA13CA14DA15EA1CA012E
:1043D000B9010F94C2339B01AC01C301B2010F9428
:1043E0002C3A9B01AC01C501B4010F948C3C18160A
:1043F000B4F520E030E0A901C701B6010F948C3C70
:1044000087FF2AC0C701B601905820E030E040EA9B
:1044100050E40F948C3C181614F5A10169857A8537
:10442000C8010E941121A6960FB6F894DEBF0FBEF8
:10443000CDBFDF91CF911F910F91FF90EF90DF9053
:10444000CF90BF90AF909F908F907F906F905F9034
:104450004F903F902F900895C701B601D6CF20E02E
:1044600030E040E050E4C501B4010F948C3C1816D4
:1044700024F4B101C8010E94E81F19821A821B822C
:104480001C82BE016F5F7F4FC1010E9408212DEC8D
:104490003CEC4CEC5CE3C701B6010F94C2339B01CA
:1044A000AC01F80160817181828193810F94C233E4
:1044B0006D837E838F839887D8019B968C919B9781
:1044C0008823C9F02AE939E949E95FE314966D9137
:1044D0007D918D919C9117970F94C23369837A8354
:1044E0008B839C83BE016F5F7F4F83E199E00E94C5
:1044F0000821F80113A6BE016B5F7F4F89859A855D
:104500000E94082190CF3F924F925F926F927F92CC
:104510008F929F92AF92BF92CF92DF92EF92FF92D3
:104520000F931F93CF93DF93CDB7DEB76C970FB682
:10453000F894DEBF0FBECDBFDB010C91142F100F1E
:10454000153008F05FC11196DC90C22ECD0CB4E09E
:10455000BC1508F457C1ED2DF0E0E55FF84FE081A0
:10456000F0E0002E02C0F595E7950A94E2F7E0FF2F
:1045700049C1EC2DF0E0E55FF84FE081F0E0012E5D
:1045800002C0F595E7950A94E2F7E0FF3BC1322EB1
:10459000642F7C01409035075090360760903707B4
:1045A0007090380780913D0790913E07A0913F079A
:1045B000B0914007898F9A8FAB8FBC8F660F770BB6
:1045C000072E000C880B990B0F9463334B015C0191
:1045D000602F000F770B880B990B0F946333298D95
:1045E0003A8D4B8D5C8D0F94C233A30192010F94D1
:1045F0002C3AA50194010F942C3A6D877E878F8702
:10460000988B612F110F770B880B990B0F946333E5
:10461000298D3A8D4B8D5C8D0F94C233A30192018D
:104620000F942C3AA50194010F942B3A69837A8355
:104630008B839C834090390750903A0760903B07EA
:1046400070903C078091410790914207A0914307E9
:10465000B0914407898F9A8FAB8FBC8F632D660F03
:10466000770B072E000C880B990B0F9463334B01CB
:104670005C016D2DDD0C770B880B990B0F94633368
:10468000298D3A8D4B8D5C8D0F94C233A30192011D
:104690000F942C3AA50194010F942C3A698B7A8BD4
:1046A0008B8B9C8B6C2DCC0C770B880B990B0F9400
:1046B0006333298D3A8D4B8D5C8D0F94C233A301EA
:1046C00092010F942C3AA50194010F942B3A6D831B
:1046D0007E838F839887F70180859185A285B38536
:1046E00089879A87AB87BC878D8B9E8BAF8BB88F62
:1046F00045E351E061E070E0CE0141960E94E78F12
:1047000045E351E061E070E0CE0105960E94E78F3D
:104710004AE351E061E070E0CE010D960E94E78F20
:104720004AE351E061E070E0CE0101960E94E78F1C
:1047300089889A88AB88BC8827E137EB41ED58EB34
:10474000C501B4010F948C3C87FD5CC023E030E0D0
:104750004BE953E4C501B4010F945C3318160CF413
:1047600051C08D849E84AF84B88827E137EB41ED3A
:1047700058EBC501B4010F948C3C87FD43C023E086
:1047800030E84DE953E4C501B4010F945C331816C9
:10479000CCF18D809E80AF80B88427E137EB41ED6E
:1047A00058EBC501B4010F948C3C87FD2BC023E06E
:1047B00030E04BE953E4C501B4010F945C331816A3
:1047C0000CF189809A80AB80BC8027E137EB41ED0A
:1047D00058EBC501B4010F948C3C87FD13C023E056
:1047E00030E84DE953E4C501B4010F945C33181669
:1047F0004CF0AE014F5F5F4FBE01635F7F4FC7015B
:104800000E9411216C960FB6F894DEBF0FBECDBF8B
:10481000DF91CF911F910F91FF90EF90DF90CF909C
:10482000BF90AF909F908F907F906F905F904F90D0
:104830003F9008950E944520CB0108950F931F9348
:10484000CF9380911407909115070097E9F0FC0130
:104850008F01C1912C2F2F7D81F0C53411F0C53609
:10486000B9F7F801108270E060E00F94EB2EF801C8
:10487000C083CF911F910F91089570E060E0CF91B8
:104880001F910F910D94EB2E60E070E0CB01F1CF02
:104890002FEB280F2A3108F047C0E22FF0E080917B
:1048A000E0099091E109A091E209B091E30904C007
:1048B000B695A795979587952A95D2F780FD02C062
:1048C00081700895EA53F64FE081EE2341F1809123
:1048D000790A90917A0AE80FF92FF11D808190ED05
:1048E000980F9A3030F08E3251F4818180538A30A3
:1048F00098F4F0931507E093140781E008958D3242
:1049000011F08B3249F4818190ED980F9A3088F341
:104910008E3211F48281EACFF0E0E0E0EACF10922B
:10492000150710921407E9CF80E008950E944824EB
:10493000882341F081E02091140730911507232B43
:1049400009F480E00895CF92DF92EF92FF926A011E
:104950007B010E949624882331F0FF90EF90DF9036
:10496000CF900C941E24C701B601FF90EF90DF900A
:10497000CF900895CF93DF93EB010E949624882374
:1049800021F0DF91CF910C941A24CE01DF91CF91C9
:104990000895CF93DF93EB010E949624882319F0AA
:1049A0000E944520EB01CE01DF91CF910895CF9376
:1049B000C62F0E949624882319F0CF910C9455207D
:1049C0008C2FCF910895CF93DF93C82FD62F0E94BD
:1049D0009624882321F0DF91CF910C9469208C2FAD
:1049E0000E944824811101C08D2FDF91CF9108953D
:1049F000CF92DF92EF92FF92CF936B017C01C42F95
:104A000080915F088F5F09F4BEC080935F0880913A
:104A10005F0880930E0980E1E8EAFEE0A0E6B8E0D6
:104A200001900D928A95E1F720E030E040E752E4F2
:104A30006091340270913502809136029091370274
:104A40000F94C2330F949F3B70937108609370086A
:104A5000C0927208D0927308E0927408F0927508C0
:104A600080910D09C0FB80F980930D098CE0E0E195
:104A7000F8E0A6E7B8E001900D928A95E1F78CE0A6
:104A8000E2E3FAE0A2E8B8E001900D928A95E1F73E
:104A90008091340790910D0980FB94F990930D0952
:104AA000882381F08091300790913107A0913207DF
:104AB000B091330780938E0890938F08A09390084D
:104AC000B09391088091621390916313909393082F
:104AD0008093920880914B1390914C13909395087A
:104AE000809394088091A00A8093960880910D0984
:104AF0009091DA0D90FB83F980930D098091870ADC
:104B00009091880AA091890AB0918A0A80939708A7
:104B100090939808A0939908B0939A080E944DC565
:104B2000609308097093090980930A0990930B090F
:104B30008091250780930C0990917B0D80910D0940
:104B400093FB81F990913F0A90FB82F980930D09C4
:104B500080E00E94A2AA40E050E0BA0181E796E11D
:104B60000E94D17F40EB50E06FE578E081E796E16D
:104B70000E94658081E796E1CF91FF90EF90DF90F2
:104B8000CF900C94928381E040CF4F925F926F92CE
:104B90007F928F929F92AF92BF92CF92DF92EF92CD
:104BA000FF921F93CF93DF9300D01F92CDB7DEB754
:104BB00019821A821B821C82CE0101964C0183E16C
:104BC000C82E89E0D82E98EAE92E9EE0F92E28EB2F
:104BD000A22E2EE0B22E10E088E5810F0E949624CE
:104BE000F40181934F01882309F4E7C00E941E2439
:104BF0002B013C01812F0E94541C882309F4D3C04F
:104C0000F7012081318142815381C301B2010F94A8
:104C10002C3AF60160837183828393831F5FF4E0F3
:104C2000CF0ED11C84E0E80EF11C94E0A90EB11C5B
:104C3000133091F685E40E9496248C83882309F42E
:104C4000C7C00E941E246B017C0183E00E94541C9B
:104C5000882371F02091B40E3091B50E4091B60EBC
:104C60005091B70EC701B6010F942C3A6B017C012D
:104C7000C0921F09D0922009E0922109F0922209E6
:104C80008091900D882391F180916C1682FF2EC047
:104C900087FD2CC08C81882349F18981811103C053
:104CA0008A81882319F12DEC3CEC4CE45DE36091A2
:104CB00068087091690880916A0890916B080F9458
:104CC0002C3A9B01AC016091B00E7091B10E8091B5
:104CD000B20E9091B30E0F948C3C18163CF440E049
:104CE00060E070E080E090E40E94F82440E050E052
:104CF000BA0186E40E94A32420E030E0A9010F94C9
:104D00008C3C181684F40E941E2420E030E040E71A
:104D100052E40F94263B60933402709335028093E3
:104D200036029093370280917B0D83FD28C08091DD
:104D3000FC07882321F12091B40E3091B50E4091EB
:104D4000B60E5091B70E60911F09709120098091A5
:104D50002109909122090F942B3A20910908309152
:104D60000A0840910B0850910C080F942C3A60935C
:104D7000090870930A0880930B0890930C080F9011
:104D80000F900F900F90DF91CF911F91FF90EF90B8
:104D9000DF90CF90BF90AF909F908F907F906F905B
:104DA0005F904F900895F5012081318142815381B8
:104DB000C301B2010F942B3A2CCFF701808191816E
:104DC000A281B381F60180839183A283B38326CF2E
:104DD0008091B40E9091B50EA091B60EB091B70E21
:104DE00080931F0990932009A0932109B093220971
:104DF00047CFEFE5F8E080EBDF011D928A95E9F7F8
:104E000008958091900D811104C00E94F9260C94A0
:104E10002EAB80916C1682FF09C087FD07C040E071
:104E200060E070E080E090E40C94F82408958091B4
:104E30005F08882361F090910E09891308C0809162
:104E40006C1684FF04C08BE998E00C94428780E0E4
:104E50000895FC01238121110C9492830895CF932E
:104E6000DF93C0916213D0916313209729F1609171
:104E70005E1370915F1380916013909161130F9492
:104E8000983B6E5F7F4F24976C177D07ACF470934F
:104E9000800760937F070E94D877605A75418F4FD3
:104EA0009F4F60938107709382078093830790934D
:104EB0008407DF91CF9108951092810710928207A5
:104EC0001092830710928407F4CFCF92DF92EF9273
:104ED000FF921F93CF93DF93182F662351F0109208
:104EE0000A071092060710920707109208071092FF
:104EF00009070E94D8776B017C0180910607909189
:104F00000707A0910807B0910907A7019601281B80
:104F1000390B4A0B5B0BDA01C901B7FD3DC020918B
:104F20000A0717FD13C0412F012E000C550B4C5FD3
:104F30005F4F822F022E000C990B4817590764F11E
:104F400084EF91E0A0E0B0E0211724F488EE93E034
:104F5000A0E0B0E08C0D9D1DAE1DBF1D8093060727
:104F600090930707A0930807B09309072170C22FF9
:104F700030E0D32F84E28C9FB0018D9F700D7C1B9D
:104F8000112460597C4F82E390E00E9466C98091B1
:104F90000A078F5F80930A07DF91CF911F91FF90DF
:104FA000EF90DF90CF900895CF93DF93C0914B1394
:104FB000D0914C13209729F16091471370914813B9
:104FC0008091491390914A130F94983B6E5F7F4FE5
:104FD00024976C177D07ACF470937807609377077C
:104FE0000E94D877605E70448D4F9F4F6093790721
:104FF00070937A0780937B0790937C07DF91CF9122
:1050000008951092790710927A0710927B071092F8
:105010007C07F4CFCF93C1E020E030E0A90160919C
:105020003D0770913E0780913F07909140070F9494
:105030005C33811101C0C0E08C2FCF9108954F9255
:105040005F926F927F928F929F92AF92BF92CF9218
:10505000DF92EF92FF920F931F93CF93DF93EC01B8
:105060002091350730913607409137075091380726
:10507000688179818A819B810F942B3A6B017C0135
:105080002091390730913A0740913B0750913C07F6
:105090006C817D818E819F810F942B3A4B015C0145
:1050A000A7019601609104027091050280910602A9
:1050B000909107020F945C33882309F450C0C0928A
:1050C0000402D0920502E0920602F09207022091BB
:1050D000FE063091FF064091000750910107C7017D
:1050E000B6010F94C2332B013C010F94CE3B6B01F0
:1050F0007C0120E030E0A9010F945C3387FD70C093
:1051000020E030E040E450E4C701B6010F948C3C4D
:1051100018162CF4C12CD12CC0E4EC2EFE2CA701C7
:105120009601C301B2010F942B3A6093F606709377
:10513000F7068093F8069093F906C701B6010F941D
:10514000983B6093F406062E000C770B6F5F7F4F41
:105150006430710514F064E070E06093F206D09161
:1051600002021091F406A501940160910802709169
:10517000090280910A0290910B020F945C33811115
:1051800033C0D11381C02091DA063091DB06409103
:10519000DC065091DD066091F6067091F70680916D
:1051A000F8069091F9060F94C2332091DE063091F3
:1051B000DF064091E0065091E1060F942C3ADF9112
:1051C000CF911F910F91FF90EF90DF90CF90BF9004
:1051D000AF909F908F907F906F905F904F900895C9
:1051E000C12CD12C76019BCF8092080290920902AB
:1051F000A0920A02B0920B0220910207309103079D
:105200004091040750910507C501B4010F94C233C2
:105210004B015C010F94CE3B6B017C0120E030E040
:10522000A9010F945C3387FDF3C020E030E040E437
:1052300050E4C701B6010F948C3C18162CF4C12C15
:10524000D12CB0E4EB2EFE2CA7019601C501B401D0
:105250000F942B3A6093FA067093FB068093FC063A
:105260009093FD06C701B6010F94983B6093F50635
:10527000062E000C770B6F5F7F4F6430710514F0C2
:1052800064E070E06093F306C091F506D11305C0A9
:10529000809103028C1709F470C08091F4069091FC
:1052A000F50690930302809302020C2E000CDD0B96
:1052B00025E01203C0011124FC01EC0FFD1FEE0FCD
:1052C000FF1FEE0FFF1FE15EF14F20813181428110
:1052D00053812093EE063093EF064093F0065093EF
:1052E000F1060091F306002E000C110BFC01E00FFB
:1052F000F11FEE0FFF1FEE0FFF1FE15EF14F608108
:105300007181828193810F942B3A6093EA067093A6
:10531000EB068093EC069093ED062091F20635E0C3
:105320002303F0011124CE0FDF1FCC0FDD1FCC0FA4
:10533000DD1FC15ED14F288139814A815B81209375
:10534000E6063093E7064093E8065093E906E00F3F
:10535000F11FEE0FFF1FEE0FFF1FE15EF14F6081A7
:105360007181828193810F942B3A6093E20670934E
:10537000E3068093E4069093E5068090FA06909009
:10538000FB06A090FC06B090FD062091EA06309145
:10539000EB064091EC065091ED06C501B4010F9467
:1053A000C2332091EE063091EF064091F006509105
:1053B000F1060F942C3A6B017C01C092DE06D0926C
:1053C000DF06E092E006F092E1062091E2063091DD
:1053D000E3064091E4065091E506C501B4010F943F
:1053E000C2332091E6063091E7064091E8065091DD
:1053F000E9060F942C3AA70196010F942B3A60937B
:10540000DA067093DB068093DC069093DD06BBCE54
:10541000C12CD12C760118CF1F93CF93DF93CDB73A
:10542000DEB72C970FB6F894DEBF0FBECDBF182F96
:10543000882321F00E940A288823F9F08091DA0D50
:105440008117D9F00E94A8B68CE0E7E7F2E0DE0110
:10545000119601900D928A95E1F7CE0101960E9476
:105460001F288091DA0D882391F088EA9EE00E943F
:10547000CBB61092DA0D0E94B8C12C960FB6F894F4
:10548000DEBF0FBECDBFDF91CF911F91089581E0A8
:105490008093DA0D88EA9EE00E94D4B5ECCF8F921B
:1054A0009F92AF92BF92EF92FF920F931F93CF9371
:1054B000DF9380E00E940C2A1092390710923A077D
:1054C00010923B0710923C07109235071092360756
:1054D0001092370710923807109241071092420736
:1054E000109243071092440710923D0710923E0716
:1054F00010923F07109240070FE11EE0C0E0812CA0
:10550000912C80ECA82E8FE7B82E7801D0E0F7011F
:1055100081929192A192B1927F016D2F8C2F0F9465
:10552000D207DF5FD53099F7CF5F0C5E1F4FC530D4
:1055300061F7DF91CF911F910F91FF90EF90BF9096
:10554000AF909F908F9008958F929F92AF92BF924D
:10555000CF92DF92EF92FF92C0903D07D0903E072E
:10556000E0903F07F090400720E030E0A901C7013C
:10557000B6010F945C338823E1F1A701960160E046
:1055800070E080E89FE30F94263B6B017C018090E4
:10559000410790904207A0904307B090440720E055
:1055A00030E0A901C501B4010F945C33882329F1CF
:1055B000A501940160E070E080E89FE30F94263B32
:1055C000C092FE06D092FF06E0920007F09201071B
:1055D0006093020770930307809304079093050775
:1055E000FF90EF90DF90CF90BF90AF909F908F9003
:1055F0000895C12CD12C7601CACF60E070E0CB01B8
:10560000DFCFEFE6F0E080818260808308958091B3
:10561000851390918613892B79F48091851390914D
:105620008613892B49F4209185133091861381E0EC
:10563000232B19F480E0089581E00895CF92DF9242
:10564000EF92FF926B017C0183E3C816D104E10461
:10565000F10470F082E3C81AD108E108F10862E3AE
:1056600070E080E090E00E94A5770E942990ECCF46
:10567000C701B6010E94A577FF90EF90DF90CF9011
:105680000C94299010923D0980911B0290911C026C
:10569000A0911D02B0911E02809351079093520772
:1056A000A0935307B093540708959091C913109293
:1056B000C9139230B9F09430C1F09130E1F48823ED
:1056C00019F0813021F008959093DB0D089582E068
:1056D0008093DB0D80913D09882369F01092680268
:1056E0000C94422B1092DC0D089585E89BE2909378
:1056F0001E0E80931D0E089590916C1694FB8827C2
:1057000080F994FF06C081E09091D317911101C0F8
:1057100080E008950E947C2B882339F080916C16DC
:1057200082FB882780F991E08927089580911209EA
:10573000811106C080918713823011F00C948A2B5E
:1057400081E008950C943DC881E00895CF93DF93E4
:10575000EC01E62F660FFF0BE159FB4DE491E2509F
:10576000E13108F0B0C0F0E08827E654F44D8F4FE7
:105770000D94233ACB2B632C632C632C632CF52BD9
:10578000D72B192C172CF72B3D2C3B2C1B2C632CC7
:10579000612C5F2C3F2C82E1E3E8F2E0DE01019016
:1057A0000D928A95E1F7CE01DF91CF91089581E0C6
:1057B00020EB30E03983288321EB30E03B832A83E0
:1057C0001D821C8223EB30E03F832E8324EB30E0EC
:1057D000398728871B861A861D861C8692E09E873D
:1057E0008F8781E0888B198ADECF80E0E1CF81E06E
:1057F0008F5F20E930E03983288321E930E03B8363
:105800002A8322E930E03D832C8328E930E03F837E
:105810002E832AE930E0398728872CE930E03B875E
:105820002A8726E930E03D872C8793E0D8CF80E0B7
:10583000DFCF80E0DECF81E08F5F20EA30E0398388
:10584000288321EA30E03B832A8322EA30E03D834B
:105850002C8328EA30E03F832E832AEA30E0398720
:1058600028872CEA30E03B872A8726EA30E03D870C
:105870002C8794E0B4CF80E0DFCF80E0DECF81E002
:105880008F5F20E231E03983288321E231E03B83DE
:105890002A8322E231E03D832C8328E231E03F83FA
:1058A0002E832AE231E0398728872CE231E03B87DA
:1058B0002A8726E231E03D872C8795E090CF80E073
:1058C000DFCF80E0DECF82E1FE0111928A95E9F719
:1058D0006ACF8F929F92AF92BF92CF92DF92EF9258
:1058E000FF920F93CF93DF931F92CDB7DEB75C018A
:1058F0007B0149016B01C40ED51EF50180819181A8
:105900000F947A398983002311F0F7018083BE0157
:105910006F5F7F4FC4010E9419F0F5018081918172
:10592000019691838083FFEFEF1AFF0AEC14FD04C8
:1059300021F780E00F90DF91CF910F91FF90EF90D2
:10594000DF90CF90BF90AF909F908F9008959091EF
:10595000D10095FD0CC09091D00095FF08C08093B8
:10596000D6008091D00080648093D000089520916B
:1059700036062F5F2F770FB607FC27C090913706AA
:10598000921328C09091D00095FF1EC090913706C9
:1059900040913606941306C09091D1009F7D90935C
:1059A000D10012C0E92FF0E0EA5CF94F32819F5F2D
:1059B0009F773093D600909337063091D0003064B3
:1059C0003093D000491741F3D9CF90913706921305
:1059D00001C0FBCFE0913606F0E0EA5CF94F82832C
:1059E000209336068091D10080628093D100089583
:1059F0008091EB099091EC092FEF3FEF981751F050
:105A0000E92FF0E0E551F64F228130E09F5F9F7370
:105A10009093EC09C90108951F920F920FB60F924F
:105A200011240BB60F922F938F939F93EF93FF93B5
:105A30008091370620913606821306C08091D100EE
:105A40008F7D8093D10012C0E82FF0E0EA5CF94F1F
:105A500092818F5F8F779093D600809337069091D5
:105A6000D00090649093D000281741F3FF91EF91FC
:105A70009F918F912F910F900BBE0F900FBE0F90A3
:105A80001F9018951F920F920FB60F9211240BB60C
:105A90000F920F931F932F933F934F935F936F93A7
:105AA0007F938F939F93AF93BF93CF93DF93EF93A6
:105AB000FF93C091D6000091EC09D091EB0911E061
:105AC0001D0F1F7390913506913108F09FC0E92F8B
:105AD000F0E08827E159F24D8F4F0D94233A802D45
:105AE000AF2DBE2DCD2DD42D062ED82D062EDC2D7E
:105AF000E02D062EE42DE82DEC2DF32D062EFE2DA7
:105B0000C03229F028F5CA3011F0CD3031F5011737
:105B100031F0ED2FF0E0E551F64FC283D12FD09355
:105B2000EB09FF91EF91DF91CF91BF91AF919F91E1
:105B30008F917F916F915F914F913F912F911F9125
:105B40000F910F900BBE0F900FBE0F901F901895E6
:105B5000CD3481F081E0CE3471F080E10CC0CA33E5
:105B600038F4C033A0F6C03291F2CD32B1F7CFCFC6
:105B7000CD3499F782E080933506C9CFC13359F00F
:105B800018F4C03221F2E9CF88E0C433A1F38BE0EE
:105B9000C83389F3E2CF83E0EECF84E0C03359F31A
:105BA00086E0C13341F3D9CF85E0C833B1F6E3CF06
:105BB00087E0C23391F6DFCF89E0C13371F6DBCFE6
:105BC0008AE0C03351F6D7CF8CE0C73331F6D3CF5C
:105BD0008DE0C63311F6CFCFC03209F498CF8EE0F6
:105BE000C33549F2BACF80ED8C0F8A3008F08FCFE1
:105BF0009FE0909335068093340689CFCA3019F020
:105C0000CD3009F084CF1092350681CFCA3019F01B
:105C1000CD3009F07CCF809160168823A1F39730B6
:105C200089F038F4953079F7109233021092DC0D38
:105C3000EACF9A3059F09F3031F7809134060E94B4
:105C4000552BE1CF81E080937E07DDCF81E080930B
:105C50007D07D9CF9091C00095FFFCCF8093C600FF
:105C60000895CF93DF93EC01FE0184912196882360
:105C700019F00E942A2EF8CFDF91CF910895CF928C
:105C8000DF92EF92FF926A017B010E94312E42E087
:105C9000C701B601FF90EF90DF90CF900C94FE8784
:105CA0000E943F2E8AE00C942A2ECF93DF9369EE58
:105CB0007EE00F949C08C3E4D3E14B855C856D8541
:105CC0007E8580EE9EE00E943F2E2CEA35EC47E276
:105CD0005EE36F85788989899A890F94263BAB01A9
:105CE000BC018DED9EE00E943F2E2CEA35EC47E290
:105CF0005EE36B897C898D899E890F94C233AB01E9
:105D0000BC018AED9EE0DF91CF910C94502ECF9391
:105D1000DF9367E47EE00F949C086091A20D709180
:105D2000A30D8091A40D9091A50D0F946133AB014B
:105D3000BC018EE39EE00E943F2E4091D20D509117
:105D4000D30D6091D40D7091D50D8BE39EE00E9430
:105D50003F2E4091D60D5091D70D6091D80D709186
:105D6000D90D88E39EE00E943F2EC0E8DDE0488127
:105D700059816A817B8181EF9EE00E943F2E4C8198
:105D80005D816E817F818DE392E30E943F2E488585
:105D900059856A857B858AE392E30E943F2E4C8574
:105DA0005D856E857F8587E392E3DF91CF910C94CB
:105DB000502ECF93DF936CEB7DE00F949C08C2E9EB
:105DC000DDE04CA95DA96EA97FA983EB9DE00E944F
:105DD0003F2E48AD59AD6AAD7BAD80EB9DE00E9492
:105DE0003F2E4CAD5DAD6EAD7FAD88E39EE0DF91A3
:105DF000CF910C94502ECF93DF9368E97DE00F9400
:105E00009C08C2E9DDE04CA15DA16EA17FA18FE8F5
:105E10009DE00E943F2E48A559A56AA57BA58DE36C
:105E200092E30E943F2E4CA55DA56EA57FA58AE357
:105E300092E30E943F2E48A959A96AA97BA987E34A
:105E400092E3DF91CF910C94502ECF93DF9363E7D1
:105E50007DE00F949C08C2E9DDE0688179818A8148
:105E60009B810F946133AB01BC018AE69DE00E94E7
:105E70003F2E6C817D818E819F810F946133AB01B8
:105E8000BC018DE392E30E943F2E688579858A8567
:105E90009B850F946133AB01BC018AE392E30E94BE
:105EA0003F2E6C857D858E859F850F946133AB0178
:105EB000BC0187E392E3DF91CF910C94502ECF93F6
:105EC0008091E009827161F48091E2098C7841F45B
:105ED0008091E309837021F481E0CF910C94872EA7
:105EE00082E40E949624882351F00E94D81F609378
:105EF000A20D7093A30D8093A40D9093A50D83E53F
:105F00000E949624882351F00E941E246093D20D93
:105F10007093D30D8093D40D9093D50D84E50E949A
:105F20009624882351F00E941E246093D60D70930E
:105F3000D70D8093D80D9093D90D88E50E949624B3
:105F4000882351F00E941E246093800D7093810D70
:105F50008093820D9093830D89E50E949624882377
:105F600051F00E941E246093840D7093850D8093E0
:105F7000860D9093870D8AE50E949624C82F88236A
:105F800051F00E941E246093880D7093890D8093B8
:105F90008A0D90938B0D85E40E949624882351F0FE
:105FA0000E941E2460938C0D70938D0D80938E0D36
:105FB00090938F0DCC23A9F02DEC3CEC4CEC5DE3E1
:105FC0006091880D7091890D80918A0D90918B0D53
:105FD0000F945C3318162CF086E09EE0CF910C9461
:105FE000312ECF910895AF92BF92CF92DF92EF9270
:105FF0000F931F93CF93DF935B01EA01690188231D
:1060000009F463C088E39DE00E94312EF5016081B0
:1060100071818281938146E00E94FE87E1100BC06E
:106020008FE29DE00E94312E688179818A819B8177
:1060300046E00E94FE8788E29DE00E94312EF60134
:10604000608171818281938143E00E94FE8781E2B9
:106050009DE00E94312EF8016081718182819381DF
:1060600043E00E94FE8788E19DE00E94312EF60108
:106070002081318142815381F80160817181828167
:1060800093810F942B3A43E00E94FE87EE20F9F0B3
:106090008AE00E942A2E83E09DE00E94312E6881D2
:1060A00079818A819B8146E00E94FE878AE00E9476
:1060B0002A2E8AE0DF91CF911F910F91EF90DF9010
:1060C000CF90BF90AF900C942A2EE110E4CFDF91D7
:1060D000CF911F910F91EF90DF90CF90BF90AF9035
:1060E00008952F923F924F925F926F927F928F927C
:1060F0009F92AF92BF92CF92DF92EF92FF920F9357
:106100001F93CF93DF93CDB7DEB7C155D1090FB63B
:10611000F894DEBF0FBECDBF2DB73EB73BAF2AAF61
:1061200087E00E946FDE81110BC061E086E50E946E
:10613000D7248DA3853060F08EED9CE00E94312E37
:10614000EAADFBAD0FB6F894FEBF0FBEEDBF56C370
:106150003DA1332321F08EEB9CE00E94312E6AE0BA
:1061600080E50E94D724182F8CEF810F8F3218F012
:106170008AE99CE0E3CF60E085E40E94E324882381
:1061800009F448C081E089AFE0909614F09097142C
:10619000D7012D913D914D915C916091A80E709128
:1061A000A90E8091AA0E9091AB0E0F942C3AAB01E0
:1061B000BC0188E50E94A32469877A878B879C8726
:1061C000F70124813581468157816091AC0E709131
:1061D000AD0E8091AE0E9091AF0E0F942C3AAB01A4
:1061E000BC0189E50E94A3246D877E878F87988BE9
:1061F000BE01635F7F4FCE0109960E94D372382E95
:1062000081110BC063E686E89CE00E941BCA8EE603
:106210009CE094CF93E099AFB7CF8CE40E944824E0
:10622000082F882309F43CC10E9455208EA3803199
:1062300018F087E49CE082CFFEA1F13009F432C16E
:1062400060E083E50E94E3248CAF882321F00111F4
:1062500002C037E03EA38DA1833020F08DE29CE0A8
:106260000E94312E9091DA0D9FAF80E00E940C2A9F
:106270000E9422BF1D8A1E8A1F8A188E198E1A8EAE
:106280001B8E1C8E83EF9FE4A3ECB7E48D8F9E8F53
:10629000AF8FB8A383EF9FE4A3ECB7EC89A39AA3D5
:1062A000ABA3BCA3A12FB0E0BCABABABEDB7FEB7CB
:1062B00024E0129FE019F10911240FB6F894FEBFF3
:1062C0000FBEEDBF8DB79EB701969EAF8DAF2DA1CE
:1062D00049ADBE01635F7F4FCE0109960E940574F0
:1062E0009B01AC010F941E3D811178C20E94D877AA
:1062F000611571058105910511F00F94E22E212C95
:106300001DAA1EAA1FAA18AEAEA1A150BB0B2E96A5
:10631000BFAFAEAF2E97812F90E0B0E0A0E06296C5
:106320008CAF9DAFAEAFBFAF6297A22DB0E0BCA760
:10633000ABA7EBA9FCA9AE17BF070CF080C2119662
:10634000B8A7AFA3FF93EF93BF93AF9389E19CE00E
:106350009F938F9383E29CE09F938F931F920E9461
:1063600096F62DB73EB7275F3F4F0FB6F8943EBF66
:106370000FBE2DBF3EA1332309F455C10F94932EB8
:106380002AE030E040E050E00F94C2390F946333CC
:1063900020E030E040EA50E40F948C3C0FEF1FEF18
:1063A000181614F001E010E00F94932E28E631E067
:1063B00040E050E00F94C2390F9463332B013C014D
:1063C0000F94932E20E230E040E050E00F94C23969
:1063D0006B5F7F4F8F4F9F4F0F9463334B015C0177
:1063E0008DA18430D1F4B501A4018BE09CE00E9422
:1063F0003F2EB301A20183E09CE00E943F2E8DEF6F
:106400009BE00E94312E0130110519F483E40E94B3
:106410002A2E89EF9BE00E94312E312CC801110FEA
:10642000AA0BBB0B2C968CAF9DAFAEAFBFAF2C971A
:106430002E96AEADBFAD2E973A161B060CF0F3C0EC
:106440002C966CAD7DAD8EAD9FAD2C970F946333C4
:106450006B017C01BCADBB2341F1AC019B010F94EE
:106460002C3A20E030E040E952E40F94C2339B0123
:10647000AC01C301B2010F942C3A2B013C0120E086
:1064800030E044EB53E40F948C3C1816FCF420E00D
:1064900030E044EB53E4C301B2010F942B3AEDCF4B
:1064A0001EA2CECE22E02EA3CBCE0F94932E24E1BB
:1064B00030E040E050E00F94C239675E7F4F8F4F6D
:1064C0009F4F0F946333A7019601CFCF20E030E0B8
:1064D000A901C301B2010F945C3387FF0BC020E018
:1064E00030E044EB53E4C301B2010F942C3A2B018A
:1064F0003C01ECCF0091961410919714F80124817F
:106500003581468157816D857E858F8598890F9469
:106510002B3A24966CAF7DAF8EAF9FAF24972BEDB7
:106520003FE049E450E4C301B2010F94C23320E0DC
:1065300030E044E353E40F94263B6B017C010F945D
:10654000213B6FA778AB89AB9AABD8012D913D91D8
:106550004D915C9169857A858B859C850F942B3A4A
:1065600028966CAF7DAF8EAF9FAF2897A5019401A1
:106570006FA578A989A99AA90F94C2339B01AC0190
:1065800028966CAD7DAD8EAD9FAD28970F942C3ABB
:1065900069837A838B839C83C701B6010F94CC3CBB
:1065A000A50194010F94C23324962CAD3DAD4EADA0
:1065B0005FAD24970F942C3A6D837E838F839887E9
:1065C0004BE351E070E060E0CE0101960E94E78F5E
:1065D00046E351E070E060E0CE0105960E94E78F4F
:1065E000BDA1B43081F449815A816B817C818DEEEB
:1065F0009BE00E943F2E4D815E816F8178858DE307
:1066000092E30E94502E198A1A8A1B8A1C8AAE01B4
:106610004F5E5F4FBE016B5F7F4FCE0101960E94C0
:106620006BC0339405CF20E049ADBE01635F7F4F5F
:10663000CE0109960E9405744B015C01312CAC011E
:106640009B010F941E3D811102C033243394A50198
:106650009401C501B4010F941E3D8111F0C0EBA55A
:10666000FCA5EE0FFF1FEE0FFF1F2DAD3EADE20F9D
:10667000F31F80829182A282B382A50194016D8D65
:106680007E8D8F8D98A10F948C3C181624F48D8EDE
:106690009E8EAF8EB8A2A501940169A17AA18BA1AB
:1066A0009CA10F945C3387FF04C089A29AA2ABA27D
:1066B000BCA2A50194016DA97EA98FA998AD0F94E4
:1066C0002C3A6DAB7EAB8FAB98AF8FA198A5092EFE
:1066D000000CAA0BBB0B8FA398A7A9A7BAA7BC0154
:1066E000CD010F9463336BA77CA78DA79EA79B0159
:1066F000AC016DA97EA98FA998AD0F94263B2B0103
:106700003C014D8A5E8A6F8A788EADADBEADB8AB66
:10671000AFA710E0C12CD12C7601EFA5F8A96191AB
:10672000719181919191F8ABEFA7A30192010F9420
:106730002B3A9B01AC010F94C2339B01AC01C70102
:10674000B6010F942C3A6B017C011F5F211628F7CC
:106750002BA53CA54DA55EA50F94263B0F94DA3CD6
:10676000698F7A8F8B8F9C8FFDA1F230A8F16FA17A
:1067700078A589A59AA50E94F7F088EE9BE00E9473
:10678000312E62966CAD7DAD8EAD9FAD62970E944D
:10679000F7F082EE9BE00E94312E43E0C501B40188
:1067A0000E94FE8780E20E942A2E81E02DA12330E4
:1067B0000CF480E0E12C8E010F5D1F4F9E01235EE3
:1067C0003F4FAE01475E5F4FBE016B5E7F4F0E9441
:1067D000F32F8AE00E942A2E2394A7CD0E947F20C7
:1067E0000E9409BF8FAD0E940C2A0E94BAC1AAADB7
:1067F000BBAD0FB6F894BEBF0FBEADBF2AAD3BAD6B
:106800000FB6F8943EBF0FBE2DBFCF5ADF4F0FB665
:10681000F894DEBF0FBECDBFDF91CF911F910F91D6
:10682000FF90EF90DF90CF90BF90AF909F908F90B0
:106830007F906F905F904F903F902F9008950E94AF
:106840007F20332069F287ED9BE00E94312E81E0AA
:106850003DA113160CF080E0EE24E3948E010F5D51
:106860001F4F9E01235E3F4FAE01475E5F4FBE014B
:106870006B5E7F4F0E94F32F698D7A8D8B8D9C8D7F
:106880000052110926E042E00F94292E9F938F9326
:1068900086EC9BE09F938F9380ED9BE09F938F937B
:1068A0001F920E9496F68DB79EB707960FB6F89482
:1068B0009EBF0FBE8DBF94CF0F931F93CF93209198
:1068C0005F16222389F0C62F8C0187EA97E00E9489
:1068D000312EC8010E94312ECC2331F08AE0CF91B5
:1068E0001F910F910C942A2ECF911F910F91089513
:1068F0000F931F93CF9320915F16222391F0C62F01
:106900008C0160E081EB97E00E945C34C8010E943A
:10691000312ECC2331F08AE0CF911F910F910C944E
:106920002A2ECF911F910F9108950F931F93CF930C
:10693000DF93D82F8B01C42F61E086E295E20E949D
:106940007834D093C91380915F168823B9F060E042
:1069500080EC97E00E94783480E20E942A2EC801E1
:106960000E94312ECC2319F08C2F0E942A2E8AE00F
:10697000DF91CF911F910F910C942A2EDF91CF912F
:106980001F910F910895CF93DF9320915F162223DB
:1069900089F0EC0160E089EB97E00E94783480E2B6
:1069A0000E942A2ECE010E94312E8AE0DF91CF91E3
:1069B0000C942A2EDF91CF9108950F931F93CF93BC
:1069C000DF938A01E90190915F16992319F040E065
:1069D0000E9495340115110519F0C8010E94C334B5
:1069E000209719F0CE010E94C33461E082E095E265
:1069F000DF91CF911F910F910C947834811107C0D2
:106A000083E492E10E94312E8AE00C942A2E87E4DE
:106A100092E1F8CFCF936AEF7FE00F949C08C0918A
:106A2000900DC05D81EF9FE00E94312E8C2F0E945F
:106A30002A2E8DEE9FE00E94312E8091900DCF91F5
:106A40000C94FE344F925F926F927F928F929F923E
:106A5000AF92BF92CF92DF92EF92FF92CF93DF93EC
:106A6000CDB7DEB72C970FB6F894DEBF0FBECDBF03
:106A700083E50E9448248823C9F00E9469208093FE
:106A800046022C960FB6F894DEBF0FBECDBFDF9145
:106A9000CF91FF90EF90DF90CF90BF90AF909F90FD
:106AA0008F907F906F905F904F90089580914602F5
:106AB000805D89838AE09FE00E94312E89810E9457
:106AC0002A2E86E09FE00E94312E809146020E948D
:106AD000FE344090B80E5090B90E6090BA0E70908F
:106AE000BB0E209148023091490240914A025091D8
:106AF0004B02C301B2010F942C3A69837A838B83D2
:106B00009C838090BC0E9090BD0EA090BE0EB09065
:106B1000BF0E20914C0230914D0240914E02509197
:106B20004F02C501B4010F942C3A6D837E838F838D
:106B30009887C090C00ED090C10EE090C20EF09029
:106B4000C30E209150023091510240915202509157
:106B50005302C701B6010F942C3A69877A878B8755
:106B60009C872091540230915502409156025091D9
:106B70005702C301B2010F942C3A2B013C01209122
:106B800058023091590240915A0250915B02C5015E
:106B9000B4010F942C3A4B015C0120915C023091BE
:106BA0005D0240915E0250915F02C701B6010F94F1
:106BB0002C3A6B017C018EEF9EE00E94312E4981C0
:106BC0005A816B817C8181EF9EE00E943F2E4D8136
:106BD0005E816F8178858DE392E30E943F2E498527
:106BE0005A856B857C858AE392E30E943F2E8CEF69
:106BF0009EE00E94312E84EF9EE00E94312EB30170
:106C0000A20181EF9EE00E943F2EB501A4018DE319
:106C100092E30E943F2EB701A6018AE392E30E940D
:106C20003F2E8AE02C960FB6F894DEBF0FBECDBF84
:106C3000DF91CF91FF90EF90DF90CF90BF90AF901A
:106C40009F908F907F906F905F904F900C942A2E22
:106C500087E897E00C94312E81E897E00C94312E70
:106C6000CF9384E50E949624C0E0882309F10E9416
:106C70005520C82F1816E4F40E942C368DE40E948B
:106C80002A2E6091E5097091E60990E080E00E946B
:106C90008DF081E190E10E94312E6C2FCC0F770BAB
:106CA000880B990B0E94F7F08AE00E942A2ECFEF02
:106CB0008C2FCF9108950F931F93CF93811116C0FE
:106CC000C42F8B010E942C368EE090E10E94312E61
:106CD000C8010E94312ECC2349F08AE30E942A2E5B
:106CE0008AE0CF911F910F910C942A2ECF911F9182
:106CF0000F910895CF93C82F41E06FEC7EE00E9482
:106D00005B36C11102C00E942C3640916513509130
:106D10006613609167137091681386EC9EE00E9481
:106D20003F2E2CEA35EC47E25EE3609169137091E7
:106D30006A1380916B1390916C130F94263BAB01F7
:106D4000BC0183EC9EE00E943F2E2CEA35EC47E22A
:106D50005EE360916D1370916E1380916F1390914B
:106D600070130F94C233AB01BC0180EC9EE00E9413
:106D70003F2E8AE0CF910C942A2ECF93811112C01E
:106D800040E068E57DE00E945B3680913407811128
:106D900004C08BE49DE00E94312E8AE00E942A2EDE
:106DA0000E942C36C091340782E49DE00E94312E6F
:106DB0008C2F0E9402214091300750913107609141
:106DC0003207709133078FE39DE0CF910C94502EE2
:106DD000CF93C82F82E0C11184E060E00E9479F275
:106DE0000E942C3687ED97E0CC2311F08CEE97E0D3
:106DF000CF910C94312ECF93DF93EB010E94312E73
:106E0000BE01DD0F880B990BDF91CF910C94F7F049
:106E10005F926F927F928F929F92AF92BF92CF922A
:106E2000DF92EF92FF920F931F93CF93DF931F9206
:106E3000CDB7DEB77C0139018B015B01A40EB51E15
:106E4000D12CC12CA016B10609F450C0F7018080E6
:106E50009180F80151908F015982C4010F947A39C1
:106E60005816B9F1652DC4010F948239FFEFCF1A7E
:106E7000DF0AC6018F779927892B21F162E070E044
:106E800080E090E00E94A577C4010F947A3999813F
:106E90008917F9F00E942C3687EC94E00E94312E7D
:106EA00081E00F90DF91CF911F910F91FF90EF90B4
:106EB000DF90CF90BF90AF909F908F907F906F901A
:106EC0005F90089562E070E080E090E00E941E2BE9
:106ED000DBCFBE016F5F7F4FC3010E9419F0F70146
:106EE00080819181019691838083ACCF80E0D9CF5E
:106EF0000E94312E8AE00C942A2E2F923F924F92BC
:106F00005F926F927F928F929F92AF92BF92CF9239
:106F1000DF92EF92FF920F931F93CF93DF93CDB742
:106F2000DEB7C659D1090FB6F894DEBF0FBECDBF8C
:106F30000E9417278823F1F18091E0099091E109DF
:106F4000A091E209B091E309AC01BD0132E176956F
:106F50006795579547953A95D1F740FF45C087ED1E
:106F60009FE00E9478378EEF80932E0A10922D0AB0
:106F700081E09AE59093EE158093ED158CE490E016
:106F80009093F0158093EF1587E08093E11582E8E8
:106F90008093E41584E890E0A0E0B0E08093E515EC
:106FA0009093E615A093E715B093E81581E995E174
:106FB0000E9473C7CA56DF4F0FB6F894DEBF0FBEEC
:106FC000CDBFDF91CF911F910F91FF90EF90DF9098
:106FD000CF90BF90AF909F908F907F906F905F9079
:106FE0004F903F902F90089522E0B695A7959795E2
:106FF00087952A95D1F780FF0CC00E94F9260E9440
:107000002EAB81E0809362160E9479870E949DCF0B
:10701000D1CF409004095090050960900609709006
:10702000070980910D0981FF05C090917B0D986043
:1070300090937B0D82FB882780F980933F0A8CEC2C
:107040009FE00E94DCDD80919408909195089E015C
:107050002F5F3F4F7901009799F09F938F9384ECB6
:107060009FE09F938F933F932F930F94F332C70129
:107070000E94AEDD0F900F900F900F900F900F9029
:107080008091920890919308843B910514F484EBCD
:1070900090E09F938F938CEB9FE09F938F93FF9251
:1070A000EF920F94F332C7010E94AEDD9091680811
:1070B000CF56DF4F9883C159D04020916908CE56F2
:1070C000DF4F2883C259D04030916A08CD56DF4F38
:1070D0003883C359D04080916B08CC56DF4F8883EA
:1070E000C459D040209172083091730840917408BF
:1070F00050917508692FCE56DF4F7881C259D04024
:10710000CD56DF4F8881C359D040CC56DF4F988190
:10711000C459D0400F942C3A962E872E382E292E03
:1071200084EB9FE00E94DCDD80910D090F900F90B1
:107130000F900F900F900F9080FDD8C1CF56DF4F6A
:10714000A880C159D040CE56DF4FB880C259D04038
:10715000CD56DF4FC880C359D040CC56DF4FD880C2
:10716000C459D0408E010F571F4F23E041E0B501B5
:10717000C6010F94292E9F938F938BEA9FE09F93D4
:107180008F93FF92EF920F94F332C7010E94AEDD0E
:107190000F900F900F900F900F900F909501A601F8
:1071A000692D782D832D922D0F948C3C1816FCF4AC
:1071B00023E041E0692D782D832D922D0F94292E07
:1071C0009F938F9381EA9FE09F938F93FF92EF921B
:1071D0000F94F332C7010E94AEDD0F900F900F9015
:1071E0000F900F900F90A92CB82CC32CD22C89E9AA
:1071F0009FE00E94DCDD87E08093910D80933E0A42
:1072000060919708709198088091990890919A08D8
:107210008E010F571F4F21E041E00F94292E9F93BD
:107220008F9380910D0983FB882780F9CB56DF4F20
:107230008883C559D040CA56DF4F1882C659D040FE
:10724000CB56DF4F88819981C559D040C0969F9316
:107250008F938EE89FE09F938F93FF92EF920F940E
:10726000F332C7010E94AEDD21E041E0B501C60165
:107270000F94292E9F938F9385E89FE09F938F9380
:10728000FF92EF920F94F332C7010E94AEDD80911E
:107290000D090FB6F894DEBF0FBECDBF84FF1FC02F
:1072A00060918E0870918F0880919008909191085C
:1072B00023E041E00F94292E9F938F938DE79FE069
:1072C0009F938F93FF92EF920F94F332C7010E9426
:1072D000AEDD0F900F900F900F900F900F90809158
:1072E000920890919308009799F09F938F9385E768
:1072F0009FE09F938F93FF92EF920F94F332C70119
:107300000E94AEDD0F900F900F900F900F900F9096
:10731000809196088823A1F01F928F931F921F924D
:107320008AE69FE09F938F93FF92EF920F94F33240
:10733000C7010E94AEDD0FB6F894DEBF0FBECDBF11
:107340006091640870916508809166089091670863
:107350008E010F581F4F23E041E00F94292ED82EA5
:10736000C92E6091600870916108809162089091C7
:107370006308005F1F4F23E041E00F94292ECF9256
:10738000DF929F938F938CE59FE09F938F93FF9263
:10739000EF920F94F332C7010E94AEDD23E041E08B
:1073A000CF56DF4F6881C159D040CE56DF4F78812C
:1073B000C259D040CD56DF4F8881C359D040CC56FA
:1073C000DF4F9881C459D0400F94292E9F938F93FB
:1073D00082E59FE09F938F93FF92EF920F94F33299
:1073E000C7010E94AEDD809171088F938091700873
:1073F0008F938CE49FE09F938F93FF92EF920F9473
:10740000F332C7010E94AEDD60916C0870916D0887
:1074100080916E0890916F0823E041E00F94292E2F
:107420009F938F9383E49FE09F938F93FF92EF92BC
:107430000F94F332C7010E94AEDD8CE0E6E7F8E07E
:10744000A0E1B8E001900D928A95E1F78CE0E2E8C6
:10745000F8E0A2E3BAE001900D928A95E1F780E0AE
:107460000E9498BB81E00E9498BB82E00E9498BB7A
:1074700080910C098093250781E08093900D0E94F4
:1074800001278BE998E09F938F9389E291E29F9384
:107490008F93FF92EF920F94F3320FB6F894DEBF02
:1074A0000FBECDBFC7010E94AEDD80910B098F9347
:1074B00080910A098F93809109098F93809108091F
:1074C0008F937F926F925F924F9287E39FE09F939B
:1074D0008F93FF92EF920F94F332C7010E94AEDDBB
:1074E0000FB6F894DEBF0FBECDBF64CDA92CB82C6B
:1074F000C32CD22C37CECF93C82F41E062E27FE07D
:107500000E945B36C11102C00E942C3640912C07AC
:1075100050912D0760912E0770912F0789E19FE010
:107520000E943F2E409128075091290760912A0719
:1075300070912B0786E19FE00E943F2E83E19FE040
:107540000E94312E8BE690E3CF910C947837CF9345
:10755000DF93CDB7DEB7A8970FB6F894DEBF0FBEA6
:10756000CDBF8C017B01942E0E94448D0115110525
:1075700009F4C8C00E942C36C8010E947837E11473
:10758000F10421F499ECE92E9DE1F92E80912F0A66
:1075900080FD89C0816080932F0ACDB6DEB684E479
:1075A00097E00E94783781E09AE59093EE158093FA
:1075B000ED1588E590E09093F0158093EF1587E046
:1075C0008093E11582E88093E41584E890E0A0E0E0
:1075D000B0E08093E5159093E615A093E715B0937E
:1075E000E81581E995E10E9473C7C8010F94A9329B
:1075F0005C01C7010F94A9328A0D9B1D03962DB71C
:107600003EB7281B390B0FB6F8943EBF0FBE2DBFF7
:107610008DB79EB701965C01FF92EF921F930F9377
:107620008DE397E09F938F93BF92AF920F94F332C5
:107630008AE289838A838B838C83D501CE01059668
:10764000EDB7FEB738960FB6F894FEBF0FBEEDBF8C
:10765000BE016F5F7F4FFC01E61BF70B2D912111DF
:107660000BC0E60FF71F8AE29F01261B370B28325B
:10767000310534F48193F8CFFC012193CF01EBCF96
:1076800020E630E140E050E081E995E10E9436F0EB
:107690006AE070E080E090E00E940BC70FB6F894BB
:1076A000DEBE0FBECDBE0E94283681E697E00E9466
:1076B000312E61E08FE497E00E945C3489EE93E024
:1076C000019739F000C00000EEE5F9E03197F0F7DE
:1076D000F7CFF89489EE93E0019739F000C00000ED
:1076E000E6EEF3E03197F0F7F7CF0E94448D992052
:1076F00031F00E94629F0E94BC1CA895FECF0E94A0
:10770000299FF9CFE114F10421F489ECE82E8DE1F1
:10771000F82E08E517E03ACF8091C40E9091C50E7F
:107720002FEF3FEF981751F0E92FF0E0EC53F14FB6
:10773000228130E09F5F9F779093C50EC901089525
:107740001F920F920FB60F9211240F900FBE0F9041
:107750001F9018951F920F920FB60F9211240BB61F
:107760000F920F931F932F933F934F935F936F93BA
:107770007F938F939F93AF93BF93CF93DF93EF93B9
:10778000FF93C091C6000091C50ED091C40E11E0C8
:107790001D0F1F7790913306913108F09FC0E92F9C
:1077A000F0E08827E952F44C8F4F0D94233AE83BE0
:1077B000173C263C353C3C3C6E3C403C6E3C443CDB
:1077C000483C6E3C4C3C503C543C5B3C6E3C663C04
:1077D000C03229F028F5CA3011F0CD3031F501174B
:1077E00031F0ED2FF0E0EC53F14FC283D12FD09365
:1077F000C40EFF91EF91DF91CF91BF91AF919F9117
:107800008F917F916F915F914F913F912F911F9138
:107810000F910F900BBE0F900FBE0F901F901895F9
:10782000CD3481F081E0CE3471F080E10CC0CA33F8
:1078300038F4C033A0F6C03291F2CD32B1F7CFCFD9
:10784000CD3499F782E080933306C9CFC13359F024
:1078500018F4C03221F2E9CF88E0C433A1F38BE001
:10786000C83389F3E2CF83E0EECF84E0C03359F32D
:1078700086E0C13341F3D9CF85E0C833B1F6E3CF19
:1078800087E0C23391F6DFCF89E0C13371F6DBCFF9
:107890008AE0C03351F6D7CF8CE0C73331F6D3CF6F
:1078A0008DE0C63311F6CFCFC03209F498CF8EE009
:1078B000C33549F2BACF80ED8C0F8A3008F08FCFF4
:1078C0009FE0909333068093340689CFCA3019F035
:1078D000CD3009F084CF1092330681CFCA3019F031
:1078E000CD3009F07CCF809160168823A1F39730CA
:1078F00089F038F4953079F7109233021092DC0D4C
:10790000EACF9A3059F09F3031F7809134060E94C7
:10791000552BE1CF81E080937E07DDCF81E080931E
:107920007D07D9CF8EBD0DB407FEFDCF08958FEF33
:107930008EBD0DB407FEFDCF8EB508959091640005
:107940009B7F90936400982F906A96959CBD80FDD4
:1079500003C091E0863009F490E09DBD0895AF9298
:10796000BF92CF92DF92EF92FF920F931F93CF932C
:10797000DF938EE897E00E94312EC0E0D7E0D1502F
:1079800021F080E20E942A2EFACF8C2F0E94E687F7
:10799000CF5FC53099F78AE00E942A2E0FE11EE0E2
:1079A000C0E080E20E942A2E8C2F0E94E6875801B8
:1079B000D5E080E20E942A2EF501C080D180E280CD
:1079C000F380A7019601C701B6010F941E3D8823DD
:1079D00069F180E20E942A2E8DE30E942A2E8DE317
:1079E0000E942A2E8DE30E942A2E8DE30E942A2EC9
:1079F0008DE30E942A2ED150F4E1AF0EB11CD111BB
:107A0000D8CF8AE00E942A2ECF5F0C5F1F4FC5306F
:107A100041F68AE0DF91CF911F910F91FF90EF9097
:107A2000DF90CF90BF90AF900C942A2E20E030E0F2
:107A3000A901C701B6010F948C3C87FD03C08BE2FE
:107A40000E942A2E43E0C701B6010E94FE87D3CFD1
:107A50002F923F924F925F926F927F928F929F925E
:107A6000AF92BF92CF92DF92EF92FF920F931F934C
:107A7000CF93DF93CDB7DEB76D970FB6F894DEBF27
:107A80000FBECDBF83E50E944824182F3090DA0D39
:107A9000882319F00E946920382E8091A80E9091B9
:107AA000A90EA091AA0EB091AB0E8A8F9B8FAC8FBE
:107AB000BD8F8091AC0E9091AD0EA091AE0EB091A5
:107AC000AF0E8E8B9F8BA88FB98F8091B00E909147
:107AD000B10EA091B20EB091B30E8A8B9B8BAC8B82
:107AE000BD8B112329F0311003C080E00E940C2AC5
:107AF0008091E0099091E109A091E209B091E30938
:107B000025E1B695A795979587952A95D1F74C01CC
:107B10005D01E1E08E229924AA24BB240E940A2858
:107B2000882309F4C0C083E40E944824882309F410
:107B30009EC00E941E242B013C018FE19EE09F838A
:107B40008E8399878887B5E0BD8300E0212CE8EC1F
:107B5000EE87F2ECFF871A861B8628EC2C8782E4DE
:107B60008D87A885B985B98BA88B15E0E889F98937
:107B7000C190D190E190F190F98BE88B2A853B85FB
:107B80004C855D85C701B6010F945C3387FF04C047
:107B9000CA86DB86EC86FD86202F322D4E855F85DA
:107BA000C701B6010F948C3C181624F40C2D2D2C13
:107BB000EE86FF861150D1F6FD81F150FD83888558
:107BC0009985449699878887F111CBCF202F322D44
:107BD0004E855F856A857B858C859D850F942C3AC3
:107BE00020E030E040E05FE30F94C233A301920154
:107BF0000F942C3A2B013C012DEB37E346E855EB73
:107C00000F948C3C87FD0AC02DEB37E346E855E323
:107C1000C301B2010F945C3318164CF580E00E944A
:107C20000C2A10E0EE80FF8000E0D7016D917D917D
:107C30008D919D917D016D01B4E0CB1AD108A30116
:107C400092010F942B3AF6016083718382839383B0
:107C5000602F812F0F94D2070F5F053031F71F5F20
:107C60008E819F8144969F838E831530D9F6892813
:107C70008A288B2829F00E940A2881110E94AF3C93
:107C80008AE50E944824882351F00E941E246983BB
:107C90007A838B839C83CE0101960F945407832DA6
:107CA0000E940C2A0CC0311004C089288A288B2815
:107CB00039F30E942C3687E09BE00E94312E33205E
:107CC00051F08091DA0D811106C00E94283688EEAD
:107CD0009AE00E94312E0E942C368AED9AE00E9492
:107CE000312E8091DA0D0E94FE340E942C368DECEC
:107CF0009AE00E94312EC090870AD090880AE090C6
:107D0000890AF0908A0A20E030E0A901C701B60193
:107D10000F948C3C18160CF051C042E0C701B6011C
:107D20000E94FE870E943A7B2A8D3B8D4C8D5D8D93
:107D30006091A80E7091A90E8091AA0E9091AB0E41
:107D40000F945C3381111FC02E893F89488D598D56
:107D50006091AC0E7091AD0E8091AE0E9091AF0E11
:107D60000F945C3381110FC02091B00E3091B10E91
:107D70004091B20E5091B30E6A897B898C899D899E
:107D80000F945C3381110E94BAC16D960FB6F894BE
:107D9000DEBF0FBECDBFDF91CF911F910F91FF903E
:107DA000EF90DF90CF90BF90AF909F908F907F909B
:107DB0006F905F904F903F902F90089588EC9AE0DD
:107DC0000E94312EB1CF2F923F924F925F926F92CD
:107DD0007F928F929F92AF92BF92CF92DF92EF925B
:107DE000FF920F931F93CF93DF93CDB7DEB7C858A1
:107DF000D1090FB6F894DEBF0FBECDBF87EB9AE076
:107E00000E94312E87E00E946FDE81116EC084E5F2
:107E10000E949624882329F00E941A2481110E942E
:107E2000EC8780E090E0A0E8BFE389839A83AB838E
:107E3000BC838D839E83AF83B8878DEC9CECACE4D0
:107E4000BEE389879A87AB87BC8780E090E0A0E299
:107E5000B1E48D879E87AF87B88B8CE390E09A8BD7
:107E6000898B8DEC90E09C8B8B8B8DEC9CECACEC3F
:107E7000BEE38D8B9E8BAF8BB88F80E090E0A0EE41
:107E8000BFE3898F9A8FAB8FBC8F1BA61CA64AE9D4
:107E900059E969E97EE38FE40E94A3246D8F7E8F08
:107EA0008F8F98A360E083E40E94E32489A360E0BD
:107EB0008BE40E94E3248AA382E40E949624882310
:107EC00081F10E941A24009761F19C012852310926
:107ED0002536310520F16CE870E089E89AE00E94CF
:107EE000FB3684E89AE00E94312EC857DF4F0FB668
:107EF000F894DEBF0FBECDBFDF91CF911F910F91E0
:107F0000FF90EF90DF90CF90BF90AF909F908F90B9
:107F10007F906F905F904F903F902F9008959A8B35
:107F2000898B8CE40E9496248823E1F00E941E2411
:107F30006B017C01C986DA86EB86FC8620E030E0A6
:107F4000A9010F948C3C87FD0AC020E030E040E09E
:107F500050E4C701B6010F945C3318161CF48CE58D
:107F60009AE0C1CF81E50E944824882331F18091B5
:107F7000140790911507892BE9F00E941E246B01CC
:107F80007C01CD82DE82EF82F8862DEC3CEC4CE465
:107F90005DE30F948C3C87FD0AC020E030E040E7B1
:107FA00051E4C701B6010F945C33181634F48BE228
:107FB0009AE099CF80E09AE096CF83E50E949624DC
:107FC0008823E9F00E941E246B017C01CD8ADE8AA1
:107FD000EF8AF88E2DEC3CEC4CEC5DE30F948C3C7E
:107FE00087FD0AC020E030E040E050E4C701B60160
:107FF0000F945C3318161CF489ED99E074CF80E57A
:108000000E944824882341F180911407909115071C
:10801000892B19F481EA99E066CF8BA58F5F8BA736
:108020000E941E246B017C01CD86DE86EF86F88AD5
:1080300020E030E0A9010F948C3C87FD0AC020E0CD
:1080400030E048EC51E4C701B6010F945C331816D8
:108050001CF489E799E047CF86E40E9496248823A0
:10806000E9F00E941E246B017C01C98EDA8EEB8E32
:10807000FC8E20E030E040E85FE30F948C3C87FD0D
:108080000AC020E030E040E850E4C701B6010F9498
:108090005C3318161CF480E599E025CFC98CDA8C86
:1080A000EB8CFC8C8D889E88AF88B88CA7019601DC
:1080B000C701B6010F94C2339B01AC0160E070E0D0
:1080C00084E490E40F94263B29813A814B815C81C2
:1080D0000F94C2332B013C01A5019401C501B401E9
:1080E0000F94C233A70196010F94C2332CEE31E5F1
:1080F00048EB5DE30F94263B9B01AC01C301B20149
:108100000F94C23369837A838B839C8388E40E94B3
:108110009624882379F00E941A24009759F09C0134
:10812000255A31092838310518F082E299E0DBCE72
:108130009C8B8B8B85E50E9448248823C9F00E9484
:10814000D877611571058105910511F00F94E22E24
:108150008091140790911507892B09F10E941E2424
:108160006093100770931107809312079093130781
:1081700082E50E9448248823B9F0809114079091E9
:108180001507892BA1F00E941A24AD969FAF8EAFE0
:10819000AD97181619068CF08AEB98E0A4CE60E033
:1081A00070E088E492E4DCCF8EEE98E09CCE2AE189
:1081B00030E0AD963FAF2EAFAD9789E50E94962493
:1081C000882381F10E941E242091BC0E3091BD0EA7
:1081D0004091BE0E5091BF0E0F942B3A6B017C0163
:1081E00088E50E949624882331F10E941E24209164
:1081F000B80E3091B90E4091BA0E5091BB0E0F944B
:108200002B3A6BA37CA38DA39EA3CFA2D8A6E9A6ED
:10821000FAA6CE0183960E947B1C811115C080E9CD
:1082200098E061CEC090AC0ED090AD0EE090AE0E56
:10823000F090AF0ED5CF6091A80E7091A90E8091ED
:10824000AA0E9091AB0EDDCF8091E0099091E109EB
:10825000A091E209B091E30933E0B695A79597950F
:1082600087953A95D1F780959095A095B0958170B6
:108270000E940C2A80E090E0A0EAB0E48DA79EA7BF
:10828000AFA7B8AB60E0CE018D960E94ACC0309134
:108290003407CF57DF4F3883C158D040109234078E
:1082A0000E9401B78FE698E00E94312E89899A8951
:1082B0008A3191050CF045C08B899C890E9406B6D5
:1082C00041E061E080E00E94998A81114CC06FEF2B
:1082D00084E898E00E941BCA8CA5811104C0CE01DD
:1082E00001960E94B67680E090E0A0EAB0E4809328
:1082F0001B0990931C09A0931D09B0931E091DA68C
:108300001EA61FA618AABE01635D7F4F83E199E0F8
:108310000E940821CF57DF4FB881C158D040B09399
:1083200034070E9401B78AA18111DFCD10924C134E
:1083300010924B130E94D42790E080E00E9406B672
:10834000D4CD8C38910514F08CE890E090934C13C8
:1083500080934B130E94D42761E081E00E94118931
:108360008111AACFB4CF1092B40E1092B50E109214
:10837000B60E1092B70E84EB9EE00E943DBA8BA51C
:10838000882309F452C020E030E040E751E46091D6
:10839000C20D7091C30D8091C40D9091C50D0F94C5
:1083A000263B6DA77EA78FA798AB80E1E8EAFEE0A9
:1083B000A3E1B9E001900D928A95E1F72D853E8504
:1083C0004F85588960911F0970912009809121097A
:1083D000909122090F942C3A60931F097093200901
:1083E0008093210990932209CE018D960E9441BF6E
:1083F0002D853E854F85588960911F097091200910
:1084000080912109909122090F942B3A60931F09C2
:108410007093200980932109909322098CA58111E2
:1084200004C0CE0101960E94B676EBE0F7E085E04D
:10843000DF011D928A95E9F780E1E8EAFEE0A3E119
:10844000B9E001900D928A95E1F789859A85AB850F
:10845000BC8580931B0990931C09A0931D09B093C0
:108460001E091DA61EA61FA618AABE01635D7F4F8A
:1084700083E199E00E940821BE01635E7F4F83E1A2
:1084800099E00E94082189A1882309F4F8C380910A
:10849000A80E9091A90EA091AA0EB091AB0EE596F0
:1084A0008CAF9DAFAEAFBFAFE5978091AC0E909112
:1084B000AD0EA091AE0EB091AF0EE1968CAF9DAF18
:1084C000AEAFBFAFE19710E000E033243A9422242E
:1084D0002A949FEFEE969FAFEE97AFE4EF96AFAF83
:1084E000EF97B3ECC158DF4FB883CF57D040E7E4E4
:1084F000C058DF4FE883C058D04021E030E0002E64
:1085000002C0220F331F0A94E2F7CE57DF4F3983A0
:108510002883C258D0408BE097E0A9969FAF8EAFDA
:10852000A997A5961FAE1EAEA597C801012E000CF7
:10853000AA0BBB0BCC57DF4F88839983AA83BB83DD
:10854000C458D040C857DF4F0883C858D040A996B8
:10855000AEADBFADA9978D91A996BFAFAEAFA997AC
:1085600090E0CE57DF4FE881F981C258D0408E238A
:108570009F23892B09F01CC1CC57DF4F688179817B
:108580008A819B81C458D0400F94633320913D076A
:1085900030913E0740913F07509140070F94C233FE
:1085A00020913507309136074091370750913807B1
:1085B0000F942C3AE9966CAF7DAF8EAF9FAFE997E1
:1085C000A5962EAD3FADA597B901330F880B990B3A
:1085D0000F94633320914107309142074091430744
:1085E000509144070F94C2332091390730913A07D4
:1085F00040913B0750913C070F942C3A4B015C0192
:10860000E9962CAD3DAD4EAD5FADE997E5966CAD0D
:108610007DAD8EAD9FADE5970F942B3A6B017C013C
:10862000A5019401E1966CAD7DAD8EAD9FADE19756
:108630000F942B3A2B013C01A7019601C701B6010B
:108640000F94C2336B017C01A3019201C301B201FB
:108650000F94C2339B01AC01C701B6010F942C3AB1
:108660000F94DA3C6B017C01E9962CAD3DAD4EAD2B
:108670005FADE9976BA17CA18DA19EA10F942B3AD0
:108680002B013C01A50194016FA178A589A59AA5AC
:108690000F942B3A4B015C01A3019201C301B2017B
:1086A0000F94C2332B013C01A5019401C501B40113
:1086B0000F94C2339B01AC01C301B2010F942C3A59
:1086C0000F94DA3C20E030E040E751E40F94263B81
:1086D000A70196010F942C3A6B017C018090100742
:1086E00090901107A0901207B090130720E030E09F
:1086F00040E85FE3C501B4010F948C3C1816F4F414
:10870000C501B4010F94983B4B015C0160E070E03F
:10871000CB01181419041A041B0434F40F94932E7B
:10872000A50194010F94C2390F9463339B01AC01EE
:10873000B601C7010F942C3A6B017C01EE962FAD68
:10874000EE97EF963FADEF97C158DF4F4881CF5777
:10875000D040C058DF4F5881C058D040B601C70143
:108760000F945C3387FF24C0A4963FACA497C857EE
:10877000DF4F2880C858D040EA96CFAEEA97EB96F4
:10878000DFAEEB97EC96EFAEEC97ED96FFAEED9784
:10879000EE96CFAEEE97EF96DFAEEF97C158DF4F74
:1087A000E882CF57D040C058DF4FF882C058D04041
:1087B000A5968EAD9FADA5970196A5969FAF8EAF5E
:1087C000A597059709F0C3CE0F5F1F4F0530110520
:1087D00009F093CEE32DF0E0E55FF84F21E030E0C3
:1087E000022C01C0220F0A94EAF78081822B808339
:1087F0006A962FAE6A976B963FAE6B97EA968FADEF
:10880000EA97EB969FADEB97EC96AFADEC97ED96B4
:10881000BFADED976F968CAF9DAFAEAFBFAF6F970B
:108820009FEF291609F410C2391609F40DC2622D02
:10883000022C000C770B880B990B0F94633320915B
:108840003D0730913E0740913F07509140070F94FC
:10885000C233209135073091360740913707509148
:1088600038070F942C3AF62E072F182FE92E862F53
:10887000902FA12FBE2D65968CAF9DAFAEAFBFAF31
:108880006597632D032C000C770B880B990B0F94C5
:108890006333209141073091420740914307509143
:1088A00044070F94C2332091390730913A07409121
:1088B0003B0750913C070F942C3A4B015C016996A1
:1088C0008CAE9DAEAEAEBFAE6997CE018F5A9F4FB4
:1088D0000E947B1C882309F4BBC120E030E040EA01
:1088E00050E46F2D702F812F9E2D0F942C3A3B0159
:1088F0006C01CB01D60121968CAF9DAFAEAFBFAF5F
:10890000219725968CAE9DAEAEAEBFAE25972110B9
:10891000EEC13110C3C120E030E040EA50E4C501AF
:10892000B4010F942C3A4B015C01332009F4D6C1F9
:10893000B3E0B3150CF4D2C122ED422E23E5522E42
:108940002BE7622E21E4722E21968CAD9DADAEAD4B
:10895000BFAD2197A7968CAF9DAFAEAFBFAFA79726
:1089600025968CAD9DADAEADBFAD2597AB968CAFCA
:108970009DAFAEAFBFAFAB979C01AD0169966CAD3B
:108980007DAD8EAD9FAD69970F942B3AE1966CAF9C
:108990007DAF8EAF9FAFE197A7962CAD3DAD4EADAD
:1089A0005FADA79765966CAD7DAD8EAD9FAD6597BC
:1089B0000F942B3A2D966CAF7DAF8EAF9FAF2D9756
:1089C000E1968CAD9DADAEADBFADE19761968CAF3C
:1089D0009DAFAEAFBFAF6197A7962CAD3DAD4EAD8D
:1089E0005FADA7976091A80E7091A90E8091AA0E15
:1089F0009091AB0E0F942B3AA7966CAF7DAF8EAFD4
:108A00009FAFA797AB962CAD3DAD4EAD5FADAB978D
:108A10006091AC0E7091AD0E8091AE0E9091AF0E44
:108A20000F942B3AAB966CAF7DAF8EAF9FAFAB97E9
:108A30008F2D902FA12FBE2D8DA79EA7AFA7B8ABCE
:108A400089AA9AAAABAABCAA89849A84AB84BC845A
:108A50008DAA9EAAAFAAB8AE2DEC3CEC4CEC5CE320
:108A6000C301B2010F94C23329813A814B815C81E9
:108A70000F94C2332091B40E3091B50E4091B60ED2
:108A80005091B70E0F942C3A69AF7AAF8BAF9CAF71
:108A9000A7962CAD3DAD4EAD5FADA797CA01B9010C
:108AA0000F94C2336B017C01AB962CAD3DAD4EAD46
:108AB0005FADAB97CA01B9010F94C2339B01AC0102
:108AC000C701B6010F942C3A20E030E040E050E4BA
:108AD0000F948C3C1816ACF420E030E040E05FE3EB
:108AE000C501B4010F942C3A29966CAF7DAF8EAFBF
:108AF0009FAF2997BE01635C7F4FCE0101960E9414
:108B0000E81F89859A85AB85BC8529968CAF9DAF7A
:108B1000AEAFBFAF2997A3961CAE1DAE1EAE1FAE63
:108B2000A397BE01615A7F4FCE01CD960E940821C6
:108B30008CA58823C1F02AE939E949E95FE36D8111
:108B40007E818F8198850F94C233A3966CAF7DAFE1
:108B50008EAF9FAFA397BE01615A7F4F83E199E02B
:108B60000E9408211CA6E090BA0DF090BB0D009168
:108B7000BC0D1091BD0DA090B60DB090B70DC0907A
:108B8000B80DD090B90D9501A601B701C8010F9499
:108B90008C3C181614F47501860180903402909074
:108BA0003502A0903602B09037022DEC3CEC4CEC34
:108BB0005DE3B701C8010F94C23360933402709330
:108BC0003502809336029093370240E0BE01675B26
:108BD0007F4FCE018D960E94AA9480E1E8EAFEE0E4
:108BE000A3E1B9E001900D928A95E1F780923402F9
:108BF00090923502A0923602B092370220E04FEFF9
:108C0000BE01675A7F4FCE0101960E94832220E069
:108C100041E0BE01675A7F4FCE0101960E94832238
:108C20002FEF40E0BE01675A7F4FCE0101960E94B0
:108C3000832221E040E0BE01675A7F4FCE010196BA
:108C40000E9483220E94A8B68091C40E8093C50E14
:108C5000AD96AEADBFADAD971197AD96BFAFAEAF10
:108C6000AD97AB2B09F433CB6A968FAD6A9787FD2E
:108C70002ECB6B968FAD6B9787FF05CC28CB8BA146
:108C80009CA1ADA1BEA1E5968CAF9DAFAEAFBFAF2D
:108C9000E5978FA198A5A9A5BAA50FCC8F2D902FE8
:108CA000A12FBE2D21968CAF9DAFAEAFBFAF219748
:108CB00020E030E040EA50E4C501B4010F942B3AC3
:108CC00025966CAF7DAF8EAF9FAF2597A3E0A31520
:108CD0000CF021CEF62C072D1C2DED2C92ED492EFB
:108CE00093E5592E9BEF692E90E4792E2DCEE3E08B
:108CF000E2150CF04AC0E315FCF420E030E040EA55
:108D000050E46F2D702F812F9E2D0F942B3A2196BA
:108D10006CAF7DAF8EAF9FAF219720E030E040EA8F
:108D200050E4C501B4010F942B3A4B015C01F3E010
:108D3000F3150CF001CED2CF8F2D902FA12FBE2D89
:108D400021968CAF9DAFAEAFBFAF219720E030E052
:108D500040EA50E4C501B4010F942C3A25966CAF5B
:108D60007DAF8EAF9FAF25973110D7CF20E030E099
:108D700040EA50E46F2D702F812F9E2D0F942B3AD7
:108D8000F62E072F182FE92EA9CF31100DC020E0A5
:108D900030E040E251E4B301C6010F942B3AF62EC5
:108DA000072F182FE92EC8CD23E023159CF420E0CF
:108DB00030E040E251E4B301C6010F942B3A219612
:108DC0006CAF7DAF8EAF9FAF2197F62C072D1C2D7A
:108DD000ED2CB2CDF62C072D1C2DED2C82ED482E5E
:108DE00083E5582E8BEF682E81E4782EADCD2F923F
:108DF0003F924F925F926F927F928F929F92AF922B
:108E0000BF92CF92DF92EF92FF920F931F93CF9377
:108E1000DF93CDB7DEB768970FB6F894DEBF0FBE0D
:108E2000CDBFB82E8091B10F843008F0D8C10E9418
:108E3000D8776B017C018091B10F811108C08091BE
:108E4000C40E9091C50E891B8F7709F424C781E663
:108E5000A82E13C08A3019F08D3009F0F6C0109298
:108E6000AC0F80914A0F90914B0FFC01EA5BF04FE1
:108E70001682892BF1F40E9429908091B10F8430E1
:108E800008F0ECC08091C40E9091C50E891B8F77BD
:108E900009F4E4C00E948C3B97FFDCCF0E94283687
:108EA0008DE096E00E94312E8091C40E8093C50E15
:108EB000E4CF10924B0F10924A0F0CE41FE0F80120
:108EC0008191803209F446C08E3409F0A9C068E06F
:108ED00076E0C8010F94D9324C01892B41F06EE441
:108EE00070E0C80104960F947A3D009709F4C80118
:108EF0004AE050E070E060E001960F9449302B01A9
:108F00003C018091460F9091470FA091480FB0917E
:108F1000490F0196A11DB11D481659066A067B0628
:108F200029F060E085ED95E0892851F16AE270E072
:108F3000C8010F94A93D9C01009729F1982F901B1F
:108F4000912C992349F09150F801E90FF11D80818E
:108F50009826F7CF8F01B3CF4AE050E070E060E091
:108F6000C90101960F944930292D30E050E040E0CE
:108F7000621773078407950751F060E086EB95E070
:108F80000E9443F87ACF60E08CE895E0F9CF4092F8
:108F9000460F5092470F6092480F7092490F809190
:108FA0005C088130E1F467E470E0C8010F947A3D19
:108FB0000097A9F04AE050E070E060E001960F945D
:108FC0004930643071058105910548F48BEE94E0D9
:108FD0000E94312E60E081EE94E00E941BCAC09294
:108FE0007B0AD0927C0AE0927D0AF0927E0A809100
:108FF0004C0F8B3309F441CF8091B10F843008F0CE
:109000003CCF8091B30F8A9DC00111246CE47FE0B6
:109010008C54904F0F94853D80E00E94FFF72DCF38
:1090200080916C1680FFBBCF62E973E2C8010F9498
:10903000D932009731F0FC01838180538A3008F0E7
:10904000AECF60E082E695E09BCF2AE43FE04CE4BF
:109050005FE06CEA7FE00E94C6DA0FCF80916C1669
:1090600083FDBDC082FFBBC087FDB9C01A821982D3
:1090700001E6F02E84E0E82E99E6D92E8091B10F1A
:10908000843008F0ACC00E94FEDA8111A8C041E033
:1090900050E0BE016D5E7F4F80ED97E10E94E5815B
:1090A0000B8910E0019711F00FEF1FEF8091D81797
:1090B0009091D917A091DA17B091DB1780936816B9
:1090C00090936916A0936A16B0936B160E94FEDA0D
:1090D0000F3F100749F4811107C00E9428368BE228
:1090E00096E00E94312ECACF4091B30F242F30E07A
:1090F0000A3061F00D3051F0882309F462C0898193
:109100009A81009719F001969A8389831092B80684
:1091100089819A81F29EF001F39EF00D1124EF54A3
:10912000F04FE80FF91F1382892B59F50E942990FF
:109130000E94FEDA882309F4A1CF80ED97E10E9416
:10914000928380916316882391F1815080936316F6
:109150008D9DC001112462E08657984F0E9493AC08
:10916000E091631624E0E29FF0011124EA57F84FE2
:1091700060817181828193810E94A8DA0E94A57B1F
:109180007DCF1A82198281E00E94FFF780916816D4
:1091900090916916A0916A16B0916B168093AD0FED
:1091A0009093AE0FA093AF0FB093B00FC1CF0E94BA
:1091B0009B8380916C16886080936C16E0925C08AB
:1091C0005DCF4F9DA00111244C54504F9E012F5F45
:1091D0003F4F68EB76E0802F0E94C6DA4FCF0E94A7
:1091E000D8776B017C01B11004C0809112098823EB
:1091F00051F0C0928113D0928213E0928313F092C7
:109200008413BB24B3948091200790912107A091EF
:109210002207B09123070097A105B105B1F0409155
:109220008113509182136091831370918413840F82
:10923000951FA61FB71FA7019601281B390B4A0BC4
:109240005B0BDA01C901B7FF08C18091150290914B
:109250001602A0911702B0911802892B8A2B8B2B32
:1092600009F00CC10E94D8774B015C011091DC0D14
:10927000111108C090919B1480919C1411E09813D7
:1092800001C010E020E030E04AE253E460915E1358
:1092900070915F1380916013909161130F948C3CD7
:1092A00087FD2FC181E0182781E04091BD065091D4
:1092B000BE066091BF067091C006452B462B472B1A
:1092C00009F480E0811799F080E090E0DC0111233F
:1092D00031F0D501C40180569444A24FBF4F809312
:1092E000BD069093BE06A093BF06B093C006409003
:1092F000B40E5090B50E6090B60E7090B70E2091DF
:10930000B9063091BA064091BB065091BC06C30124
:10931000B2010F945C33882319F18091BD069091BE
:10932000BE06A091BF06B091C0064092B906509209
:10933000BA066092BB067092BC06892B8A2B8B2BD7
:1093400009F449C0D501C40180569444A24FBF4FCF
:109350008093BD069093BE06A093BF06B093C0064F
:109360008091BD069091BE06A091BF06B091C00647
:109370000097A105B10579F1881A990AAA0ABB0AD2
:10938000B7FC29C01092BD061092BE061092BF060F
:109390001092C0068BE896E00E94312E60E087E7CD
:1093A00096E00E941BCA8091621390916313181675
:1093B000190624F490E080E00E9406B680914B13D9
:1093C00090914C131816190634F410924C13109205
:1093D0004B130E94D4278091C9069091CA06A09190
:1093E000CB06B091CC0646015701881A990AAA0A01
:1093F000BB0AD501C401B7FD2FC230919B149091D7
:109400009C142091000280912402391709F47BC03A
:10941000E0919C143BE5E39FF0011124E750F54FE8
:109420009081899FC0011124880F892F881F990B73
:109430009195281709F4CEC0809300020E94D87736
:1094400020910002211162C01092C1061092C20642
:109450001092C3061092C4067CC00E942836609108
:10946000790A70917A0A8AE396E00E9436AA40E06F
:1094700070E060E090E080E00E94A73A90919B1439
:1094800080919C14981749F0C0928113D092821356
:10949000E0928313F0928413E5CEBB2019F0109272
:1094A000CD06E0CE0E94D8770091811310918213EF
:1094B00020918313309184138090150290901602AE
:1094C000A0901702B0901802080D191D2A1D3B1D0F
:1094D000601B710B820B930B97FDE1CF8091CD0642
:1094E0008111C0CE81E08093CD0680E00E94389F3C
:1094F00081E00E94389F82E00E94389F0E94299F4D
:10950000B1CE10E0D1CE9091A00A8BCF0091C106D0
:109510001091C2062091C3063091C40601151105B1
:109520002105310581F46C597F4F8F4F9F4F609318
:10953000C1067093C2068093C3069093C4068FEF52
:109540008093000206C0601B710B820B930B97FD8A
:10955000F6CF00910002002309F401C110E061E0A0
:109560000F3F110509F4FCC069E0CE0101960E948D
:10957000A62B8989882309F4EEC0E981FA819F85A9
:1095800088899111ABC0608190E023E030E0A901AF
:10959000481B590B440F551F042E01C0220F0A947B
:1095A000EAF72095262362E070E001C0660F4A9535
:1095B000EAF7262B2083FC013396EE0FFF1F41E0D4
:1095C00050E04C0F5D1FE40FF51F0190F081E02D7E
:1095D0001183008380918507882309F430C10091AD
:1095E000420210914302C801029720916213309108
:1095F0006313281739070CF422C180909C148C8ABD
:109600001D8A1E8A1F8A188E80919B149C8889153A
:1096100009F4AAC0892D90E03BE5A32EA89EF00195
:10962000A99EF00D1124ED55F54F4589568967899E
:10963000708D452B462B472B81F4418D528D638DC8
:10964000748D452B462B472B41F4458D568D678DE8
:1096500070A1452B462B472BE1F12BE5B22EB89E8E
:109660009001B99E300D1124A9014D55554F1A0195
:10967000FA0161817281838194810F94DA3C4B01FC
:109680005C01F10161A172A183A194A10F946133E6
:109690002B013C01F10165A176A187A190A50F9452
:1096A00061339B01AC01C301B2010F94263BA501BC
:1096B00094010F94C2334B015C012D893E894F897F
:1096C000588D0F948C3C181624F48D8A9E8AAF8A8C
:1096D000B88E8C898F5F87708C8B96CF2A892111E9
:1096E00079CFAFEFB0E0923029F0AD85BE850D9017
:1096F000BC91A02D608190E023E030E0A901481BDF
:10970000590B440F551F042E01C0220F0A94EAF78B
:109710002095262362E070E001C0660F4A95EAF7C3
:10972000262B20830396880F991FE1E0F0E0EC0FD1
:10973000FD1F8E0F9F1FFC01A080B18098010F9428
:10974000F4392FEF30E040E050E00F94A039F501FC
:10975000318320833FCF61E00F37110508F460E0CB
:1097600089E00E94D67636CF20913C0230913D02AE
:1097700040913E0250913F026D897E898F89988D7C
:109780000F94C2334B015C01B801012E000C880B11
:10979000990B0F9463339B01AC01C501B4010F9485
:1097A0002C3A69837A838B839C8340914002509149
:1097B0004102B801CE0101960E94E78F49805A808C
:1097C0006B807C808090C5069090C606A090C706EE
:1097D000B090C806A5019401C301B2010F945C3397
:1097E00087FF1CC020E037ED43EA5CE3C301B20110
:1097F0000F94C2332B013C0128E431EE4AE75FE3CA
:10980000C501B4010F94C2339B01AC01C301B20185
:109810000F942C3A69837A838B839C8369817A8144
:109820008B819C816093C5067093C6068093C706A2
:109830009093C8060F94983BCB010E9406B6F4E6BD
:10984000CF0ED11CE11CF11CC092C906D092CA06F1
:10985000E092CB06F092CC060E94299080915C08A1
:10986000882309F4DCC180916802882309F49FC031
:1098700080913D0981119BC08091120981110AC01C
:1098800080918713813031F080916C1682FF8FC0F8
:1098900087FD8DC0F894649B10C080911B0290914D
:1098A0001C02A0911D02B0911E028093510790935B
:1098B0005207A0935307B0935407609151077091DA
:1098C00052078091530790915407789420E030E03C
:1098D000A9010F945C3387FF6AC081E080933D0942
:1098E00080911209811161C080EA96E00E94783768
:1098F00084E08093A20E81E09AE59093EE15809328
:10990000ED158EE490E09093F0158093EF1587E0CD
:109910008093E11582E88093E41584E890E0A0E06C
:10992000B0E08093E5159093E615A093E715B0930A
:10993000E81581E995E10E9473C780915F1688233D
:1099400031F040E364EE76E081E00E94953461E01E
:1099500082E095E20E9478341091240781E060E073
:10996000182782E698E069F482ED96E00E945C3464
:1099700080E30E942A2E8AE00E942A2E60E085EB76
:1099800096E00E945C3480EC96E00E94312E80E3E9
:109990000E942A2E8AE00E942A2E112331F08BEB9E
:1099A00096E090931E0E80931D0E0E94A8B6909193
:1099B0000901892F80958170109101021817C9F053
:1099C00020916C16206420936C168093010290FD08
:1099D0003FC164EF71E080E090E00E941E2B0E9486
:1099E000C38380916C1684FD79C1111133C10E942B
:1099F00058D00E94D8776B017C011091140211237A
:109A0000F1F080913E098823D1F04091CE0650912B
:109A1000CF066091D0067091D10646015701841A95
:109A2000950AA60AB70AB501A40177FD1AC08330CA
:109A300009F42CC10CF01BC181300CF020C1212F86
:109A400030E0A8EEB3E00F94F439C60ED71EE81E3E
:109A5000F91EC092CE06D092CF06E092D006F092C8
:109A6000D10680918713813009F073C00E94D877A6
:109A70006B017C018091D6069091D706A091D80603
:109A8000B091D906A7019601281B390B4A0B5B0B35
:109A9000DA01C901B7FD3AC0D701C601805F984D10
:109AA000AF4FBF4F8093D6069093D706A093D806AA
:109AB000B093D9068090440A9090450AA090460A37
:109AC000B090470A0E944DC5AB01BC014093440AC7
:109AD0005093450A6093460A7093470A80910108A3
:109AE00090910208A0910308B0910408881999097F
:109AF000AA09BB09840F951FA61FB71F80930108F1
:109B000090930208A0930308B09304088091D206B2
:109B10009091D306A091D406B091D5064601570185
:109B2000881A990AAA0ABB0AD501C401B7FD11C057
:109B300020E8C20E2EEED21E26E3E21EF11CC092D9
:109B4000D206D092D306E092D406F092D5060E94B7
:109B50007FB50E94E0C80E949FE280911F07882382
:109B600079F10E94D8776B017C0180911B0790915D
:109B70001C07A0911D07B0911E0746015701881AC6
:109B8000990AAA0ABB0AD501C401B7FD19C02091E0
:109B90001F0730E0A8EEB3E00F94F439C60ED71ECD
:109BA000E81EF91EC0921B07D0921C07E0921D0709
:109BB000F0921E0780E00E94A0888AE00E942A2E70
:109BC00080911A07882359F10E94D8776B017C0194
:109BD0008091160790911707A0911807B091190767
:109BE000A7019601281B390B4A0B5B0BDA01C9014F
:109BF000B7FD15C020911A0730E0A8EEB3E00F942E
:109C0000F439C60ED71EE81EF91EC0921607D09270
:109C10001707E0921807F09219070E94727B689666
:109C20000FB6F894DEBF0FBECDBFDF91CF911F916D
:109C30000F91FF90EF90DF90CF90BF90AF909F90EB
:109C40008F907F906F905F904F903F902F900895EE
:109C50000E94AB83123008F0CCCE0E9458D0C9CEFF
:109C600085EF96E090931E0E80931D0EC2CE843039
:109C700009F0E5CE0E942C368CEF96E004C00E94DD
:109C80002C368BE297E00E94312ED9CE0E942C36E2
:109C900084E197E0F8CF80917B0A90917C0AA091B3
:109CA0007D0AB0917E0AA7019601281B390B4A0B49
:109CB0005B0BDA01C901885E9340A109B109B7FDC8
:109CC000C6C885E296E00E94312EC0927B0AD092EF
:109CD0007C0AE0927D0AF0927E0AB9C8123018F42C
:109CE0000E94E9E086CE123009F083CE0E94D2872E
:109CF000882379F081E00E94A2AA40EB50E06FE552
:109D000078E081E796E10E94E58181E796E10E9493
:109D100092830E9417278111A3CF0E94F9260E94E7
:109D20002EAB81E0809362160E94798762CE2F92DB
:109D30003F924F925F926F927F928F929F92AF92DB
:109D4000BF92CF92DF92EF92FF920F931F93CF9328
:109D5000DF93CDB7DEB7E9970FB6F894DEBF0FBE3D
:109D6000CDBF8091DA0D888B8091E0099091E10957
:109D7000A091E209B091E309AC01BD0126E176951D
:109D80006795579547952A95D1F740FF16C10E94D0
:109D90000A28811107C00E94283684EB9BE00E94AC
:109DA000312E22C18AE50E949624882339F10E942F
:109DB0001E242091C00E3091C10E4091C20E5091D0
:109DC000C30E0F942B3A6B017C0120E030E040E29F
:109DD00051ECC701B6010F948C3C87FD0AC020E00E
:109DE00030E040E251E4C701B6010F945C3318162D
:109DF00074F40E94283687EA9BE0D1CFC090B00E61
:109E0000D090B10EE090B20EF090B30EDECF40E0F5
:109E100050E060EC7FE788E50E94A3242091B80E13
:109E20003091B90E4091BA0E5091BB0E0F942B3A5F
:109E30002B013C0140E050E060EC7FE789E50E94A7
:109E4000A3242091BC0E3091BD0E4091BE0E5091C6
:109E5000BF0E0F942B3A4B015C016FEF89E40E9417
:109E6000D724182F6FEF8AE40E94D724082FA3016C
:109E70009201C301B2010F941E3D81116EC0A50174
:109E80009401C501B4010F941E3D811166C08BA1E0
:109E90009CA1ADA1BEA18FA798ABA9ABBAAB2091F5
:109EA0003507309136074091370750913807C30185
:109EB000B2010F942B3A2B013C0120E030E040E04E
:109EC0005FE36FA578A989A99AA90F94C2339B0172
:109ED000AC01C301B2010F942C3A2FA538A949A9AE
:109EE0005AA90F94263B0F94983B162F4FA058A4C5
:109EF00069A47AA42091390730913A0740913B0731
:109F000050913C07C501B4010F942B3A4B015C0101
:109F100020E030E040E05FE3C301B2010F94C233C0
:109F20009B01AC01C501B4010F942C3AA30192012D
:109F30000F94263B0F94983B062F812F012E000C87
:109F4000990B97FD32C0059794F5802F002E000CD9
:109F5000990B97FD2EC0059774F5153008F044C095
:109F6000053008F041C080E00E940C2A95E01902FB
:109F7000F0011124E00FF11D07FDFA95EE0FFF1F10
:109F8000EE0FFF1FE15EF14FC082D182E282F382C9
:109F9000602F812F0F94D20788890E940C2A88890C
:109FA000882311F10E94BAC11FC010E0CECF14E087
:109FB000CCCF00E0D2CF04E0D0CF19E0B695A79582
:109FC000979587951A95D1F780FD0CC070E060E0F9
:109FD00086E50E94BA249A8389830597F0F082E887
:109FE0009BE0DDCE0E944F2AE9960FB6F894DEBFC3
:109FF0000FBECDBFDF91CF911F910F91FF90EF90DA
:10A00000DF90CF90BF90AF909F908F907F906F9098
:10A010005F904F903F902F90089560E084E40E94FD
:10A02000E3248F8740E050E0BA018AE50E94A32430
:10A030006BA77CA78DA79EA740E050E86BE376E472
:10A0400083E50E94A32420E030E040E752E40F942F
:10A05000263B609338027093390280933A029093C2
:10A060003B020091961410919714D801CD90DD9089
:10A07000ED90FC9020E030E0A901C701B6010F94FB
:10A080002C3A6EAB7FAB88AF99AF20E030E040E276
:10A0900051E40F945C3387FF06C01EAA1FAAB0E2EA
:10A0A000B8AFE1E4E9AF20E030E84DE953E4C7019F
:10A0B000B6010F942C3A6FA7672E8BAB9CAB20E0B8
:10A0C00030E041E953E40F948C3C181634F41FA699
:10A0D000612CF1E9FBAB23E42CABD80114968D90F5
:10A0E0009D90AD90BC90179720E030E0A901C5018C
:10A0F000B4010F942C3A7B018C0120E030E040EA5F
:10A1000051E40F945C3387FF04C0E12CF12C00EA8A
:10A1100011E420E030E04BE953E4C501B4010F94B1
:10A120002C3AB62EC72ED82E9DAB20E030E04CE85E
:10A1300053E40F948C3C181634F4B12CC12CFCE879
:10A14000DF2EB3E4BDAB88E40E944824882309F4E1
:10A1500009C20E941E240F94983B1B0177FF02C086
:10A160006F5F7F4F759567957195619571096A5617
:10A170007F4F072E000C880B990B0F946333762EBC
:10A18000872E982EA92E9701A8010F948C3C1816A3
:10A1900024F4E72CF82C092D1A2D2EA93FA948AD3F
:10A1A00059AD672D782D892D9A2D0F948C3C18165A
:10A1B00024F07EA88FA898ACA9AC872D982DA92D46
:10A1C000BA2D8B8B9C8BAD8BBE8BC701D8018F8B2F
:10A1D000988FA98FBA8FB101330C880B990B0F940C
:10A1E00063331B012C01AC019B01B701C8010F9423
:10A1F0002C3A7B018C012B2D3C2D4D2D5DA90F940C
:10A200005C3387FF04C0BE2CCF2CD02E1DABA20127
:10A210009101672D782D892D9A2D0F942C3A7B0171
:10A220008C012FA5362D4BA95CA90F945C3387FFB9
:10A2300004C0EFA66F2C0BAB1CAB8FA5962DABA962
:10A24000BCA98B8F9C8FAD8FBE8F8B2D9C2DAD2D80
:10A25000BDA98F8F98A3A9A3BAA3BE01695E7F4F42
:10A26000CE0143960E94D372882309F4AAC1BE018D
:10A27000615E7F4FCE014B960E94D372E82E8823F9
:10A2800009F49FC12F89388D498D5A8D6F8D78A122
:10A2900089A19AA10F942B3A20E030E040E85EE3D8
:10A2A0000F94C2334B015C012B893C894D895E8937
:10A2B0006B8D7C8D8D8D9E8D0F942B3A20E030E040
:10A2C00040E85EE30F94C2336BA37CA38DA39EA3EF
:10A2D0008FA298A6A9A6BAA689819A8118161906EE
:10A2E00074F480E59BE00E94312E8F85882321F055
:10A2F00086E49BE00E94312E8AE00E942A2E0E9472
:10A30000A8B60E9422BF80E00E940C2A80915E08BD
:10A31000811103C081E00E9436C320913D07309136
:10A320003E0740913F07509140076BA17CA18DA152
:10A330009EA10F945C33811130C020914107309170
:10A34000420740914307509144076FA178A589A522
:10A350009AA50F945C33811120C02091350730916C
:10A36000360740913707509138076B897C898D8972
:10A370009E890F945C33811110C020913907309170
:10A380003A0740913B0750913C076F89788D898D42
:10A390009A8D0F945C338823A9F00E944F2A88E09D
:10A3A000FE01B396ADE3B7E001900D928A95E1F717
:10A3B00088E0FE017396A5E3B7E001900D928A95BF
:10A3C000E1F7188A60E085E40E94E324882309F419
:10A3D000FBC0E1E0EFA71B861C861D861E861A8A3D
:10A3E0009E2C46E1C42E4BE0D42E54E2A52E5BE019
:10A3F000B52E1A8915300CF0F7C06B857C858D85DC
:10A400009E859B01AC010F941E3D8111EDC09920EA
:10A4100009F4DDC021E02BAB35E0232E91E0992635
:10A42000F12EFF0CFF0CF10EF394898B19896A89C8
:10A43000121509F4D5C0062E000C770B880B990B6A
:10A440000F9463332FA138A549A55AA50F94C233A1
:10A450002F89388D498D5A8D0F942C3A2B013C0150
:10A46000612F110F770B880B990B0F9463332BA17E
:10A470003CA14DA15EA10F94C2332B893C894D892B
:10A480005E890F942C3A6B837C838D839E834F82ED
:10A49000588669867A8689819A81892B89F082E338
:10A4A0009BE00E94312E8F2D0E94E68769E170E0CB
:10A4B00080E39BE00E94FB368DE29BE00E94312E00
:10A4C0001F9289E18F931F92FF92DF92CF92BF92EA
:10A4D000AF921F920E9496F629814FA5BE01695F37
:10A4E0007F4FCE0103960E9405742B013C014B86E1
:10A4F0005C866D867E860FB6F894DEBF0FBECDBF3C
:10A50000AC019B010F941E3D811167C089883A8878
:10A5100025E0382D320380011124030D111D37FC75
:10A520001A95000F111F000F111F015E114FA3019B
:10A5300092016BA57CA58DA59EA50F942C3AD80100
:10A540006D937D938D939C931397632D882D0F941A
:10A55000D207188A81E00E94F746F3948989BBA943
:10A560008B0F63CFA701B80186E40E94A3241B01CF
:10A570002C014EA95FA968AD79AD8CE40E94A3249B
:10A580006B8B7C8B8D8B9E8B2F8A388E498E5A8E4F
:10A590004B2D5C2D6D2D7DA982E40E94A3246B01BF
:10A5A0007C014FA5562D6BA97CA982E50E94A324AE
:10A5B0006B8F7C8F8D8F9E8FCF8ED8A2E9A2FAA24F
:10A5C0004CCE86E69BE0EBCBF3E0FFA704CF3FEF5A
:10A5D0003BAB22242A9484E021CF88890E940C2A54
:10A5E0008A898F5F8A8B05CF0E9405F30E947F20A6
:10A5F000882359F088890E940C2A80E090E0A0EC22
:10A60000BFE78B879C87AD87BE876B857C858D85F3
:10A610009E859B01AC010F941E3D811159C08F8511
:10A62000811126C082E0F82E02E094E0C92E12E0EB
:10A63000DC2CD11A21E041E0612F802F0E94BF1C49
:10A6400021E04FEF612F8F2D0E94BF1C2FEF41E0C3
:10A650006D2D802F0E94BF1C2FEF4FEF6D2D8F2D82
:10A660000E94BF1C115020F70150F3940F3FF9F6E0
:10A670000E94AF3C0E94A42A8F85811124C080EBE8
:10A680009EE00E9488204B015C0188EA9EE00E94C7
:10A690001F289B01AC01C501B4010F94C2339B017B
:10A6A000AC016091B00E7091B10E8091B20E90919C
:10A6B000B30E0F942B3A6093B00E7093B10E80934B
:10A6C000B20E9093B30E8F858111E888E092DA0D77
:10A6D0000E9409BF8091DA0D81110E94B8C10E94C9
:10A6E000BE1F60CCCF93DF93C82FD62F80917B0DF8
:10A6F00083FD14C080913F0A811110C080914402F3
:10A70000909145029C012150310940916213509172
:10A7100063134217530714F40E9406B66D2F8BE0A3
:10A720000E9479F2CC2339F040E061E080E0DF91D3
:10A73000CF910C94998A80913F0A91E08927809368
:10A740003302809133028823F1F020E030E040E0D2
:10A750005FE360915E1370915F138091601390913D
:10A7600061130F942C3A0F94983B2091621330910F
:10A770006313621B730B77FF03C0719561957109B9
:10A780006230710544F41092330280917B0D83FF97
:10A7900006C0C1E01AC080E00E94F746D2CFC09147
:10A7A0003F0AC11112C08091440290914502019765
:10A7B00020916213309163132817390754F70E94D0
:10A7C0002C3686EC97E00E94312E8C2FDF91CF91B2
:10A7D0000895AF92BF92CF92DF92EF92FF920F93C4
:10A7E0001F93CF93DF93CDB7DEB764970FB6F8947E
:10A7F000DEBF0FBECDBF0E94303687FDABC08AE5FD
:10A800000E949624882309F4B6C040E050E0BA01C3
:10A810008AE50E94A3247B018C0163E085E00E940D
:10A8200079F22091B00E3091B10E4091B20E50915C
:10A83000B30E60E070E088EC93E40F942B3A5B0178
:10A840006C019701A8010F948C3C181614F0750147
:10A850008601C701D8018D839E83AF83B88720E02E
:10A8600030E0A901B701C8010F945C33882321F0BF
:10A87000CE0105960E94601E80E090E0A0EAB1E45F
:10A8800089879A87AB87BC871D861E861F86188A94
:10A890008CE40E944824882309F472C00E941E247C
:10A8A0006B017C0120E030E0A901C701B6010F94E3
:10A8B0008C3C87FF04C0F7FAF094F7F8F094C98A4B
:10A8C000DA8AEB8AFC8A00916213109163130430D8
:10A8D0001105DCF020E030E040E05FE360915E13C2
:10A8E00070915F1380916013909161130F942C3AD3
:10A8F0000F94983B601B710B77FF03C071956195B6
:10A90000710901E0643071050CF400E063E080E05F
:10A910000E94725381113DC063E089E00E9479F288
:10A920006D817E818F8198858B019C0130580983D0
:10A930001A832B833C8320E030E0A9010F945C3321
:10A94000882321F0CE0101960E94601E60E089E01C
:10A950000E9479F264960FB6F894DEBF0FBECDBFA9
:10A96000DF91CF911F910F91FF90EF90DF90CF90EB
:10A97000BF90AF900895E12CF12C00E211E44DCF8F
:10A98000C0902C07D0902D07E0902E07F0902F0755
:10A9900089CF83E0E82E22E0AE01475F5F4FBE0122
:10A9A0006F5E7F4FCE010D960E94CA71B9CF4F9254
:10A9B0005F926F927F92AF92BF92CF92DF92EF92AF
:10A9C000FF921F93CF93DF9300D000D01F921F926E
:10A9D000CDB7DEB75C01E62EF42E642F80E00E9436
:10A9E0007253182F81111BC0EE2021F060E089E026
:10A9F0000E9479F2812F28960FB6F894DEBF0FBE21
:10AA0000CDBFDF91CF911F91FF90EF90DF90CF905E
:10AA1000BF90AF907F906F905F904F900895EE2021
:10AA200021F06F2D83E00E9479F280E090E0A0E7B2
:10AA3000B2E48D839E83AF83B88780E090E0A0E886
:10AA4000B0EC89839A83AB83BC83BE016B5F7F4F7D
:10AA5000CE0101960E94FCC068E873E180E090E0BE
:10AA60000E941E2BC12CD12C88ECE82E81E4F82EFC
:10AA7000CD82DE82EF82F88680E090E0A0E8B0E44C
:10AA800089839A83AB83BC83BE016B5F7F4FCE010A
:10AA900001960E94FCC04090CA0D5090CB0D609072
:10AAA000CC0D7090CD0DC092CA0DD092CB0DE0921E
:10AAB000CC0DF092CD0D80E090E0A0EAB1E48D8362
:10AAC0009E83AF83B887F50180819181A281B38194
:10AAD00089839A83AB83BC83BE016B5F7F4FCE01BA
:10AAE00001960E94FCC04092CA0D5092CB0D60921C
:10AAF000CC0D7092CD0D0E94299F64E670E080E03D
:10AB000090E00E941E2B76CF2F923F924F925F9241
:10AB10006F927F928F929F92AF92BF92CF92DF926D
:10AB2000EF92FF920F931F93CF93DF9300D000D04B
:10AB300000D0CDB7DEB74C018B014987590161E0E8
:10AB400082E698E00E945C3441EF54E269E678E0E6
:10AB500085E00E9470F29091120981E0890F809344
:10AB6000120980916C1682FB222720F9288782FF28
:10AB700008C087FDCDC08B7F80936C169E5F90933D
:10AB800012090E94DCC980E1E8EAFEE0A3E2B9E034
:10AB900001900D928A95E1F787E00E94B8BB782E6C
:10ABA00060E070E080E090E4711040C02090B00E52
:10ABB0003090B10E4090B20E5090B30E20E030E0D5
:10ABC00040E050E4C201B1010F942C3A6B017C01CA
:10ABD00020E030E048EC53E40F948C3C181634F439
:10ABE000C12CD12C88ECE82E93E4F92EF801608476
:10ABF000F185FD83F801F285FE83F801F385FF837B
:10AC00009601A701662D7D818E819F2F0F948C3C2C
:10AC1000181624F06C2CDD82EE82FF82A2019101D5
:10AC2000662D7D818E819F810F942B3A288522236A
:10AC300049F02091900D222329F041E0711040E06D
:10AC40000E94F8240E94A8B680911009811109C0C1
:10AC500081E0809310098091A00A80930F091092DF
:10AC6000A00A20E030E0A901F401608171818281B5
:10AC700093810F945C33882391F00E9412B6811166
:10AC80000EC080E090E0A0E7B2E489839A83AB83B2
:10AC9000BC83BE016F5F7F4FC4010E94FCC0711076
:10ACA00004C0B80180E00E949AC520E030E0A9010C
:10ACB000F50160817181828193810F945C338823D7
:10ACC00029F042E06985C5010E94D7540E94299F5E
:10ACD00064E670E080E090E00E941E2B81E02996FF
:10ACE0000FB6F894DEBF0FBECDBFDF91CF911F919D
:10ACF0000F91FF90EF90DF90CF90BF90AF909F901B
:10AD00008F907F906F905F904F903F902F9008951D
:10AD1000188637CFCF92DF92EF92FF92CF93DF93D7
:10AD20006B017C01D42FC0913E0983E080933E09E2
:10AD300081E08093DC0DC114D104E104F10431F011
:10AD40000E94D877C60ED71EE81EF91E8091DC0D32
:10AD5000882389F0C114D104E104F10421F48D2F7A
:10AD60000E94F746F3CF0E94D8776C197D098E09AF
:10AD70009F0997FDF4CF1092DC0DC0933E09DF913F
:10AD8000CF91FF90EF90DF90CF900895FF920F93B7
:10AD90001F93CF93DF93CDB7DEB72D970FB6F894FF
:10ADA000DEBF0FBECDBF082F162F0E94E83661E030
:10ADB000812F0E9465270E94D877685370458F4F76
:10ADC0009F4F6093330970933409809335099093B2
:10ADD000360910923709F0903E0983E080933E09CE
:10ADE00030E020E04AE255E264E578E082E00E944B
:10ADF000DD3484E598E00E946BCF81E08093DC0D28
:10AE00008091DC0D882309F467C060E0812F0E94E7
:10AE1000652780913709882309F45AC060E08AE0E9
:10AE20000E9479F20E942C368AE398E00E94312E2B
:10AE300030E020E044E258E06BE278E082E00E94FB
:10AE4000DD348BE298E00E946BCF41E060E070E07F
:10AE5000CB010E948A5630E020E050E040E067E1FC
:10AE600078E085E00E94DD3467E178E0CE0101966C
:10AE70000F94A232CE0101960E9493C90E9446C649
:10AE800060E080E00E947253802F0E94E8360E94AA
:10AE9000D877685370458F4F9F4F609333097093F5
:10AEA000340980933509909336091092370930E0C0
:10AEB00020E04AE255E26BE078E082E00E94DD3477
:10AEC0008BE098E00E946BCF61E0812F0E946527A4
:10AED00081E00E94F74694CFF0923E092D960FB67E
:10AEE000F894DEBF0FBECDBFDF91CF911F910F91C0
:10AEF000FF900895BF92CF92DF92EF92FF920F934F
:10AF00001F93CF93DF93CDB7DEB7A0970FB6F8941A
:10AF1000DEBF0FBECDBF0E94303687FDDCC061E0D2
:10AF200081E00E9479F285E40E949624882309F446
:10AF3000E2C00E941E246B017C0120E030E0A901E8
:10AF40000F948C3C87FF04C0F7FAF094F7F8F09464
:10AF5000F7FAF094F7F8F094C98EDA8EEB8EFC8E47
:10AF60008CE0E5E9F2E0DE01119601900D928A9500
:10AF7000E1F788E50E949624882351F040E050E0F4
:10AF8000BA0188E50E94A32469837A838B839C831A
:10AF900089E50E949624882351F040E050E0BA01F0
:10AFA00089E50E94A3246D837E838F8398878AE539
:10AFB0000E949624882351F040E050E0BA018AE5CF
:10AFC0000E94A32469877A878B879C87C090280773
:10AFD000D0902907E0902A07F0902B0785E50E9482
:10AFE0009624882321F00E941E246B017C0120E01E
:10AFF00030E0A901C701B6010F948C3C87FF04C063
:10B00000F7FAF094F7F8F094F7FAF094F7F8F09470
:10B01000CD8EDE8EEF8EF8A262E070E082E40E94B8
:10B02000BA24B82E80911209811155C09E01235E69
:10B030003F4F41E0BE016F5F7F4FCE0149960E94B6
:10B040008455882309F447C06B2D81E00E94C656C1
:10B0500070E060E082E50E94BA248C0180E090E01C
:10B06000A0EAB1E48D8B9E8BAF8BB88FC0902C077C
:10B07000D0902D07E0902E07F0902F078CE40E94CF
:10B080009624882321F00E941E246B017C0120E07D
:10B0900030E0A901C701B6010F948C3C87FF04C0C2
:10B0A000F7FAF094F7F8F094C98ADA8AEB8AFC8A06
:10B0B0001D861E861F86188A80911209882359F0E2
:10B0C0002B2DAE014B5E5F4FBE016F5E7F4FCE01F9
:10B0D0000D960E9431B2A0960FB6F894DEBF0FBE57
:10B0E000CDBFDF91CF911F910F91FF90EF90DF9037
:10B0F000CF90BF900895C12CD12C80E8E82E80E439
:10B10000F82E26CFCF92DF92EF92FF920F931F93EC
:10B11000CF93DF93CDB7DEB76C970FB6F894DEBF51
:10B120000FBECDBF8CE40E949624882309F4AFC0E3
:10B130000E941E246B017C0120E030E0A9010F94E5
:10B140008C3C87FF04C0F7FAF094F7F8F094F7FA14
:10B15000F094F7F8F094C98EDA8EEB8EFC8E8CE0CA
:10B16000E5E9F2E0DE01119601900D928A95E1F792
:10B1700088E50E9496248823A1F040E050E0BA01BF
:10B1800088E50E94A3242091B80E3091B90E409119
:10B19000BA0E5091BB0E0F942B3A69837A838B833E
:10B1A0009C8389E50E9496248823A1F040E050E02A
:10B1B000BA0189E50E94A3242091BC0E3091BD0EF6
:10B1C0004091BE0E5091BF0E0F942B3A6D837E833B
:10B1D0008F8398878AE50E949624882351F040E067
:10B1E00050E0BA018AE50E94A32469877A878B8799
:10B1F0009C8761E080E00E9479F21D861E861F8692
:10B20000188A80911209811133C09E01235F3F4F3C
:10B2100040E0BE016F5F7F4FCE0149960E9484558A
:10B22000882331F160E080E00E94C656898D9A8DB6
:10B23000AB8DBC8DB0588D8B9E8BAF8BB88F198A20
:10B240001A8A1B8A1C8A1D861E861F86188A809170
:10B250001209882369F010E000E020E0AE014B5EA7
:10B260005F4FBE016F5E7F4FCE010D960E9431B2DF
:10B270006C960FB6F894DEBF0FBECDBFDF91CF91B5
:10B280001F910F91FF90EF90DF90CF900895C12C08
:10B29000D12C80E8E82E80E4F82E59CF2F923F92EF
:10B2A0004F925F926F927F928F929F92AF92BF92D6
:10B2B000CF92DF92EF92FF920F931F93CF93DF9382
:10B2C000CDB7DEB7E5970FB6F894DEBF0FBECDBFA2
:10B2D0008DAB20913E092CAB21E020933E0980915B
:10B2E000E7098D3409F4C3C4843511F40C94CA6D94
:10B2F000873409F091C18091E5099091E6098B317D
:10B30000910509F4DDC108F079C18430910508F098
:10B3100030C120915C088230910508F48EC1233041
:10B3200008F491C111E0029709F010E00E94C525D0
:10B3300019821A821B821C821D821E821F8218861D
:10B3400082E50E949624882309F490C10E941E245D
:10B350006B017C0120E030E0A9010F945C3388236D
:10B3600009F4EAC04090A80E5090A90E6090AA0E71
:10B370007090AB0E8091AC0E9091AD0EA091AE0E80
:10B38000B091AF0E8CA79DA7AEA7BFA78090130961
:10B3900090901409A0901509B09016098091170992
:10B3A00090911809A0911909B0911A0988AB99AB2D
:10B3B000AAABBBABA5019401C301B2010F945C33EE
:10B3C00081110DC028A939A94AA95BA96CA57DA541
:10B3D0008EA59FA50F945C33882309F4ADC0A3010B
:10B3E0009201C501B4010F942B3A20E030E040E017
:10B3F0005FE30F94C23368A779A78AA79BA72CA500
:10B400003DA54EA55FA568A979A98AA99BA90F9416
:10B410002B3A20E030E040E05FE30F94C2332B0191
:10B420003C0120E030E0A901C701B6010F945C3374
:10B43000881F8827881F181709F40FC180E090E043
:10B44000A0E8BFEB8CA79DA7AEA7BFA728A539A5ED
:10B450004AA55BA5CA01B9010F94C2334B015C0137
:10B46000A3019201C301B2010F94C2339B01AC014D
:10B47000C501B4010F942C3A0F94DA3C4B015C01E6
:10B48000AC019B01C701B6010F942B3A68AB79ABB5
:10B490008AAB9BABA5019401C701B6010F942C3A6E
:10B4A0009B01AC0168A979A98AA99BA90F94C23311
:10B4B0006B017C0120E030E0A9010F948C3C87FDFA
:10B4C000D1C0C701B6010F94DA3C6B017C01C30106
:10B4D000B2019058A50194010F94263B2CA53DA5DF
:10B4E0004EA55FA50F94C233A70196010F94C233F6
:10B4F00028A539A54AA55BA50F942C3A69837A83C0
:10B500008B839C83A501940168A579A58AA59BA539
:10B510000F94263B2CA53DA54EA55FA50F94C233E5
:10B52000A70196010F94C233A30192010F942C3A04
:10B530006D837E838F83988720E030E0A901698145
:10B540007A818B819C810F945C338111A3C020E0B0
:10B5500030E0A9016D817E818F8198850F945C33E5
:10B56000811198C00E94283684E290E10E94312E19
:10B570006AC08531910509F466C08A31910509F4E4
:10B580009CC0049709F048C080E50E949624C12C15
:10B59000D12C7601882321F00E94D81F6B017C01F9
:10B5A00083E50E949624882361F00E941E2420E0F7
:10B5B00030E04AE754E40F94C2330F949F3B6B0191
:10B5C0007C010E94A8B680918813811105C060E0BB
:10B5D0008AE390E10E941BCA0E94D877C60ED71E4C
:10B5E000E81EF91E0E94D8776C197D098E099F0903
:10B5F00097FF29C080E00E94F746F4CF8A32910578
:10B6000009F4A9C160F48D31910509F4FBC008F477
:10B6100070C04E9709F428C10F94EF0814C08B3501
:10B62000910509F47BC28C35910509F47BC28A35FA
:10B63000910591F71092250706C0233020F00E9453
:10B64000C5250E947ABC8DA9811102C00F948B255B
:10B650009CA990933E090C94556580E090E0A0E889
:10B66000BFE3F0CEC12CD12C760131CF89E40E940A
:10B670009624882331F00E941E2469837A838B8369
:10B680009C838AE40E949624882309F455CF0E9463
:10B690001E244ECF412FBE016F5F7F4F83E199E0A3
:10B6A0000E94AA940E94D8776093811370938213AA
:10B6B0008093831390938413C6CF0E94E33EC3CF3D
:10B6C00087E00E946FDE8111BECF8CE0E1EAF2E0FC
:10B6D000DE01119601900D928A95E1F770E060E02D
:10B6E00080E50E94C924BE016F5F7F4F0E949AC50A
:10B6F000AACF87E00E94B8BB811111C08091E009F8
:10B700009091E109A091E209B091E3091EE0B6959C
:10B71000A795979587951A95D1F780FD94CF0E94AC
:10B72000A8B6109247026091DA0D8CE40E94E324DF
:10B73000A82E80E00E940C2A0E94D8776093811383
:10B740007093821380938313909384130E9422BF7B
:10B7500081E080930E080E9427C3C090E009D0903A
:10B76000E109E090E209F090E309A9E1F694E79499
:10B77000D794C794AA95D1F7C0FE0DC081E00E946E
:10B78000B8BB182F82E00E94B8BB11110C94366F21
:10B7900011E0811101C010E08091E0099091E10970
:10B7A000A091E209B091E309F7E1B695A7959795C5
:10B7B0008795FA95D1F780FF02C00C94DF6D1123B5
:10B7C00011F40C94E26DB12E10E00C2D01700C946C
:10B7D000F36D60E070E080E890E40C94FC6DA301F0
:10B7E0009201C701B6010C94456E60E085E590E1D9
:10B7F0000E941BCA0E942C3683E490E10E94312EE5
:10B800000C941D6F0E94D8776093811370938213FC
:10B8100080938313909384138091DA0D81111DC05E
:10B820008091E0099091E109A091E209B091E309CA
:10B83000EDE0B695A79597958795EA95D1F780FFA6
:10B8400004C086E690E10E94DCDD87E00E946FDEA6
:10B850008111F9CE0E94974EF6CE60E08FE40E94EF
:10B86000E3248823E9F2EFCE009196141091971407
:10B87000D8012D913D914D915C916091A80E7091F0
:10B88000A90E8091AA0E9091AB0E0F942C3AAB01A9
:10B89000BC0188E50E94A32469837A838B839C83FF
:10B8A000F80124813581468157816091AC0E7091F9
:10B8B000AD0E8091AE0E9091AF0E0F942C3AAB016D
:10B8C000BC0189E50E94A3246D837E838F839887C2
:10B8D000BE016B5F7F4FCE0101960E94D372882319
:10B8E00009F4B1CE80E00E940C2A0E9422BF61E0E0
:10B8F00085E40E94E324182F21E0482FBE016B5FEE
:10B900007F4FCE0101960E9405746B017C01AC0152
:10B910009B010F941E3D811116C049815A816B8194
:10B920007C8186E790E10E943F2E4D815E816F8190
:10B93000788581E790E10E943F2EB701A6018CE651
:10B9400090E10E94502E0E9409BF11110E94BE1F5B
:10B950000E94BAC178CE80915C08833008F473CE1F
:10B9600089E40E949624082FF12C882319F00E9464
:10B970001A24F82E8AE40E949624E82E882379F06F
:10B980000E941A24182F002309F4C0C0F4E0FF1508
:10B9900008F0B9C08EE790E10E94312E54CE10E03D
:10B9A0000111F4CF80E1E8EAFEE0A3E1B9E0019003
:10B9B0000D928A95E1F7002319F16F2DFF0C770B9B
:10B9C000880B990B0F94633320913D0730913E070C
:10B9D00040913F07509140070F94C23320913507A3
:10B9E0003091360740913707509138070F942C3A21
:10B9F00060931309709314098093150990931609A5
:10BA0000EE2019F1612F110F770B880B990B0F9412
:10BA10006333209141073091420740914307509191
:10BA200044070F94C2332091390730913A0740916F
:10BA30003B0750913C070F942C3A60931709709381
:10BA400018098093190990931A0960E080E50E9413
:10BA5000E3248823C1F10023D1F0E0919614F09102
:10BA60009714208131814281538160911309709133
:10BA7000140980911509909116090F942B3A60933F
:10BA80001309709314098093150990931609EE20F9
:10BA9000D1F0E0919614F09197142481358146817C
:10BAA0005781609117097091180980911909909137
:10BAB0001A090F942B3A6093170970931809809311
:10BAC000190990931A0940E050E0BA0186E40E94F7
:10BAD000A3246B017C0120E030E0A9010F948C3C91
:10BAE0001816C4F420E030E040E752E4C701B60184
:10BAF0000F94263B69837A838B839C83CE010196C6
:10BB00000E9441BFA0CDEE2009F44CCF153008F4BF
:10BB100049CF40CF60E070E0CB01ECCF8FE0809365
:10BB2000250791CD8091E409882381F1893009F0BE
:10BB30008ACD6DEAA62E62E0B62E78EAC72E7EE0A8
:10BB4000D72EE12C00E010E0D5018D915D010E941F
:10BB50009624F82E882361F0133011F0E82EF02E91
:10BB60000E941E24F60160837183828393830F2DCC
:10BB70001F5FF4E0CF0ED11C143031F7EE2009F432
:10BB800064C00E94B8C10E94BAC15DCD5DEAC52EF5
:10BB900052E0D52EF12CE12C00E010E0D6018D9181
:10BBA0006D010E949624382E882309F447C00E9414
:10BBB0001E244B015C01133059F0F701E854F14F9A
:10BBC00020813181428153810F942B3A4B015C01DA
:10BBD000F701E855F14F2081318142815381C50140
:10BBE000B4010F942B3A2B013C012DEB37E346E8CF
:10BBF00055EB0F948C3C87FD0AC02DEB37E346E8EC
:10BC000055E3C301B2010F945C331816BCF4133032
:10BC100021F1F701EE5CF54F5F01A3019201608114
:10BC20007181828193810F942C3AD5016D937D931C
:10BC30008D939C931397812F0E9498BB1F5FB4E054
:10BC4000EB0EF11C143009F0A9CF002309F49BCFAF
:10BC500084EB9EE00E943DBA96CF8092B40E909203
:10BC6000B50EA092B60EB092B70E032DE7CF80911D
:10BC7000E5099091E6098837910511F40C94316734
:10BC800008F0C7C18D34910509F472C608F0EDC003
:10BC90008A31910509F485C508F093C08431910576
:10BCA00009F4BEC408F06EC08131910509F461C485
:10BCB00008F042C0029708F0AFCC80E50E949624BD
:10BCC000C12CD12C7601882321F00E94D81F6B0152
:10BCD0007C0183E50E949624882361F00E941E2443
:10BCE00020E030E04AE754E40F94C2330F949F3BC6
:10BCF0006B017C010E94A8B68091E8099091E90946
:10BD0000009709F431C40E94A9CD8091E509909172
:10BD1000E6096FE970E1892B11F467E970E130E021
:10BD200020E04AE255E282E00E94DD3440E0C701B3
:10BD3000B6010E948A5687CC429709F06DCC83E504
:10BD40000E949624882309F469C70E94D8776093DB
:10BD500081137093821380938313909384130E94B2
:10BD60001E2420E030E04AE754E40F94C2330F94DD
:10BD70009F3B609315027093160280931702909375
:10BD8000180261CC8731910509F487C480F48531AC
:10BD9000910509F47EC4469709F03ECC80916C165B
:10BDA00082FF02C087FF4FCC0E94AB834CCC88310E
:10BDB000910509F48CC4499709F02ECC0E94825851
:10BDC00042CC8032910509F47CC5A8F58D319105EE
:10BDD00009F460C570F48B31910509F4F5C44C97F2
:10BDE00009F01ACC8091E8099091E9090E9456AABD
:10BDF0002ACC8E31910509F454C54F9709F00CCC2B
:10BE00000E944DC56C8F7D8F8E8F9F8FBE016F5F9F
:10BE10007F4FCE014C960E94C9D9CE0101960E9457
:10BE2000C9F20E942C36BE016F5F7F4F82E191E123
:10BE30000E9436AA08CC8934910509F471C550F4E2
:10BE40008132910509F468C5C09709F0E5CB0E94DD
:10BE50007130F9CB8B34910509F486C58C3491058A
:10BE600009F0DACB0E94DCC9EECB8B36910509F4E0
:10BE700035C608F094C08435910509F460CF30F5DB
:10BE80008135910509F4AAC690F48E34910509F024
:10BE9000C3CB70E060E083E50E94BA248E34910544
:10BEA00009F06BC50E94A5B50E9405F3CCCB823585
:10BEB000910509F4ABC68335910509F0ADCB8091AE
:10BEC00025078F7E806280932507BDCB883691053C
:10BED00009F4D4C5E0F58535910509F4E2C68C3541
:10BEE000910509F099CB0E94303687FDACCB80914B
:10BEF000E00984FD09C08091E20987FD05C08091B9
:10BF0000E309837009F455C7ADEACA2EA2E0DA2E20
:10BF1000B2E9EB2EBDE0FB2E10E0D6018D916D0154
:10BF20000E949624882351F0133009F4DFC60E9442
:10BF30001E24F701648B758B868B978B1F5FF4E053
:10BF4000EF0EF11C143049F70E9484B67CCB893681
:10BF5000910509F498C58A36910509F05DCB60E03A
:10BF600080E50E94D72481116ECB8091E009609119
:10BF7000A00A062F80FD02C00FEF10E083E50E94AB
:10BF80009624882349F00E9445208B016F3F71055C
:10BF900019F010F00FEF10E00093A00A54CB813796
:10BFA000910509F4F5C5D0F48E36910509F4A1C5C3
:10BFB00060F48C36910509F446CB8D36910509F075
:10BFC0002BCB81E00E942AD93ECB8F36910509F414
:10BFD000A3C58037910509F436CB1ECB8537910573
:10BFE00009F4F4C658F48237910509F4E7C683379B
:10BFF000910509F011CB0E94D3DC25CB8637910542
:10C0000009F4F6C68737910509F006CB0E9404C3F0
:10C010001ACB8239E1E09E0711F40C94426A08F0D1
:10C0200026C18E3C910511F40C942A6808F06CC06E
:10C030008E3B910509F4CDC5E8F58D37910509F4DE
:10C04000BDCE58F48937910509F0E6CA10920E0862
:10C0500010920D080E9427C3F6CA8C38910509F486
:10C06000B3C58B39910509F0D7CA83E50E949624A0
:10C07000882309F4E8CA0E945520182F8C3308F051
:10C080008CE380931F070E94D8776B017C01212FDE
:10C0900030E0A8EEB3E00F94F439C60ED71EE81EC8
:10C0A000F91EC0921B07D0921C07E0921D07F09268
:10C0B0001E07C9CA8B3C910509F443C7D0F4883CDC
:10C0C000910509F4D6C6893C910509F0A5CA80916D
:10C0D000E00984FD0CC78091E209887809F007C760
:10C0E0008091E309837009F002C781E00E94252F47
:10C0F000AACA8C3C910509F458C78D3C910509F0FA
:10C100008BCA0E945F2F9FCA8D3221E0920711F4E3
:10C110000C94396908F06DC08D3D910509F4CCC7C8
:10C1200008F049C0833D910509F4C2C78C3D9105D3
:10C1300009F072CA82E40E944824882341F0809169
:10C1400060029091610290931A028093190282E535
:10C150000E944824882341F08091190290911A028C
:10C16000909361028093600283E50E949624882365
:10C1700031F00E941A2490936102809360028091B2
:10C18000E0099091E109A091E209B091E309892BBE
:10C190008A2B8B2B09F057CA609160027091610263
:10C1A00089EB91E10E94FB3685E20E942A2E8AE00B
:10C1B0000E942A2E48CA8232A1E09A0709F4D3C706
:10C1C0008C32914009F028CA64E071E083E50E9456
:10C1D000C9248C0168EE73E080E50E94C924893887
:10C1E000F3E19F0710F088E893E1B8010E9466C967
:10C1F0002ACA8033E1E09E0711F40C94836900F5AC
:10C200008E3221E0920711F40C94CD698F32914067
:10C2100009F002CA70E060E085E40E94BA24F82EBA
:10C220002FEF821711F40C943B6A882311F40C94BD
:10C23000136A8FE192E10E94312E0E945CF503CADD
:10C240008039A1E09A0711F40C943E6A813991403B
:10C2500009F0E2C983E50E9448248111F4C9809164
:10C260005E08811190CC81E00E9436C38CCC883F5F
:10C27000E1E09E0711F40C94F96B08F047C0853A91
:10C2800021E0920711F40C94C96AC8F48C39A1E03A
:10C290009A0711F40C944A6A28F48A39914009F4F7
:10C2A000D2C9BAC98D39F1E09F0711F40C94B46D6D
:10C2B000843A914009F0B0C90E94283DC4C9853F25
:10C2C00031E0930711F40C94F16B68F48C3AB1E00F
:10C2D0009B0711F40C94426B843F914009F09CC978
:10C2E0000E9466CAB0C9863FF1E09F0711F40C9422
:10C2F000F56B873F914009F08FC961E083E50E94AB
:10C30000E32491E089270E94C6E19DC9833533E08B
:10C31000930711F40C94BE6C08F0D1C08B35B2E0D9
:10C320009B0711F40C94216C68F48C30F2E09F07A9
:10C3300011F40C940B6C8835924009F06DC90E9481
:10C340007A5781C98D3B32E0930711F40C94AE6C9F
:10C350008E3B924009F060C90E943036182F87FD4D
:10C3600072C98AE50E949624812C912C90E2A92E14
:10C3700091E4B92E882341F040E050E0BA018AE50B
:10C380000E94A3244B015C0164E083E00E9479F2E7
:10C3900020E030E0A901C501B4010F948C3C1816CF
:10C3A0007CF580E090E0A0EAB0E489839A83AB83D7
:10C3B000BC832091B00E3091B10E4091B20E5091DD
:10C3C000B30EC501B4010F942C3A6B017C0120E03F
:10C3D00030E048EC53E40F945C3387FD06C0C12C79
:10C3E000D12C88ECE82E83E4F82ECC8EDD8EEE8EF8
:10C3F000FF8EBE016F5F7F4FCE014C960E948DC0B5
:10C4000085E50E944824882311F40C94B26C0E94A4
:10C410001E246B017C0120E030E0A901C701B601B8
:10C420000F948C3C87FF04C0F7FAF094F7F8F0946F
:10C43000F7FAF094F7F8F094C982DA82EB82FC8282
:10C4400044E061E0CE0101960E94D75420E030E044
:10C45000A901C501B4010F948C3C18165CF580E06D
:10C4600090E0A0EAB0E489839A83AB83BC83A50102
:10C4700094016091B00E7091B10E8091B20E9091C6
:10C48000B30E0F942B3A6B017C0120E030E0A90140
:10C490000F948C3C18161CF0C12CD12C7601CC8E3C
:10C4A000DD8EEE8EFF8EBE016F5F7F4FCE014C960C
:10C4B0000E948DC060E089E00E9479F2C4C8873E86
:10C4C000B3E09B0711F40C94A46DB0F48C36F3E048
:10C4D0009F0709F4B8C8803A934009F09DC820919D
:10C4E000E8093091E90990916C16926090936C166E
:10C4F000C9010E9456AAA7C8883E33E0930711F4E9
:10C500000C94C66D893E934009F086C80E94A8B677
:10C5100080916C16877F8B7F80936C160E94798741
:10C52000811191C80E94F9260E942EAB0E944DC530
:10C530006D3371058105910520F089E693E10E9434
:10C54000DCDD85E693E10E94DCDD80E197EA9093F3
:10C55000310A8093300A81E593E10E94312E8DE407
:10C5600093E10E94DCDD6FC887EA90E10E946BCF07
:10C57000CCCB0E946A1C882309F441C085E40E9448
:10C580004824882361F08091140790911507892B26
:10C5900021F00E941A24811102C00E94319F8091D3
:10C5A000E0099091E109A091E209B091E30947E126
:10C5B000B695A795979587954A95D1F780FF03C0C3
:10C5C00080E00E946D9F8091E30980FF03C081E0BD
:10C5D0000E946D9F8091E0099091E109A091E2098C
:10C5E000B091E30939E1B695A795979587953A9566
:10C5F000D1F780FF28C882E00E946D9F24C860E0C8
:10C600008AEB90E10E941BCA80E00E946D9F81E04E
:10C610000E946D9F82E00E946D9F0E94319F13C80F
:10C6200080916C1684FF2DC082ED90E10E94312E26
:10C6300060E08CE40E94E324182F80916C1684FF44
:10C640001AC08CE896E10E942D848BE1ECE8F6E1BB
:10C65000DE01119601900D928A95E1F730E020E01D
:10C66000412F70E060E0CE0101960E9439ABCE010F
:10C6700001960E94292783EC90E10E94312E0C94B0
:10C68000235B0E942C3683EE90E10E94312E0C94A5
:10C69000235B0E94C3830C94235BE091E809F09133
:10C6A000E9098191882331F08032D9F7DF011197B0
:10C6B0001C92F7CF60E08091E8099091E9090E940F
:10C6C00093AC1092310A1092300A0C94235B83E5EC
:10C6D0000E949624882321F00E9445200E94A8DA17
:10C6E00084E50E9496248823A9F00E9445206B01CE
:10C6F0007C010E947FC5C092400AD092410AE0921C
:10C70000420AF092430ACD28CE28CF2819F081E0C2
:10C7100080938713809112098823F9F080E090E0DC
:10C72000A0EAB1E489839A83AB83BC831C8E1D8EFF
:10C730001E8E1F8E18A219A21AA21BA210E000E0E2
:10C7400020E0AE014F5F5F4FBE01645E7F4FCE01C0
:10C7500080960E9431B20C94235B0E947C2B88232C
:10C7600081F00E94A57B0E94A22B8BE998E00E9499
:10C770004B831092AD0F1092AE0F1092AF0F10922C
:10C78000B00F61E08EE79BE20E945C3441EF54E21F
:10C790006DEE70E185E00E9470F20E9405F30C944A
:10C7A000235B80916C1684FD02C00C94235B83E5AF
:10C7B0000E949624882311F40C94235B0E94452048
:10C7C0000E94A8DA0C94235B8091E0099091E10922
:10C7D000A091E209B091E30922E0B695A79597955B
:10C7E00087952A95D1F780FF2CC083E091E10E94C4
:10C7F000312E8091D3178823F9F0BE016F5F7F4FF0
:10C8000080ED97E10E94DE82CE0101960E94407B7E
:10C81000CE0101960E9473848091D713882339F04A
:10C8200080E20E942A2E87ED93E10E94407B8AE0FD
:10C830000E942A2E0C94235B89EF90E10E94312EF6
:10C84000F6CF83E50E949624882301F10E945520AB
:10C85000182F8C3308F08CE380931A070E94D87746
:10C860006B017C01212F30E0A8EEB3E00F94F43986
:10C87000C60ED71EE81EF91EC0921607D0921707E3
:10C88000E0921807F09219070C94235B0E94727BC8
:10C890000C94235B80916C168E7F80936C160C94A5
:10C8A000235B80916C1684FD02C00C94235B0F9473
:10C8B000D5088091E8099091E9090E94C9AA0C94D1
:10C8C000235B80916C1682FF03C087FF0E94A8B68D
:10C8D00080916C1684FD02C00C94235B60E080E5BF
:10C8E0000E94E324182F682F8091E8099091E909AC
:10C8F0000E9493AC83E50E949624882321F00E9435
:10C9000045200E94A8DA0E94A57B11110C94235B9C
:10C910000E94A22B0C94235B0E94FAE00C94235BF0
:10C9200080E50E9496248823A1F00E941E2420E026
:10C9300030E048EC52E40F94C2330F949F3B6031D7
:10C94000B7E27B0710F060E177E27093310A609301
:10C95000300A82E50E949624882311F40C94235B0C
:10C960000E94D81F0C94235B0E94A22B0C94235B83
:10C9700081E00E94E1CF0C94235B8DE791E10E945E
:10C98000312E6091FD077091FE0784E791E10E94CE
:10C990004AC76091FF077091000887E691E10E9405
:10C9A0004AC76091FD077091FE078091FF07909143
:10C9B0000008681B790B80918713815021E030E0DB
:10C9C000823010F030E020E0621B730B8CE591E1C7
:10C9D0000E9469C784E591E10E94312E809101088F
:10C9E00090910208A0910308B09104088C8F9D8F4C
:10C9F000AE8FBF8FBE016F5F7F4FCE014C960E94FE
:10CA0000C9D9BE016F5F7F4F87E491E10E94C3DE09
:10CA10008091050890910608A0910708B091080838
:10CA20008C8F9D8FAE8FBF8FBE016F5F7F4FCE010A
:10CA30004C960E94C9D9BE016F5F7F4F87E391E199
:10CA40000E94C3DE20E030E04AE754E46091090828
:10CA500070910A0880910B0890910C080F94263B66
:10CA6000AB01BC018FE191E10E943F2E8DE60E9457
:10CA70002A2E8AE00E942A2E0C94235B80E00E94DA
:10CA80002AD90C94235B0E943036182F87FD0AC0E8
:10CA900085E891E10E94312E812F0E94A0888AE0D2
:10CAA0000E942A2EECA9E0933E09E5960FB6F89471
:10CAB000DEBF0FBECDBFDF91CF911F910F91FF90D1
:10CAC000EF90DF90CF90BF90AF909F908F907F902E
:10CAD0006F905F904F903F902F90089560E080E5B9
:10CAE0000E94D72481110C94235B1092A00A0C940D
:10CAF000235B8EE40E949624882311F40C94235B1C
:10CB00000E9445206093460F7093470F8093480F13
:10CB10009093490F0C94235B83E50E94962488230D
:10CB200021F00E94552080937B0D0E942C3686E9CF
:10CB300091E10E94312E80917B0D882331F110E02C
:10CB400000E020E080917B0D90E0002E02C09595E2
:10CB500087950A94E2F780FF12C0FF24F394F20E47
:10CB6000222319F08CE20E942A2EF801EE0FFF1FFB
:10CB7000E457FE4E859194910E94312E2F2D0F5F28
:10CB80001F4F05301105F1F652CE88E891E156CEDF
:10CB900083E50E949624882369F00E9455208D33F6
:10CBA00020F4809314020C94235B8CE38093140292
:10CBB0000C94235B0E942C36609114028DE991E164
:10CBC0000E9494E20C94235B80E00E94DAD80C94DB
:10CBD000235B81E00E94DAD80C94235B0E94B9B6F3
:10CBE0001092A00A0E94448D81E00E94E1CF68EE7D
:10CBF00073E080E090E00E941E2B60E084EA91E107
:10CC00000E941BCA0E94BC1C0C94235B80912507C8
:10CC10008F7D8061809325070C94235B0E946A1CA2
:10CC20008823D9F10E94A8B685E40E944824811186
:10CC30000E94299F8091E0099091E109A091E20969
:10CC4000B091E30907E1B695A795979587950A9561
:10CC5000D1F780FF03C080E00E94389F8091E309F4
:10CC600080FF03C081E00E94389F8091E00990918D
:10CC7000E109A091E209B091E30919E1B695A79500
:10CC8000979587951A95D1F780FD02C00C94235B88
:10CC900082E00E94389F0C94235B0E94B9B60C94EA
:10CCA000235B83E50E944824882311F40C94235BC2
:10CCB0000E94D877609381137093821380938313BB
:10CCC000909384130E941E2420E030E04AE754E44D
:10CCD0000F94C2330F949F3B6093200770932107FA
:10CCE00080932207909323070C94235B0E941E24B9
:10CCF0004B015C0120E030E040EA51E40F945C33EA
:10CD000087FF4EC0A50194016091B20D7091B30DE3
:10CD10008091B40D9091B50D0F94263B2B013C01F1
:10CD2000AC019B0160918C0D70918D0D80918E0DE9
:10CD300090918F0D0F94C23360938C0D70938D0D75
:10CD400080938E0D90938F0DA30192016091C20D7F
:10CD50007091C30D8091C40D9091C50D0F94C23395
:10CD60006093C20D7093C30D8093C40D9093C50D55
:10CD70006091980A7091990A80919A0A90919B0A01
:10CD80000F946133A30192010F94C2330F949F3B20
:10CD90006093980A7093990A80939A0A90939B0AD9
:10CDA0008092B20D9092B30DA092B40DB092B50DD9
:10CDB000C5C881E00F94A8080C94235B0E9467F813
:10CDC0008DE994E10E948C9E0C94235B8091E8098C
:10CDD0009091E909009741F0DC012C91222321F088
:10CDE0000E94C9F20C94235B0E9405F30C94235B10
:10CDF0000091E8091091E90994E0F12C40E091508C
:10CE0000F9F0F8018081282F2B7F213499F42181BA
:10CE10002133B1F4813411F1853409F441E09801F2
:10CE20002E5F3F4F89012F5F3F4FF8018081803295
:10CE3000C9F3E5CF803521F4818180538A3078F3BE
:10CE400041110E942C36FF2021F086EB91E10E94D7
:10CE5000312EC8010E944EDE0C94235BFF24F39414
:10CE6000DECF20930E0820930D080E9427C30C9458
:10CE7000235B8091E00983FD09C08091E2098C70F9
:10CE800029F481E00E94BD360C94235B0E94303669
:10CE9000182F87FF02C00C94235B0091340784E4B1
:10CEA0000E949624F82E8823B1F00E941E244B0184
:10CEB0005C0120E030E0A9010F945C338823A9F0E5
:10CEC00024E01202F0011124E05DF84F808291828B
:10CED000A282B3820F2D602F83E50E94E32480930A
:10CEE00034070E9401B70C94235B80E0F8CF0E94C6
:10CEF000303687FF02C00C94235B0DEA12E0E2E9B2
:10CF0000EE2EEDE0FE2EF1EBCF2EF2E0DF2ED8017B
:10CF10008D918D010E949624882359F00E941E2431
:10CF20000F949F3BF70160837183828393830E94F8
:10CF300036B6F4E0EF0EF11CC016D10641F70C94A2
:10CF4000235B8091E00984FD0DC08091E20988781F
:10CF500049F48091E309837029F481E00E94FB2E5B
:10CF60000C94235B0E94303687FF02C00C94235B35
:10CF70007DEAE72E72E0F72E10E000E0D7018D91F8
:10CF80007D010E949624882349F00E941E24F80106
:10CF9000EE56F24F64A375A386A397A30C5F1F4FB1
:10CFA0000031110559F70C94235B8091E10987FD4D
:10CFB00009C08091E2098E7029F481E00E94D92E87
:10CFC0000C94235B83E50E949624882391F00E94B1
:10CFD0001E246093C60D7093C70D8093C80D909367
:10CFE000C90D6093CE0D7093CF0D8093D00D9093AB
:10CFF000D10D80E50E949624882351F00E941E24C2
:10D000006093C60D7093C70D8093C80D9093C90DA2
:10D0100082E50E949624882351F00E941E2460938A
:10D02000CA0D7093CB0D8093CC0D9093CD0D84E5FC
:10D030000E949624882311F40C94235B0E941E24E2
:10D040006093CE0D7093CF0D8093D00D9093D10D42
:10D050000C94235B8091E0099091E109A091E20991
:10D06000B091E30960E1E62E68E0F62E10E0892B2E
:10D070008A2B8B2B29F481E00E948CDD0C94235B9E
:10D0800088E5810F0E944824882351F00E941E24C5
:10D09000F7016083718382839383812F0E9498BB01
:10D0A0001F5FF4E0EF0EF11C133051F70C94C35DD9
:10D0B0000E9422350C94235B0E943036082F87FF94
:10D0C00002C00C94235B83E50E949624002E000C82
:10D0D000110B7801EE0CFF1C882359F10E941A24D1
:10D0E000F701EA59FD4F91838083000F111F000F54
:10D0F000111F98012E593D4F7901BC01990F880BE2
:10D10000990B0F9463332AE037ED43E25CE30F940D
:10D11000C2330458124FD8012D913D914D915C912D
:10D120000F94C233F70160837183828393830C94DD
:10D13000235B0E942C3685E40E942A2E80E3800F18
:10D140000E942A2EF701EA59FD4F608171818DEB13
:10D1500091E10E94FB3685E20E942A2E8AE00E941D
:10D160002A2E0C94235B8AE50E949624882309F4D6
:10D170005CC00E941E2420E030E040E050EC0F94A0
:10D180005C33C12CD12CE12C30ECF32E87FD13C085
:10D190000E941E2420E030E040E050E40F948C3CDC
:10D1A000C12CD12CE12C20E4F22E181624F00E9480
:10D1B0001E246B017C012091AE0D3091AF0D40918A
:10D1C000B00D5091B10DC701B6010F94C2330F9449
:10D1D000983BCB010E9429F361E080E50E94E324A3
:10D1E000882341F1A70196016091921470919314E4
:10D1F00080919414909195140F942C3A609392140A
:10D200007093931480939414909395140E942C36E9
:10D2100040919214509193146091941470919514CC
:10D2200084ED91E10E94502E05C083E50E94962472
:10D2300081119FCF8091E20987FD14C08091E3099D
:10D24000837081F40E942C36409192145091931473
:10D25000609194147091951485EC91E10E94502E88
:10D260000C94235B82E50E9448248111EBCF0C943F
:10D27000235B8091E00983FD09C08091E1098178F9
:10D2800029F481E00E947A360C94235B80E50E94A9
:10D290009624882351F00E941E2460936513709396
:10D2A0006613809367139093681389E40E94962411
:10D2B000882381F00E941E242CEA35EC47E25EE3CD
:10D2C0000F94C2336093691370936A1380936B1346
:10D2D00090936C1384E40E949624882311F40C9498
:10D2E000235B0E941E242CEA35EC47E25EE30F9498
:10D2F000263B60936D1370936E1380936F1390931E
:10D3000070130C94235B8091E00983FD09C0809128
:10D31000E109817829F481E00E94552E0C94235B69
:10D3200080E50E944824882351F00E941E246093C7
:10D330004E1370934F13809350139093511389E4BD
:10D340000E944824882381F00E941E242CEA35EC98
:10D3500047E25EE30F94C23360935213709353130A
:10D36000809354139093551384E40E944824882397
:10D3700011F40C94235B0E941E242CEA35EC47E246
:10D380005EE30F94263B609356137093571380937C
:10D390005813909359130C94235B83E50E944824FF
:10D3A000182F882369F00E941A249C01909345024B
:10D3B0008093440291E0232B09F090E090933F0A80
:10D3C00080E50E944824882361F020914402309136
:10D3D0004502232B11F00E94692080933F0A0C9490
:10D3E000235B11110C94235B0E942C368FEF91E18B
:10D3F0000E94312E80913F0A882391F087EE91E1BF
:10D400000E94312E60914402709145028EEE91E1AE
:10D410000E94FB368AEE91E10E94312E0C94235B30
:10D4200083EE91E1EDCF04EB10E083E40E949624BB
:10D4300095E0E92E882319F00E941A24E82E83E54E
:10D440000E949624882319F00E941A248C0160E01F
:10D4500085E50E94E324D82E60E082E192E10E94FB
:10D460001BCA2D2D4E2D6F2DC8010E9446990E947A
:10D4700005F30C94235B06E410E0D7CF0E94A8B616
:10D480000C94235B0E947F200E94BE1F0E94BAC1A1
:10D490000C94235B8091E0098878C9F58091E209BA
:10D4A0008670A9F50E942C368CE692E10E94312EFE
:10D4B00080916802882329F187E492E10E94312E4D
:10D4C00040911B0250911C0260911D0270911E023E
:10D4D0008FE592E10E943F2E8CE592E10E94312E71
:10D4E0008AE492E10E94312E80912407882361F022
:10D4F00087E492E10E94312E8AE00E942A2E0C9449
:10D50000235B83E492E1DACF83E492E1F3CF88E412
:10D510000E944824882321F00E94692080932407D8
:10D52000C090E009D090E109E090E209F090E309B1
:10D5300081E1F694E794D794C7948A95D1F731E0C6
:10D54000C322DD24EE24FF2483E50E944824182F03
:10D55000CD28CE28CF2811F4882341F00E94422BF9
:10D56000112321F00E9469208093680284E40E94C4
:10D570004824882311F40C94235B0E941E2460939A
:10D580001B0270931C0280931D0290931E020C9448
:10D59000235B6FEF7FEF89E40E94BA24082F6FEFBF
:10D5A0007FEF8AE40E94BA24182F8AE50E9496240D
:10D5B000D12C811107C081E50E949624D82E8823A2
:10D5C00009F44CC4C02E81E0800F863008F052C0B0
:10D5D000912E81E0810F863008F04CC00E941E24FD
:10D5E0002B013C01F02E07FDF12C07FF02C004E0E7
:10D5F000C02E812E17FD812C17FF02C014E0912E42
:10D60000B5E03B2ECF1410F40C94235BE82C3F9C28
:10D61000500111249E1460F10E2D10E020E030E046
:10D62000A901DD2069F0F501E00FF11FEE0FFF1FEA
:10D63000EE0FFF1FE15EF14F208131814281538166
:10D640000A0D1B1D000F111F000F111F015E114F4E
:10D65000C301B2010F942C3AD8016D937D938D9341
:10D660009C9313976E2D8F2D0F94D207E394D2CFF6
:10D67000F394C8CF0E9428368DE992E10E94312EA2
:10D680000C94235B87E00E946FDE81110C94235B76
:10D6900077E7C72E7CE2D72EE8EAFEE0F9A7E8A7F5
:10D6A0009E012F5F3F4F1901790110E000E0C60194
:10D6B0000E947920A8A5B9A58D909D90AD90BD90B0
:10D6C000B9A7A8A7A50194010F942B3A2B013C01FF
:10D6D000F701408251826282738220E030E040EAAA
:10D6E00051EC0F948C3C87FD0AC020E030E040EA0A
:10D6F00051E4C301B2010F945C33181684F4F801AD
:10D70000EB54FB4DE4911E1654F4B7FAB094B7F8FD
:10D71000B094D7018D929D92AD92BC921397F70170
:10D7200081909190A190B1907F0120E030E040EA9B
:10D7300051ECC501B4010F948C3C87FD3FC020E043
:10D7400030E040EA51E4C501B4010F945C3318168F
:10D75000ACF10F5F1F4FF4E0CF0ED11C0330110569
:10D7600009F0A5CF60E1E62E68E0F62E10E0F101A9
:10D7700081919191A191B1911F01F70181939193B1
:10D78000A193B1937F01812F0E9498BB1F5F13303B
:10D7900071F70E94BAC160E086EB92E10E941BCA59
:10D7A00063E972E084E690E00E9466C96AEB72E089
:10D7B00084E690E00E9466C90C94235B0E942836A0
:10D7C00084ED92E10E94312E61E086EC92E10E94AC
:10D7D0001BCA68E270E088EC90E00E9466C90C9475
:10D7E000235B0E94D1D70C94235B0E9442D60C94F9
:10D7F000235B209349070E9464B510924907882350
:10D8000011F40C94235B0E942C3682EF92E10E946B
:10D81000312E0C94235B10916C1612FF0AC017FD79
:10D8200008C00E947C2B80FB17F910936C160C9497
:10D83000235B14FD02C00C94235B0F94D5080C9459
:10D84000235B8091E10983FD09C08091E209887121
:10D8500029F481E00E947B3A0C94235B0E943036CD
:10D86000082F87FF02C00C94235B85E50E944824A3
:10D87000882359F10E941E244B015C01E02E002EEA
:10D88000000CFF0820E030E0A9010F948C3C87FFDA
:10D8900004C0B7FAB094B7F8B09420E030E84BE396
:10D8A00054E4C501B4010F948C3C970153E0220F5E
:10D8B000331F5A95E1F7285D384F1816D4F1D90176
:10D8C0008D929D92AD92BC9213978CE40E94482455
:10D8D000882311F40C94235B0E941E246B017C01AD
:10D8E000002E000C110B20E030E0A9010F948C3CBD
:10D8F00087FF04C0F7FAF094F7F8F09420E030E8DE
:10D900004BE354E4C701B6010F948C3C980143E00B
:10D91000220F331F4A95E1F7285D384F18169CF007
:10D92000D9011496CD92DD92ED92FC9217970C944A
:10D93000235B80E090E8ABE3B4E4F901808391835A
:10D94000A283B383C2CF80E090E8ABE3B4E4F901F3
:10D9500084839583A683B7830C94235B0E94E95349
:10D960000C94235B28E01202F0011124E85DF84FCB
:10D97000C080D180E280F3800C940B628091E20938
:10D9800087FD09C08091E309837029F481E00E943A
:10D990001ADB0C94235B20908A1430908B144090F7
:10D9A0008C1450908D1460908E1470908F14809011
:10D9B00090143091911438A7C0909214D090931481
:10D9C000E0909414F090951488E50E949624182F06
:10D9D000882309F48AC00E941E24962EA72EB82EF2
:10D9E000092F20E030E046E953EC0F948C3C87FD92
:10D9F0000DC020E030E046E953E4692D7A2D8B2DEF
:10DA0000902F0F945C3318160CF071C06CE271E02B
:10DA10008AE393E10E94FB366CE271E085E393E1D7
:10DA20000E94FB3682E393E10E94312E10E089E5EB
:10DA30000E949624882361F10E941E24962EA72E10
:10DA4000B82E092F20E030E046E953EC0F948C3CCF
:10DA500087FD0DC020E030E046E953E4692D7A2DC2
:10DA60008B2D902F0F945C3318160CF045C06CE290
:10DA700071E08FE193E10E94FB366CE271E08AE194
:10DA800093E10E94FB3687E193E10E94312E10E082
:10DA90008AE50E9496248823A1F10E941E246B012E
:10DAA0007C0120E030E040E151EC0F948C3C87FD9C
:10DAB0000AC020E030E040E151E4C701B6010F9414
:10DAC0005C331816F4F467EF7FEF85E093E10E9472
:10DAD000FB3669E070E080E093E10E94FB368DEF59
:10DAE00092E10E94312E0C94235B11E0A0CF292CEF
:10DAF0003A2C4B2C502E9BCF692C7A2C8B2C08A7C0
:10DB0000C7CF112311F40C94235BC101D201809380
:10DB10008A1490938B14A0938C14B0938D14C3012A
:10DB2000A82DB8A580938E1490938F14A093901471
:10DB3000B0939114C0929214D0929314E0929414E2
:10DB4000F09295140C94235B83E080935C08109210
:10DB5000C81360E083E50E94E32481110C94235BE9
:10DB60000E9428F80C94235B83E50E9448248823B4
:10DB700041F00E9469208093900D0E9401270C942F
:10DB8000235B81E00E940A350C94235B0E947D3761
:10DB90000C94235B1091E5090E94D8776093811360
:10DBA000709382138093831390938413112311F441
:10DBB0000C94235B812F0E94EC870C94235B111142
:10DBC00008C011E08091E3098170B82E81130C9494
:10DBD000E55B8C2D8170B12E81130C94E55B11E017
:10DBE000BB24B39401E082E50E949624882311F4BB
:10DBF0000C94E95B0E941E246CA37DA38EA39FA3BB
:10DC000020E030E0A9010F945C33882361F011110A
:10DC100005C0B11003C0002309F40FC160E0CE01BC
:10DC200084960E94ACC0112309F480C0BB2009F483
:10DC30007AC01092A80E1092A90E1092AA0E1092FD
:10DC4000AB0E1092AC0E1092AD0E1092AE0E109262
:10DC5000AF0E0E94B8C183E89CE20E9479206B015C
:10DC60007C0187E89CE20E9479202B013C01AC01F9
:10DC70009B01C701B6010F948C3C181614F00C944C
:10DC8000EF5BA7019601C301B2010F94263B9B01F4
:10DC9000AC010F94C23320E030E040E85FE30F9422
:10DCA0002C3A0F94DA3C20E030E048E452E40F9440
:10DCB000C23368A379A38AA39BA320E030E040ECA1
:10DCC0005FE3C301B2010F94C233905869837A8332
:10DCD0008B839C8320E030E040EC5FE3C701B6011A
:10DCE0000F94C23390586C8F7D8F8E8F9F8FAE01B3
:10DCF000405E5F4FBE016F5F7F4FCE014C960E942A
:10DD00006BC00E943FC51092A80E1092A90E1092EF
:10DD1000AA0E1092AB0E1092AC0E1092AD0E109295
:10DD2000AE0E1092AF0E80E00E94A3C3BB2019F08C
:10DD300081E00E94A3C3002309F47FC083E00E9416
:10DD40006FDE81117AC00E94B8C120911008309115
:10DD50001108409112085091130860E070E086E1CC
:10DD600093E40F942B3A2B013C012091140830913D
:10DD70001508409116085091170860E070E086E1A0
:10DD800093E40F942B3A6B017C018091B00E90913B
:10DD9000B10EA091B20EB091B30E80931F09909373
:10DDA0002009A0932109B0932209009196141091A3
:10DDB0009714D8012D913D914D915C91C301B20111
:10DDC0000F942B3A609313097093140980931509EB
:10DDD00090931609F8012481358146815781C70146
:10DDE000B6010F942B3A609317097093180980932A
:10DDF000190990931A0983E199E00E947B1C8823FA
:10DE000011F40C94F55B1C8E1D8E1E8E1F8E88E007
:10DE1000E3E1F9E0DE01119601900D928A95E1F7B8
:10DE2000AE01445E5F4FBE016B5F7F4FCE01019636
:10DE30000E946BC082E00E94A3C30E94B8C180917F
:10DE40000D0880930E08AA2019F081E00E940C2A88
:10DE50000E9409BF0E94BAC10C94235B0E9428361D
:10DE60008DE792E10E94312E0C94235B882309F404
:10DE7000A8CEB5CE3FB7F8948091C2099091C3095E
:10DE8000A091C409B091C50926B5A89B05C02F3F34
:10DE900019F00196A11DB11D3FBFBA2FA92F982FD0
:10DEA0008827BC01CD01620F711D811D911D42E0CB
:10DEB000660F771F881F991F4A95D1F708958BE148
:10DEC000ECE8F6E1A7EAB6E101900D928A95E1F758
:10DED00080916C16806480936C1610926116089580
:10DEE000CF9380914013C1E08823C9F08091411302
:10DEF00090914213409138135091391360913A1325
:10DF000070913B13DC01ED91FC910288F389E02DC7
:10DF100028E331E11995C82F811104C0C0E08C2F8E
:10DF2000CF91089540913C1350913D1360913E1361
:10DF300070913F134115510561057105B9F080914C
:10DF4000411390914213DC01ED91FC910288F38919
:10DF5000E02D28E331E11995882301F310923C1359
:10DF600010923D1310923E1310923F1310924013E3
:10DF7000D6CF0F931F93CF93DF93CDB7DEB76097C4
:10DF80000FB6F894DEBF0FBECDBF8C01DC01ED9162
:10DF9000FC910280F381E02DBE016F5F7F4F1995E8
:10DFA000882309F464C08981807CC9F56F8163701E
:10DFB00070E0762F6627770F770F8885B4E08B9F08
:10DFC000C0011124682B792B8985829586958695C9
:10DFD0008370682B6F5F7F4F90E080E02A8523700D
:10DFE000220F3B8537FB332730F9232B3E813F70CF
:10DFF000230F3327331F2750310904C0660F771FC3
:10E00000881F991F2A95D2F760960FB6F894DEBF45
:10E010000FBECDBFDF91CF911F910F910895803436
:10E0200019F568856695669570E090E080E0CB0113
:10E03000772766272A85622B098510E0102F002795
:10E04000012E000C220B330B602B712B822B932B98
:10E050006F5F7F4F8F4F9F4F4AE0660F771F881F7C
:10E06000991F4A95D1F7D0CF8BE0F801848360E007
:10E0700070E0CB01C9CF0895FC01828108958F9291
:10E080009F92AF92BF92CF92DF92EF92FF920F9347
:10E090001F93CF93DF93B0E2A0E06A2F70E0AB0153
:10E0A0004B0F511D55954795411119C0E7E9FFE107
:10E0B00065917491072E000C880B990B0F946333B4
:10E0C000DF91CF911F910F91FF90EF90DF90CF9054
:10E0D000BF90AF909F908F900895B42FE0CFA4177A
:10E0E00011F0B41303C0E3E1F0E2E2CF9A01215052
:10E0F0003109220F331F220F331FF901EB56F04E67
:10E10000E590F490F901E756F04EC591D4918E1543
:10E110009F051CF3A42FC817D9070CF4BECFF90133
:10E12000E956F04E05911491F901E556F04EC5906F
:10E13000D490BC016E197F09072E000C880B990B37
:10E140000F9463334B015C01B601601B710B072E0A
:10E15000000C880B990B0F9463339B01AC01C50134
:10E16000B4010F94C2334B015C01BE016E197F09EB
:10E17000072E000C880B990B0F9463339B01AC01A5
:10E18000C501B4010F94263B6B017C01B801110F4E
:10E19000880B990B0F9463339B01AC01C701B60147
:10E1A0000F942C3A8DCFEF92FF920F931F93E09232
:10E1B0004D07F0924E0700934F071093500760935E
:10E1C000550770935607809357079FEFFF27621BF1
:10E1D000730B840B30F4809570956195790B890BE6
:10E1E000992790932C06A6E06A9F00922006512D55
:10E1F000EE277A9F500DE11D8A9FE00D5093210676
:10E20000E0932206AFE06A9F00922406512DEE278C
:10E210007A9F500DE11D8A9FE00D50932506E093F3
:10E220002606AAE06A9F00922806512DEE277A9FC3
:10E23000500DE11D8A9FE00D50932906E0932A06B8
:10E240001F910F91FF90EF900895000080910F08AB
:10E2500080FF23C089988FEF8093400980910F0839
:10E2600081FF1EC08F9A8FEF8093410980910F0824
:10E2700082FF19C080910B01809582708093090103
:10E280008FEF8093420980910F0883FF13C0169887
:10E290008FEF8093430900000895899A81E0DCCFD5
:10E2A0008F9881E0E1CF80910B018270809309010A
:10E2B00081E0E7CF169A81E0ECCF0F9300914907F8
:10E2C00021E002272AE437E04CE050E0BC0186E27E
:10E2D00097E00E94692C0F9108950F9300914907D0
:10E2E00021E002272AE437E044E050E0BC0186E266
:10E2F00097E00E94692C0F9108950F9300914907B0
:10E3000021E002272AE437E041E050E0BC0186E248
:10E3100097E00E94692C0F9108950F93009149078F
:10E3200021E002272AE437E041E050E0BC0186E228
:10E3300097E00E94692C0F9108950F93009149076F
:10E3400021E002272AE437E048E050E0BC0186E201
:10E3500097E00E94692C0F9108950F93009149074F
:10E3600021E002272AE437E04CE050E0BC0186E2DD
:10E3700097E00E94692C0F9108950F9301E02AE421
:10E3800037E041E050E0BC0186E297E00E94692C52
:10E390000F9108954F925F926F927F928F929F920A
:10E3A000AF92BF92CF92DF92EF920F931F93CF93D2
:10E3B000DF9300D01F92CDB7DEB74C015B016A013D
:10E3C000122F002309F43EC06E2D84E00E9479F2E2
:10E3D0000E942C3681E595E20E94312E61E0812F6A
:10E3E0000E94652700913E0983E080933E0981E009
:10E3F0008093DC0D83E495E20E946BCF80915F16E1
:10E40000882331F040E363E375E282E00E949534B3
:10E410008AE295E20E94C33461E082E095E20E94C4
:10E4200078348091DC0D882359F060E0812F0E94C0
:10E43000652764991092DC0D81E00E94F746F1CFC8
:10E4400000933E096E2D85E00E9479F220E030E0D5
:10E45000A901F40160817181828193810F945C3301
:10E46000882371F080E090E0A0ECB0E489839A8387
:10E47000AB83BC83BE016F5F7F4FC4010E94FCC0B1
:10E4800020E030E0A901F5016081718182819381F2
:10E490000F945C33882351F14090CA0D5090CB0DFE
:10E4A0006090CC0D7090CD0D80E090E0A0E7B1E4DD
:10E4B0008093CA0D9093CB0DA093CC0DB093CD0D4E
:10E4C00080E090E0A0EAB1E489839A83AB83BC83C7
:10E4D000BE016F5F7F4FC5010E94FCC04092CA0D14
:10E4E0005092CB0D6092CC0D7092CD0D812C912C61
:10E4F00080E4A82EBA2C03E020E030E0A901F60168
:10E5000060817181828193810F948C3C181674F420
:10E5100060E086E00E9479F289829A82AB82BC82B6
:10E52000BE016F5F7F4FC6010E94FCC080913D0914
:10E530002AE235E2882311F027E035E245E155E291
:10E540006FE175E281E00E94DD3410913E09009395
:10E550003E091092DC0D1092DB0D8091DB0D8111D4
:10E5600004C081E00E94F746F8CF10933E09813045
:10E5700019F261E086E295E20E94783481E00F9022
:10E580000F900F900F90DF91CF911F910F91EF900F
:10E59000DF90CF90BF90AF909F908F907F906F90C3
:10E5A0005F904F9008954F925F926F927F928F92FB
:10E5B0009F92AF92BF92CF92DF92EF92FF92CF9352
:10E5C000DF9300D000D01F921F92CDB7DEB75C0161
:10E5D000DB01CD90DD90ED90FC90E0919614F091F0
:10E5E0009714FE83ED8384819581A681B781898309
:10E5F0009A83AB83BC839C01AD01C701B6010F9424
:10E600002B3A2B013C01F50180809180A280B380E0
:10E61000AD81BE818D919D910D90BC91A02D8D837A
:10E620009E83AF83B88727E137EB41ED58EBC301F9
:10E63000B2010F948C3C87FDD1C023E030E04BE960
:10E6400053E4C301B2010F945C3318160CF4C6C036
:10E650002D813E814F815885C501B4010F942B3A1D
:10E660002B013C0127E137EB41ED58EB0F948C3C3B
:10E6700087FDB4C023E030E84DE953E4C301B201A3
:10E680000F945C3318160CF4A9C020E030E0A90107
:10E690006D817E818F8198850F942C3A2B013C01EE
:10E6A00020E030E040E251E40F945C3387FF06C085
:10E6B000412C512C30E2632E31E4732E27E137EBED
:10E6C00041ED58E3C301B2010F942B3A9B01AC0119
:10E6D000C501B4010F948C3C87FD80C020E030E878
:10E6E0004DE953E46D817E818F8198850F942C3A9A
:10E6F0002B013C0120E030E041E953E40F948C3CD5
:10E70000181634F4412C512C21E9622E23E4722E88
:10E7100027E137EB41ED58E3C301B2010F942C3AE6
:10E720009B01AC01C501B4010F945C3318160CF4C5
:10E7300055C020E030E0A90169817A818B819C81FC
:10E740000F942C3A4B015C0120E030E040EA51E4A8
:10E750000F945C3387FF06C0812C912C90EAA92E80
:10E7600091E4B92E27E137EB41ED58E3C501B4013F
:10E770000F942B3A9B01AC01C701B6010F948C3C5E
:10E7800087FD2CC020E030E04BE953E469817A81B9
:10E790008B819C810F942C3A4B015C0120E030E08E
:10E7A0004CE853E40F948C3C181634F4812C912CD3
:10E7B0008CE8A82E83E4B82E27E137EB41ED58E32F
:10E7C000C501B4010F942C3A9B01AC01B1E0B983AF
:10E7D000C701B6010F945C3318160CF419828981B5
:10E7E00028960FB6F894DEBF0FBECDBFDF91CF9154
:10E7F000FF90EF90DF90CF90BF90AF909F908F9061
:10E800007F906F905F904F9008952F923F924F921C
:10E810005F926F927F928F929F92AF92BF92CF92B0
:10E82000DF92EF92FF920F931F93CF93DF93CDB7B9
:10E83000DEB76C970FB6F894DEBF0FBECDBF1C01DC
:10E840007B8F6A8F498F2C8FFC01408051806280C2
:10E85000738049825A826B827C82FB01C080D180A6
:10E86000E280F380CD82DE82EF82F8868090B00E67
:10E870009090B10EA090B20EB090B30E89869A8699
:10E88000AB86BC86BE016B5F7F4FCE0101960E94B6
:10E89000D372882309F444C10091961410919714FF
:10E8A000F8012081318142815381C301B2010F946B
:10E8B0002B3A2B013C0149825A826B827C82F801FF
:10E8C0002481358146815781C701B6010F942B3AC7
:10E8D0009B01AC012D833E834F8358878091380282
:10E8E00090913902A0913A02B0913B028D879E87A8
:10E8F000AF87B88BCE010D966C0185017401C30101
:10E90000B2010E94B0BF80915E08811103C081E016
:10E910000E9436C38091910D82FFE8C0209192142D
:10E9200030919314409194145091951460E070E0EC
:10E9300080EA90EC0F942B3A6D8B7E8B8F8B988FA7
:10E9400080E090E0A0E4B1E4898B9A8BAB8BBC8B28
:10E95000BE016F5E7F4FCE0145960E948DC0109123
:10E960005D0810925D0882E00E942CC10E94B8C12F
:10E97000C090B00ED090B10EE090B20EF090B30EF9
:10E9800020919214309193144091941450919514C5
:10E9900060E070E080EA90E40F942B3A9B01AC01B8
:10E9A000C701B6010F948C3C18160CF0C0C060E093
:10E9B00070E080EC9FE72091921430919314409185
:10E9C0009414509195140F942C3A6B017C01AC0176
:10E9D0009B010F941E3D811161C0898D835082304F
:10E9E00008F089C06091B00E7091B10E8091B20EA6
:10E9F0009091B30EE98D20E030E040EA50E4E4303D
:10EA000021F420E030E048EC51E40F942C3A6D8B77
:10EA10007E8B8F8B988F69ED72E0CE0145960E94B8
:10EA20008DC0FC8DF33008F446C02091B80E3091B3
:10EA3000B90E4091BA0E5091BB0EF1016081718107
:10EA4000828193810F942C3AAB01BC0181EE94E258
:10EA50000E943F2E2091BC0E3091BD0E4091BE0E03
:10EA60005091BF0EEA8DFB8D60817181828193810F
:10EA70000F942C3AAB01BC018CED94E20E943F2E26
:10EA8000B701A60187ED94E20E94502EA7019601DE
:10EA9000C701B6010F941E3D882369F00E947F20B4
:10EAA00060E088EC94E20E941BCA0E94283688EB42
:10EAB00094E20E94312EC701B6016C960FB6F8940D
:10EAC000DEBF0FBECDBFDF91CF911F910F91FF90A1
:10EAD000EF90DF90CF90BF90AF909F908F907F90FE
:10EAE0006F905F904F903F902F90089560E070E09E
:10EAF00080E291EC21CF898D8150823008F091CF56
:10EB00000E947F20882309F48CCFFC8DC12CD12C4E
:10EB100080ECE82E8FE7F82EF33008F4BFCF85CFD6
:10EB2000C12CD12C90ECE92E9FE7F92EC4CF12FF17
:10EB30003ECF20E030E040EA50E4C701B6010F9438
:10EB40002C3A6D877E878F87988B69ED72E0CE01B6
:10EB50000D960E948DC080E090E0A0ECB0E48D871F
:10EB60009E87AF87B88BBE01635F7F4FCE0145960E
:10EB70000E948DC010915D0810925D0882E00E9495
:10EB80002CC10E94B8C14090B00E5090B10E609060
:10EB9000B20E7090B30E2091921430919314409164
:10EBA00094145091951460E070E080EA90E40F9422
:10EBB0002B3A9B01AC01C301B2010F948C3C181697
:10EBC0000CF4F5CE12FFF3CE20E030E040E450E448
:10EBD000C301B2010F94C2332B013C01A70196017E
:10EBE000C701B6010F942C3A9B01AC01C301B201DD
:10EBF0000F942C3A2DEC3CEC4CE45EE30F94C233C2
:10EC0000DACE4F925F926F927F928F929F92AF92E5
:10EC1000BF92FF920F931F93CF93DF93CDB7DEB7D1
:10EC200068970FB6F894DEBF0FBECDBFF82E4A012D
:10EC30005B012801390120E030E0A901C301B801DE
:10EC40000F945C33811111C0FF2019F081E0F8129C
:10EC500088C060E070E88BE395E420E030E040E7B6
:10EC600052E40F94263B2B013C014D8A5E8A6F8A49
:10EC7000788E0F2D10E0F801EB54FB4DE4917724D2
:10EC800073941E160CF4712CFF24F39420E030E0F2
:10EC9000A901C501B4010F948C3C18160CF0F12C9D
:10ECA00080E00E942ABB69837A838B839C8381E006
:10ECB0000E942ABB6D837E838F83988782E00E94A7
:10ECC0002ABB69877A878B879C8783E00E942ABB4F
:10ECD0006D877E878F87988B000F111F000F111F84
:10ECE000E1E0F0E0EC0FFD1F0E0F1F1FF801108296
:10ECF000118212821382CE0101960E9475BAF80128
:10ED000080829182A282B382198A1A8A1B8A1C8A03
:10ED10008091A10A9091A20A892B51F4AE014F5E15
:10ED20005F4FBE016B5E7F4FCE0101960E9484F95A
:10ED30000E94A8B67F100E943FC568960FB6F8944F
:10ED4000DEBF0FBECDBFDF91CF911F910F91FF901E
:10ED5000BF90AF909F908F907F906F905F904F90FB
:10ED6000089560E070E086E194E477CFCF93DF937D
:10ED700000D01F92CDB7DEB721E0FC0123A784812C
:10ED80009581A681B781B05889839A83AB83BC8370
:10ED9000BE016F5F7F4F83E199E00E9408210F90D1
:10EDA0000F900F900F90DF91CF910895282F30E0B2
:10EDB000F901E159FB4D9491F901E75DFB4D449157
:10EDC0002D513C4DF9012491222309F435C099239A
:10EDD00011F191509231F8F4E92FF0E08827EC50CE
:10EDE000F9488F4F0D94233A2577297706771D77B9
:10EDF00021770B772C77327736773C7740774477DB
:10EE00004A774E770B77527758775C7780918000FE
:10EE10008F7780938000E22FF0E0EE0FFF1FE75323
:10EE2000FC4DA591B4918FB7F894EC91611148C055
:10EE300040954E234C938FBF0895809180008F7D25
:10EE4000E8CF80918000877FE4CF84B58F7784BD41
:10EE5000E2CF84B58F7DFBCF8091B0008F77809318
:10EE6000B000D9CF8091B0008F7DF9CF8091900014
:10EE70008F7780939000CFCF809190008F7DF9CFD6
:10EE800080919000877FF5CF8091A0008F7780934D
:10EE9000A000C1CF8091A0008F7DF9CF8091A0000C
:10EEA000877FF5CF809120018F7780932001B3CFAA
:10EEB000809120018F7DF9CF80912001877FF5CF50
:10EEC0004E2BB8CFCF93DF93EC018D810E949E3CF7
:10EED00060E08B81DF91CF910C94D67661E0FC01EC
:10EEE00083810E94D6768FEF0C94923CCF93DF9370
:10EEF000EC016EBDFA01CA019E5F0DB407FEFDCFA5
:10EF000020812EBD0DB407FEFDCF21812EBD32968E
:10EF1000E817F90791F70DB407FEFDCF8FEF0E94B8
:10EF2000923C8FEF0E94923C0E94973C8E838F719F
:10EF3000853049F083E18C83CE010E946E7780E0BA
:10EF4000DF91CF91089581E0FBCF8F929F92AF9296
:10EF5000BF92CF92DF92EF92FF926B017C010E94F1
:10EF60003A6F4B015C01C114D104E104F104B9F022
:10EF70000E943A6F681979098A099B09683E7340B3
:10EF80008105910580F321E0C21AD108E108F1085A
:10EF900088EE880E83E0981EA11CB11CE4CFFF9080
:10EFA000EF90DF90CF90BF90AF909F908F9008959B
:10EFB0002FB7F8946091BE097091BF098091C00984
:10EFC0009091C1092FBF0895CF92DF92EF92FF92E7
:10EFD0000E94D8776B017C0128E5C20E22E0D21E88
:10EFE000E11CF11C0E94973C8F3F71F00E94D87782
:10EFF0006C197D098E099F0997FDF4CF80E0FF9081
:10F00000EF90DF90CF90089581E0F9CF0F931F9399
:10F01000CF938C010E9462770E94E477C82F8823E7
:10F0200071F08DEF0E94923C0E94E477C82FC801D6
:10F030000E946E778C2FCF911F910F91089582E1DE
:10F04000F8018483F4CF0F931F93CF93DF93EC01E8
:10F050008B010E9462770E94E47781110CC085E1E8
:10F060008C8310E0CE010E946E77812FDF91CF91CB
:10F070001F910F910895A8016CEFCE010E94767741
:10F08000182F882361F3EECFDF92EF92FF920F9358
:10F090001F93CF93DF938C01C62FD22FF32EE42E34
:10F0A000D52E0E9462770E94E4778C2F80640E94A4
:10F0B000923C8D2D0E94923C8E2D0E94923C8F2D71
:10F0C0000E94923C8D2F0E94923C87E8C11101C0A2
:10F0D00085E90E94923CCC3011F40E94973CC0E03C
:10F0E0000E94973CF801868387FF04C0CF3F11F050
:10F0F000CF5FF6CFDF91CF911F910F91FF90EF90EF
:10F10000DF9008958F929F92AF92BF92CF92DF923D
:10F11000EF92FF920F931F93CF93DF93EC016A015D
:10F120007B01590120E030E0A90167E30E944478A7
:10F13000A501980167E1CE010E944478811127C0A2
:10F140008F81833039F089E0CC0CDD1CEE1CFF1C74
:10F150008A95D1F7A701960169E1CE010E94447812
:10F1600011E0882319F010E087E08C83CE010E9423
:10F170006E77812FDF91CF911F910F91FF90EF90CC
:10F18000DF90CF90BF90AF909F908F90089589E0CF
:10F190008C8310E0EBCF0F931F93CF93DF93EC01A1
:10F1A00089018F81833039F089E0440F551F661F34
:10F1B000771F8A95D1F79A01AB0168E1CE010E94D1
:10F1C000447881112AC0A8016EEFCE010E947677A3
:10F1D000182F8823B1F00E94E477182F8823D1F0EC
:10F1E00020E030E0A9016DE0CE010E944478882340
:10F1F00021F086E18C8310E004C00E94973C8111CD
:10F20000F8CFCE010E946E77812FDF91CF911F91B1
:10F210000F91089587E18C83F4CF86E0EBCF1F93A5
:10F22000CF93DF93EC010E94627720E030E0A901E8
:10F230006CE0CE010E94447811E0882319F010E0C0
:10F2400083E08C83CE010E946E77812FDF91CF9176
:10F250001F9108951F93CF93DF93EC018F8183302B
:10F2600039F089E0440F551F661F771F8A95D1F743
:10F270009A01AB0162E1CE010E94447811E088233B
:10F2800019F010E085E08C83CE010E946E77812F0B
:10F29000DF91CF911F9108958F929F92AF92BF926D
:10F2A000EF92FF920F931F93CF93DF938C01EB01AB
:10F2B0007A010E94D8774B015C012CE2820E21E09A
:10F2C000921EA11CB11C0E94973CF80186838F3FBF
:10F2D00069F40E94D877681979098A099B0997FD12
:10F2E000F2CF81E1F8018483C0E021C08E3F71F547
:10F2F000F1E0EF1AF1088FEF8EBDFE012FEF0DB494
:10F3000007FEFDCF8EB581932EBDCF018C1B9D0BCB
:10F310008E159F05A0F30DB407FEFDCF8EB5CE0D63
:10F32000DF1D88830E94973C0E94973CC1E0C80182
:10F330000E946E778C2FDF91CF911F910F91FF90DC
:10F34000EF90BF90AF909F908F9008958FE0CACFBD
:10F350000F931F93CF93DF93EC018B010E94627791
:10F3600040E052E0B801CE01DF91CF911F910F91A3
:10F370000C944C790F931F93CF93DF93EC01890189
:10F380008F81833039F089E0440F551F661F771F46
:10F390008A95D1F79A01AB0161E1CE010E944478D0
:10F3A00081110AC040E052E0B801CE01DF91CF9157
:10F3B0001F910F910C944C7984E08C83CE010E94B4
:10F3C0006E7780E0DF91CF911F910F9108950F9399
:10F3D0001F93CF93DF93EC018B0120E030E0A90174
:10F3E00069E00E94447881110AC040E150E0B80110
:10F3F000CE01DF91CF911F910F910C944C7980E158
:10F400008C83CE010E946E7780E0DF91CF911F91B7
:10F410000F9108958F929F92AF92BF92CF92DF92F9
:10F42000EF92FF920F931F93CF93DF93EC01162F70
:10F430001F821C824B830E94D8776B017C0120EDD8
:10F44000C20E27E0D21EE11CF11CA89561E08B8161
:10F450000E94D6768B8190E0FC01E75DFB4D249104
:10F460008D519C4DFC018491882399F090E0880F88
:10F47000991FFC01E756FF4DA591B491FC01E7539C
:10F48000FC4D859194918FB7F894EC912E2B2C9391
:10F490008FBF209A289A219A2398229A81E00E946D
:10F4A0009E3C85E08D830E949E3C0AE08FEF0E9487
:10F4B000923C0150D9F7A89520E030E0A90160E026
:10F4C000CE010E9444788E83813081F00E94D877EB
:10F4D0006C197D098E099F0997FDEECF81E08C8321
:10F4E000CE010E946E771A8280E06AC0A8952AEA4F
:10F4F00031E040E050E068E0CE010E944478853081
:10F5000041F581E08F83A8958F81812C912C540146
:10F51000823029F4812C912CA12C80E4B82E20E09B
:10F5200030E0A90167E3CE010E944478A50194016F
:10F5300069E2CE010E9444788E838823F1F00E9414
:10F54000D8776C197D098E099F0997FDE8CF8AE06D
:10F55000C6CF04E00E94973C8E830150D9F78A3AC7
:10F5600011F482E0CFCF0E94D8776C197D098E0903
:10F570009F0997FDBCCF82E0B2CF8F818230C1F46A
:10F5800020E030E0A9016AE3CE010E94447888239C
:10F5900011F088E0A4CF0E94973C807C803C11F45D
:10F5A00083E08F830E94973C0E94973C0E94973C87
:10F5B000CE010E946E7781E08A83173070F41D833C
:10F5C000DF91CF911F910F91FF90EF90DF90CF903F
:10F5D000BF90AF909F908F90089588E18C8384CFE7
:10F5E0001F920F920FB60F9211242F933F938F9378
:10F5F0009F93AF93BF938091BE099091BF09A09153
:10F60000C009B091C1093091BD0923E0230F2D3706
:10F6100058F50196A11DB11D2093BD098093BE0927
:10F620009093BF09A093C009B093C1098091C2090A
:10F630009091C309A091C409B091C5090196A11D7B
:10F64000B11D8093C2099093C309A093C409B093DC
:10F65000C509BF91AF919F918F913F912F910F90CD
:10F660000FBE0F901F90189526E8230F0296A11D3C
:10F67000B11DD2CF8DE00E942A2E8AE00C942A2E52
:10F68000CF93DF93EC018991882319F00E942A2EF1
:10F69000FACFDF91CF910895809161168823C1F050
:10F6A000815080936116ECE8F6E1882351F0815097
:10F6B000990B2BE1289FF001299FF00D1124EE53A7
:10F6C000F94E8BE1A7EAB6E101900D928A95E1F738
:10F6D00080916116811105C090916C169064909391
:10F6E0006C160895CF92DF92EF92FF9280916C1684
:10F6F00082FF23C0C0906816D0906916E0906A1609
:10F70000F0906B168FEF91E20E94312EC701B60187
:10F710000E948DF08FE20E942A2E609164167091F3
:10F72000651680916616909167160E948DF0FF9085
:10F73000EF90DF90CF900C943A7B81E192E2FF90C2
:10F74000EF90DF90CF900C94312E80916C1684FF57
:10F7500004C08460877F80936C160895CF92DF92F7
:10F76000EF92FF920F931F93CF93DF93CDB7DEB746
:10F77000EDB6FEB6DC010D900020E9F79D01281BD7
:10F78000390B285F3F4FEDB7FEB7E21BF30B0FB607
:10F79000F894FEBF0FBEEDBF0DB71EB70F5F1F4F32
:10F7A0009F938F9389E291E29F938F931F930F937F
:10F7B0000F94F3326801F4E0CF0ED11C0F900F903C
:10F7C0000F900F900F900F90D6018D916D018823AF
:10F7D00049F0082E000C990B0F943E3DF60131972D
:10F7E0008083F2CF64E271E2C8010F948C324FE360
:10F7F00050E0B8018CE198E00F949A3D0FB6F89470
:10F80000FEBE0FBEEDBEDF91CF911F910F91FF9015
:10F81000EF90DF90CF900895FC01938591FD13C088
:10F82000987121E0903109F020E080916C1620FB66
:10F8300085F980936C16903141F08085873419F4F6
:10F8400081858E3711F480E0089581E00895FC01F0
:10F8500020E03EE2DB014D91BD01403249F028300D
:10F8600011F430833196DB0111974C91408331962E
:10F870002F5F2B3079F710820895EF92FF920F934C
:10F880001F93CF93DF93CDB7DEB7A0970FB6F89451
:10F89000DEBF0FBECDBF7C018B01BE016F5F7F4F0E
:10F8A000C7010E9412F11816A4F4CE0101960E941D
:10F8B0000C7C882391F3BE016F5F7F4F8AEC93E14C
:10F8C0000E94277C6AEC73E1C8010F945C3D892B90
:10F8D00021F7A0960FB6F894DEBF0FBECDBFDF9123
:10F8E000CF911F910F91FF90EF900895CF92DF92EB
:10F8F000EF92FF92CF936B017C01C42F809138135C
:10F9000090913913A0913A13B0913B138C159D053A
:10F91000AE05BF0529F10E94706F811108C0C0E0DB
:10F920008C2FCF91FF90EF90DF90CF900895809132
:10F93000411390914213DC01ED91FC910088F18913
:10F94000E02D28E331E1B701A6011995882339F3A9
:10F95000C0923813D0923913E0923A13F0923B13CD
:10F96000CC2321F081E080934013DACFC1E0D8CFDF
:10F970004F925F926F927F928F929F92AF92BF92BF
:10F98000CF92DF92EF92FF920F931F93CF93DF936B
:10F99000EC01423051056105710590F480E0DF9182
:10F9A000CF911F910F91FF90EF90DF90CF90BF907C
:10F9B000AF909F908F907F906F905F904F90089541
:10F9C00089859A85AB85BC850196A11DB11D8417DB
:10F9D0009507A607B70710F38F898031C9F5852EE3
:10F9E000962EA72EBB248B899C89AD89BE89880E53
:10F9F000991EAA1EBB1E280139016A017B0141E044
:10FA0000C501B4010E94767C882341F29F89903120
:10FA100081F5DD24EE24FF24F601EE0FFF1FE85CE4
:10FA2000FE4E118300839A89923008F4B8CF4D813D
:10FA30005E816F817885840E951EA61EB71E80920A
:10FA40003C1390923D13A0923E13B0923F13A7CF68
:10FA5000803209F0A3CF8B899C89AD89BE894A0188
:10FA60005B01E7E0B694A79497948794EA95D1F761
:10FA7000BECFE894C7F8DD24EE24FF24F601EE0F94
:10FA8000FF1FEE0FFF1FE85CFE4E40825182628234
:10FA90007382C9CFCF92DF92EF92FF920F931F93A1
:10FAA000CF93DF93FC0181859285A385B485019670
:10FAB000A11DB11D84179507A607B70750F480E074
:10FAC000DF91CF911F910F91FF90EF90DF90CF903A
:10FAD000089587898031A9F5BB27A72F962F852FF9
:10FAE000C388D488E588F6888C0D9D1DAE1DBF1D8A
:10FAF000E9016A017B018F0140913813509139135C
:10FB000060913A1370913B1384179507A607B707C6
:10FB100049F5F8018789803169F5B701A6015527B4
:10FB200066277727440F551F485C5E4EFA01808197
:10FB30009181B0E0A0E088839983AA83BB8381E0B0
:10FB4000BFCF803209F0BBCFC388D488E588F68860
:10FB5000DB01CA01C7E0B695A79597958795CA9529
:10FB6000D1F7C2CF40E0BC01CD010E94767C81116B
:10FB7000D0CFA5CFB701A6014F77552766277727A6
:10FB8000440F551F440F551F485C5E4EFA0180819B
:10FB90009181A281B381BF70CECF4F925F926F925D
:10FBA0007F92AF92BF92CF92DF92EF92FF920F932C
:10FBB0001F93CF93DF9300D01F92CDB7DEB78C0198
:10FBC00049835A836B837C835901C12CD12C7601E4
:10FBD000412C82E0582E612C712C49815A816B8115
:10FBE0007C819E012F5F3F4FC8010E944A7D882380
:10FBF00019F1F8018585A301920104C0220F331F7A
:10FC0000441F551F8A95D2F7DA01C901C80ED91EC3
:10FC1000EA1EFB1E49815A816B817C818789803174
:10FC2000F1F481E0483F5F4F61057105B0F2F501E5
:10FC3000C082D182E282F3820F900F900F900F90DA
:10FC4000DF91CF911F910F91FF90EF90DF90CF90B8
:10FC5000BF90AF907F906F905F904F90089581E03C
:10FC6000483F5F4F6F4F7F4008F4B7CFE0CF0F930F
:10FC70001F93CF93DF93FC012381222331F080E097
:10FC8000DF91CF911F910F9108958B01EC01FB0142
:10FC90008789803139F582E08B831D8A1E8A1F8A0D
:10FCA000188E808D918DB0E0A0E025E0880F991F1F
:10FCB000AA1FBB1F2A95D1F7898B9A8BAB8BBC8B64
:10FCC0001A8F098F81E08983188619861A861B8608
:10FCD0001C821D821E821F82188A1C861D861E861B
:10FCE0001F86CECF803259F683E08B83428D538DB1
:10FCF000648D758D4D8B5E8B6F8B788F9E012F5E23
:10FD00003F4FC8010E94CD7D8111DACFB8CF3F921D
:10FD10004F925F926F927F928F929F92AF92BF921B
:10FD2000CF92DF92EF92FF920F931F93CF93DF93C7
:10FD3000CDB7DEB72C970FB6F894DEBF0FBECDBFA0
:10FD40005C01DC0159968D909C90F401818592852F
:10FD5000A385B4859C01AD012F5F3F4F4F4F5F4F8F
:10FD600029873A874B875C87D50114964D905D9023
:10FD70006D907C901797411451046104710409F44B
:10FD800059C0BFEF4B1A5B0A6B0A7B0A312C730117
:10FD900062011D821E821F821886F4018185928570
:10FDA000A385B4852D813E814F8158852817390759
:10FDB0004A075B0708F056C089859A85AB85BC85E4
:10FDC0008C159D05AE05BF0550F482E0C82ED12CE0
:10FDD000E12CF12C92E0492E512C612C712C9E01CA
:10FDE0002F5F3F4FB701A601C4010E944A7D8823BF
:10FDF000C9F189819A81AB81BC81892B8A2B8B2B9C
:10FE000001F1260137019FEF491A590A690A790A57
:10FE10002D813E814F8158852F5F3F4F4F4F5F4F60
:10FE20002D833E834F8358873FEFC31AD30AE30ADB
:10FE3000F30AB3CF408051806280738033243394BF
:10FE4000A6CFC414D504E604F70411F70FEF1FEF93
:10FE50002FEF3FE0B701A601C4010E94B87C782EC5
:10FE600081111AC0712C872D2C960FB6F894DEBF25
:10FE70000FBECDBFDF91CF911F910F91FF90EF90FB
:10FE8000DF90CF90BF90AF909F908F907F906F90BA
:10FE90005F904F903F900895F501448155816681B0
:10FEA0007781411551056105710539F0970186018A
:10FEB000C4010E94B87C8823A9F2D5011496CD9282
:10FEC000DD92ED92FC921797332051F0D701C601D5
:10FED0000196A11DB11DF40180839183A283B38398
:10FEE000F50185899689A789B08D892B8A2B8B2B63
:10FEF00009F0B9CFC58AD68AE78AF08E81818068F9
:10FF00008183B1CFCF93DF93EC01462F41706C8595
:10FF10007D858E859F850E94767C882351F0888917
:10FF200020E2829FC0011124885C9E4EDF91CF9118
:10FF3000089590E080E0FACFCF93DF93EC018B81BE
:10FF4000882349F1898187FF22C061E0CE010E94A8
:10FF5000827FFC01892BF9F08081853EE1F08B8165
:10FF6000823040F489899A89AB89BC89848F958FC6
:10FF7000A68FB78F8D899E89938F828F8D899E8959
:10FF8000AF89B88DB58BA48B89818F778983DF91F9
:10FF9000CF910C94706F81E0888380E0DF91CF91E6
:10FFA00008958F929F92AF92BF92CF92DF92EF927D
:10FFB000FF920F931F93CF93DF93EC018B818111FD
:10FFC0000EC080E0DF91CF911F910F91FF90EF90D5
:10FFD000DF90CF90BF90AF909F908F900895098948
:10FFE0001A892B893C89041715072607370748F318
:10FFF0004A015B01823031F488869986AA86BB86E5
:020000021000EC
:1000000081E0E0CF81149104A104B10449F4188681
:1000100019861A861B861C821D821E821F82F0CFC3
:10002000088519852A853B85E98DFA8D858590E0BF
:100030000996B901A8014150510961097109082EB9
:1000400004C076956795579547950A94D2F7750140
:100050006401E1E0CE1AD108E108F10804C0F69489
:10006000E794D794C7948A95D2F7C416D506E606C6
:10007000F70620F0012B022B032B11F58D899E89A9
:10008000AF89B88D8C839D83AE83BF838E010C5F57
:100090001F4FC114D104E104F10409F4ADCF4C8128
:1000A0005D816E817F819801898D9A8D0E944A7D44
:1000B00091E0C91AD108E108F1088111EACF81CF96
:1000C000C41AD50AE60AF70AE1CF2F923F924F925F
:1000D0005F926F927F928F929F92AF92BF92CF92D8
:1000E000DF92EF92FF920F931F93CF93DF9300D095
:1000F0001F92CDB7DEB78C014B011A01DC011396BC
:100100008C911397813009F0CFC011968C9181FFAB
:10011000CBC082FDB5C06101D80118964D915D91AB
:100120006D917C911B97C114D10409F41BC15996A0
:100130008D919C915A97FC0174802FEF270D2A0115
:100140003B0139E076946794579447943A95D1F7F8
:10015000722E74207A01F1E0FF22711020C0E114A8
:10016000F104E9F414964D915D916D917C9117978E
:10017000411551056105710509F09CC055968D9199
:100180009D910D90BC91A02D0097A105B10509F09E
:10019000AAC0C8010E94877E882309F485C0A12CCB
:1001A00082E0B82EAE18BF08CA14DB0408F456016A
:1001B000D80159964D915C915A9714968D919D91C5
:1001C0000D90BC91A02D0297A109B109FA012585D6
:1001D00004C0880F991FAA1FBB1F2A95D2F7468516
:1001E000578560897189840F951FA61FB71F9C01D1
:1001F000AD01270D311D411D511D29013A01A114E9
:1002000032E0B30609F07DC0809138139091391324
:10021000A0913A13B0913B13481659066A067B0623
:1002200069F4109240138FEF9FEFDC018093381335
:1002300090933913A0933A13B0933B1380914113D9
:1002400090914213DC01ED91FC910288F389E02D3D
:100250009401B301A2011995882331F1F801808539
:100260009185A285B3858A0D9B1DA11DB11D808737
:100270009187A287B3878A0C9B1CCA18DB084CCFD6
:10028000F801418952896389748980859185A285A5
:10029000B385481759076A077B0709F43CCFC801A3
:1002A0000E94D17F811137CF81E0D8018C938FEFED
:1002B0009FEF6EC09E012F5F3F4F0E944A7D8823B3
:1002C00099F389819A81AB81BC81F801218D328DAE
:1002D000F9012789203169F4883FFFEF9F07A105C5
:1002E000B10508F056CFF80184839583A683B783C0
:1002F00056CF883F2FEF9207A2072FE0B20798F35F
:1003000048CFE114F10431F5F8014085518562854B
:10031000738581899289A389B489481759076A0727
:100320007B07C0F00E94706F882309F4BDCF81E085
:1003300080934013409238135092391360923A13CD
:1003400070923B13A501B401C701885C9E4E0F94C7
:10035000533D84CF41E0C301B2010E94767C8111FC
:10036000F1CFA2CFF80181899289A389B48984173A
:100370009507A607B70738F48181418B528B638BB1
:10038000748B80688183F801818183FD18C0C1016D
:100390000F900F900F900F90DF91CF911F910F91C1
:1003A000FF90EF90DF90CF90BF90AF909F908F9095
:1003B0007F906F905F904F903F902F900895C8016D
:1003C0000E949C7F8111E3CF6FCF2F923F924F927B
:1003D0005F926F927F928F929F92AF92BF92CF92D5
:1003E000DF92EF92FF920F931F93CF93DF93EC0175
:1003F0004B017A018B81811115C08FEF9FEFDF9147
:10040000CF911F910F91FF90EF90DF90CF90BF9011
:10041000AF909F908F907F906F905F904F903F90A4
:100420002F900895898180FFE8CF89899A89AB89C7
:10043000BC89488559856A857B85841B950BA60BED
:10044000B70BA70170E060E084179507A607B70710
:1004500008F47C0167011E0124E0220E311CC11446
:10046000D10409F4A9C0488559856A857B855A015C
:1004700081E0B822898D9A8D2A013B0129E076948A
:100480006794579447942A95D1F72B81FC01223029
:1004900081F5628D738D848D958D640D751D861D1E
:1004A000971D00E012E00A191B09C016D10608F4D6
:1004B00086010115E2E01E0771F440903813509058
:1004C000391360903A1370903B13641575058605D7
:1004D000970509F04EC040E00E94767C882309F41D
:1004E0008CCFB501685C7E4EA801C4010F94533DCA
:1004F00052C0148111501421A114B10471F41111CE
:100500000CC0452B462B472B51F58D899E89AF8911
:10051000B88D8C839D83AE83BF83E98DFA8D4C802B
:100520005D806E807F8022E0421A51086108710868
:10053000858504C0440C551C661C771C8A95D2F72F
:1005400086859785A089B189480E591E6A1E7B1E33
:10055000C301B201610F711D811D911DA2CF4C819C
:100560005D816E817F8191010E944A7D8111D5CF8D
:1005700044CFA0914113B0914213ED91FC9111979A
:100580000088F189E02D9401AB01BC01CD011995E2
:10059000882309F432CF800E911E88859985AA851B
:1005A000BB85800F911FA11DB11D88879987AA87E0
:1005B000BB87C01AD10A53CFC70121CFCF93DF9396
:1005C000EB01FC012381211104C080E0DF91CF9178
:1005D00008952250223028F48FE28883198281E026
:1005E000F5CF60E00E94827F009779F3DC0160E044
:1005F00080E09EE22D91203299F0883031F49E0106
:10060000260F311DF90190836F5F9E01260F311D6A
:10061000AD0141505109FA014081F90140836F5FFA
:100620008F5F8B3039F7FE01E60FF11D1082D7CFB7
:10063000CF93DF93EC01CB01E881F9816081718177
:100640000E94DE8228813981D901ED91FC91AA8135
:10065000BB818C919081992359F08936C8F4CF01E0
:100660000196F901918380838C918F5F8C93EACFFF
:10067000893670F48FE28083E881F98180819181ED
:10068000019691838083EA81FB8180818F5F8083E3
:10069000DF91CF9108950F931F93CF93DF9300D0F5
:1006A00000D01F92CDB7DEB79C012F5F3F4F3F8335
:1006B0002E832FE2FC01208381E08D83CE010696FC
:1006C0009A83898301979C838B8310E00BE180914F
:1006D0006116181758F4109FB00111246E53794E0B
:1006E000CE0101960E9418831F5FF1CF8D818B355B
:1006F00058F460ED77E1CE0101960E9418838E8157
:100700009F8101979F838E83EE81FF8110822796C0
:100710000FB6F894DEBF0FBECDBFDF91CF911F9112
:100720000F910895CF93DF93EC010E949C7F1B8271
:10073000DF91CF9108951092120980916C168F77F6
:1007400080936C160E947C2B882321F080ED97E12A
:100750000C9492830895CF93C0916C16C2FF10C081
:10076000C7FD0EC00E947C2B80FBC7F9C0936C169E
:1007700080916C168F7E806480936C16CF91089563
:100780000E949B83F5CFCF93DF9380916C168F7E71
:1007900080936C1680918F16882321F08CE896E167
:1007A0000E94928380916D1690916E16DC01ED91FE
:1007B000FC910190F081E02D45E360E019958111F5
:1007C0000EC00E942C3688E191E20E94312E809169
:1007D0006C1684FF34C0DF91CF910C945F6FC09191
:1007E0006D16D0916E1661E0CE010E94B0F68111B7
:1007F0000BC060E0CE010E94B0F6811105C00E94DE
:10080000283684E091E2E1CF6AE574E18CE896E174
:100810000E94377E811105C00E94283683EF90E246
:10082000D4CF80916C16806180936C160E942C3618
:1008300087EE90E20E94312E0E94E9E0C8CF8091BD
:100840005C08882339F06FEF87ED90E2DF91CF915C
:100850000C941BCADF91CF91089540E050E0BA019B
:100860000C94D17F0F931F93CF93DF93CDB7DEB757
:10087000EB970FB6F894DEBF0FBECDBF80916C161C
:1008800000E010E084FF23C087EA96E10E942D84F7
:100890008BE1E7EAF6E1DE01919601900D928A95EF
:1008A000E1F710E000E0BE016F5F7F4FCE0181965F
:1008B0000E9412F118163CF4CE0101960E940C7CA5
:1008C000080F111DF0CFCE0181960E942927C80183
:1008D000EB960FB6F894DEBF0FBECDBFDF91CF9180
:1008E0001F910F9108950F931F93CF93DF93CDB76F
:1008F000DEB76B970FB6F894DEBF0FBECDBF8C018D
:1009000087EA96E10E942D848BE1E7EAF6E1DE01B9
:10091000119601900D928A95E1F7B801CE010196EA
:100920000E943D7CCE0101960E9429276B960FB64E
:10093000F894DEBF0FBECDBFDF91CF911F910F9115
:1009400008952F923F924F925F926F927F928F9273
:100950009F92AF92BF92CF92DF92EF92FF920F934E
:100960001F93CF93DF93CDB7DEB7C454D1090FB631
:10097000F894DEBF0FBECDBF7C014B015A01222E81
:1009800019821C821C8E1F8E6115710511F410E0F6
:10099000B3C1DC0113968C918111F9CFFA018081EA
:1009A0008B018F32D1F4DB0113968C911397825017
:1009B000823060F059966D917C91CE014C960E94E8
:1009C000377E8E01045E1F4F882309F3C5015C0149
:1009D0000196F50120812F32D1F39E012F5F3F4F09
:1009E0006901290130E2332E2496CFAE2497259653
:1009F000DFAE25973E013CE1630E711C22963FAEAF
:100A0000229721963FAE21973FAE3EAE3DAE3CAE23
:100A10003BAE3AAE39AE38AE3FAA950190E047E022
:100A2000D9018D91882361F18F3251F18E3239F4E1
:100A30004A3009F4ACCF98E04AE09D01F1CFE3EBF6
:100A4000F0E22491222321F031968213FACF9FCF36
:100A5000491708F49CCF813208F499CF8F3709F4F5
:100A600096CF3FE9380F3A3108F420EEE7E3F0E0A3
:100A7000EC0FFD1FE90FF11D820F80839F5FDDCF1B
:100A80008FA9803209F483CF5901D9018C912F5F4E
:100A90003F4F8F32C9F38823A9F00815190519F0C3
:100AA000C8010E94928324969FAD249725968FAD0E
:100AB00025974C145D0411F4962D872D8601C92EBF
:100AC000D82E9CCFF801818D928DD7015A969C9398
:100AD0008E935997C8010E942D84C12CF8018085FE
:100AE0009185A285B3854189528963897489841768
:100AF0009507A607B70708F053C025E0B695A79558
:100B0000979587952A95D1F7F82FFF70DF2ED8019A
:100B100013968C91823008F43ACF41E050E0BE0148
:100B20006E5B7F4FC8010E94E581019709F02FCFCE
:100B3000F80180859185A285B3854F96A11DB11DD1
:100B400080879187A287B387F0E2DF9EB0011124EE
:100B5000685C7E4E6115710509F419CFDB018C913B
:100B6000882341F0853E09F04DC0CC2029F0CC24EB
:100B7000C394B4CFC1100EC0809138139091391333
:100B8000A0913A13B0913B13F70184879587A6870C
:100B9000B787D08ADB018C918111E9CFCC24C39433
:100BA000822D8274823409F0F2CECC2009F4C7C0C1
:100BB000F701D08861E0C7010E94827F009709F4A5
:100BC000E6CE20E2DC011D922A95E9F72BE0FE013A
:100BD000F796DC0101900D922A95E1F721E238E2C7
:100BE000FC01318B208B40E058E057874687338BE0
:100BF000228B318F208F578B468B0E94706F811113
:100C00000AC0C5CE4BE050E0CE01C7960F94463DDA
:100C1000892B09F063CF2D2D30E0F901B5E0EE0FFF
:100C2000FF1FBA95E1F7DF01A85CBE4E1B968C91C1
:100C3000817121F0822D827109F020C1D70159966E
:100C40008D919C915A97409138135091391360912E
:100C50003A1370913B131C964D935D936D937C9367
:100C60001F975096DC925097E85CFE4E84889588DA
:100C7000B12CA12C54019924882455968D929D92D3
:100C8000AD92BC925897428D538D70E060E0482938
:100C900059296A297B2955964D935D936D937C93D1
:100CA0005897A5E0220F331FAA95E1F7D901A85C58
:100CB000BE4E1B962C91287109F0D2C0848D958D63
:100CC000A68DB78DF701818B928BA38BB48B81E0BE
:100CD0008383822D8F70F70181831482158216829F
:100CE0001782108611861286138611E024FE04C036
:100CF000C7010E94A0F3182FCE014C960E9429270D
:100D0000CE0101960E942927812FCC5BDF4F0FB6C1
:100D1000F894DEBF0FBECDBFDF91CF911F910F9131
:100D2000FF90EF90DF90CF90BF90AF909F908F900B
:100D30007F906F905F904F903F902F900895D801D3
:100D400013968C911397823009F421CE51968D9190
:100D50009D910D90BC91A02D803E9F4FAF41B1055C
:100D600008F015CEC8010E94877E882309F40FCEB3
:100D70000E94706F882309F40ACED8015996ED912C
:100D8000FC915A9714968D909D90AD90BC901797BA
:100D9000B2E08B1A9108A108B108858504C0880CBF
:100DA000991CAA1CBB1C8A95D2F786859785A089B9
:100DB000B189880E991EAA1EBB1E81E08093401344
:100DC0008092381390923913A0923A13B0923B1349
:100DD000E8E3F1E180E092E0DF019C011D92215007
:100DE0003040E1F7DD24D394D8015996ED91FC9180
:100DF0008481D816C0F48091411390914213DC0194
:100E0000ED91FC910288F389E02D28E331E1B501F1
:100E1000A4014D0D511D611D711D1995882309F403
:100E2000B6CDD394E1CF258580E092E0A0E0B0E09C
:100E300004C0880F991FAA1FBB1F2A95D2F7F8017B
:100E40004189528963897489840F951FA61FB71F32
:100E5000818B928BA38BB48B88E391E1D12CB1CEA3
:100E6000203161F497012F5E3F4F0E94CD7D882392
:100E700029F084E0D70113968C932BCFD7011396DA
:100E80001C9285CD1F93CF93DF93CDB7DEB76D97BF
:100E90000FB6F894DEBF0FBECDBF1D8E1C8EAC0109
:100EA000BE01645E7F4F80E00E9434F410E0009742
:100EB000A9F019821C826C8D7D8D21E0AC01CE01E0
:100EC00001960E94A184182F882321F0CE0101965B
:100ED0000E949283CE0101960E942927812F6D9650
:100EE0000FB6F894DEBF0FBECDBFDF91CF911F913B
:100EF0000895EF92FF921F93CF93DF9300D000D01D
:100F000000D01F92CDB7DEB780916216882309F416
:100F100047C080916C1684FF0E94C38380916C1639
:100F200084FF3CC00E941727811138C0809162164F
:100F300090E08F969F938F9382E292E29F938F939C
:100F4000CE0101967C019F938F930F94F332809191
:100F50006C160F900F900F900F900F900F9084FFD2
:100F60001DC0C7010E944287182F8823B9F00E9434
:100F70005F6FC7010E94AE7B809162168F5F809386
:100F80006216812F2A960FB6F894DEBF0FBECDBF32
:100F9000DF91CF911F91FF90EF900895109262160C
:100FA00010E0EFCFCF9321E044ED52E06CE876E122
:100FB00081E796E10E94A184C82F882321F081E770
:100FC00096E10E9492838C2FCF910895682F70E054
:100FD00090E080E00C948DF0CF93C82F0E942C36C7
:100FE00084E50E942A2E8C2F0E94E68780E20E94D0
:100FF0002A2E87E890E2CF910C94312E8F929F9207
:10100000AF92BF92CF92DF92EF92FF92CF936B019C
:101010007C01B42E20E030E0A9010F945C3387FFFF
:1010200007C08DE20E942A2EF7FAF094F7F8F094A8
:10103000C0E060E070E080E09FE3CB1541F02DEC74
:101040003CEC4CEC5DE30F94C233CF5FF6CFA701CD
:1010500096010F942C3A6B017C010F949F3B4B013E
:101060005C010E948DF0CC2371F1C501B4010F9495
:1010700061339B01AC01C701B6010F942B3A6B01A0
:101080007C018EE20E942A2EC150E8F020E030E080
:1010900040E251E4C701B6010F94C2336B017C01F9
:1010A0000F949F3B4B015C010E948DF0C501B40180
:1010B0000F9461339B01AC01C701B6010F942B3A29
:1010C0006B017C01E1CFCF91FF90EF90DF90CF904B
:1010D000BF90AF909F908F900895EF92FF920F93E3
:1010E0001F93CF937B018A01C2E48F3F09F0C4E5CF
:1010F00080E20E942A2E8C2F0E942A2E8AE30E94D0
:101100002A2EF701608171818281938142E00E94E1
:10111000FE8783E790E20E94312EF80160817181A1
:101120008281938142E00E94FE8762E070E080E06D
:1011300090E0CF911F910F91FF90EF900C94A577C5
:101140001F93CF93DF9300D000D01F921F92CDB793
:10115000DEB7182F6091621370916313072E000C95
:10116000880B990B0F9463336D837E838F839887ED
:1011700080915E1390915F13A0916013B091611301
:1011800089839A83AB83BC83AE014B5F5F4FBE0103
:101190006F5F7F4F80E80E946D8860914B13709164
:1011A0004C13072E000C880B990B0F9463336D833F
:1011B0007E838F8398878091471390914813A091E5
:1011C0004913B0914A1389839A83AB83BC83AE01E0
:1011D0004B5F5F4FBE016F5F7F4F8FEF0E946D8847
:1011E00060914D131F3F39F087E11802F00111247F
:1011F000E65AFC4E628570E08BE790E20E94FB3677
:1012000060914D1370E086E790E20E94FB362896CD
:101210000FB6F894DEBF0FBECDBFDF91CF911F9107
:1012200008952F923F924F925F926F927F928F928A
:101230009F92AF92BF92CF92DF92EF92FF920F9365
:101240001F93CF93DF93CDB7DEB764970FB6F894B3
:10125000DEBF0FBECDBF898B6A8B81E080933302E6
:101260001A821B821C821D8219861A861B861C8686
:101270001D862CE32E873CE13F8746E4488B312CCA
:10128000212C50E85B8B8FEB8C8B198291E0988737
:10129000812C912C540160914B1370914C13072EAB
:1012A000000C880B990B0F9463337B018C01232D69
:1012B000322D4B895C890F945C338823B9F02091DF
:1012C0004713309148134091491350914A13A9890B
:1012D000B701C801A111EEC00F945C33881F8827A5
:1012E000881F89833E2C2F2C0B8B1C8B0E94D87758
:1012F0006B017C01DC01CB0129853A854B855C853E
:10130000821B930BA40BB50BB7FD2EC0D701C601F2
:1013100088519C4FAF4FBF4F89879A87AB87BC8757
:1013200080E00E94A08883E890E20E94312E811420
:101330009104A104B10409F4EAC0C501B4016857DD
:101340007C4E8F4F9F4F6C197D098E099F0928EEA7
:1013500033E040E050E00F94A039CA01B9010E9487
:10136000F7F08AE00E942A2E80E00E94F7460E9451
:10137000D877609381137093821380938313909333
:101380008413909147139E83A0914813AF830091DB
:10139000491310914A13292F3A2FA801632D722D5A
:1013A0008B899C890F942B3A2B013C0120E030E083
:1013B000A9010F948C3C87FF04C077FA709477F8EA
:1013C000709481149104A104B10409F0A4C020E038
:1013D00030E040E050E4C301B2010F945C3387FF7A
:1013E00010C0B885812C912C5401BB2331F082E8C8
:1013F000882E86E0982EA12CB12C8C0C9D1CAE1C46
:10140000BF1C29812223A9F18A819B81AC81BD81E6
:10141000892B8A2B8B2B61F0D701C6012A813B8156
:101420004C815D81821B930BA40BB50BB7FD21C0D2
:101430002E813F81A8016D857E858F8598890F94C7
:101440002B3A20E030E040E85FE30F945C3387FD07
:1014500035C0D701C601805A9541AF4FBF4F8A832F
:101460009B83AC83BD839E819D87AF81AE870F87B1
:10147000188BBA89BB2339F08091B8091092B8094A
:10148000811110923302809133028823B9F08114C4
:101490009104A104B10461F028E8C21A23E1D20A40
:1014A000E108F108C818D908EA08FB08F7FE06C0E9
:1014B0001886F1CE0F945C3387FF23C0B0913302BE
:1014C000B983BB2321F0109233020E9405F3898176
:1014D00064960FB6F894DEBF0FBECDBFDF91CF91FB
:1014E0001F910F91FF90EF90DF90CF90BF90AF9042
:1014F0009F908F907F906F905F904F903F902F9034
:1015000008953E2C2F2C0B8B1C8B1982EFCE8FE372
:101510000E942A2E26CF20E030E040E450E4C301B0
:10152000B2010F948C3C18160CF06BCF460157019A
:1015300068CF2F923F924F925F926F927F928F92DD
:101540009F92AF92BF92CF92DF92EF92FF920F9352
:101550001F93CF93DF93CDB7DEB766970FB6F8949E
:10156000DEBF0FBECDBF8A8B6B8B4C8B2091850766
:10157000298B1092850781E0809333021A821B82A7
:101580001C821D8219861A861B861C861D863CE3DA
:101590003E874CE14F8756E4588B312C212C80E854
:1015A0008D8B9FEB9E8B1982A1E0A887812C912CBB
:1015B00054016091621370916313072E000C880B25
:1015C000990B0F9463337B018C01232D322D4D89B0
:1015D0005E890F945C338823B9F020915E133091BB
:1015E0005F134091601350916113BB89B701C8012B
:1015F000B111EEC00F945C33881F8827881F898340
:101600003E2C2F2C0D8B1E8B0E94D8776B017C01FA
:10161000DC01CB0129853A854B855C85821B930BC8
:10162000A40BB50BB7FD2EC0D701C60188519C4F46
:10163000AF4FBF4F89879A87AB87BC878A890E9443
:10164000A0888FE790E20E94312E81149104A104BA
:10165000B10409F4EDC0C501B4016053784F8F4F58
:101660009F4F6C197D098E099F0928EE33E040E0F9
:1016700050E00F94A039CA01B9010E94F7F08AE046
:101680000E942A2E80E00E94F7460E94D87760933D
:10169000811370938213809383139093841390919A
:1016A0005E139E83A0915F13AF830091601310912E
:1016B0006113292F3A2FA801632D722D8D899E89E0
:1016C0000F942B3A2B013C0120E030E0A9010F944C
:1016D0008C3C87FF04C077FA709477F8709481147B
:1016E0009104A104B10409F0A7C020E030E040E873
:1016F0005FE3C301B2010F945C3387FF10C0B8856C
:10170000812C912C5401BB2331F08AE9882E82E090
:10171000982EA12CB12C8C0C9D1CAE1CBF1C2981B9
:101720002223A9F18A819B81AC81BD81892B8A2BDF
:101730008B2B61F0D701C6012A813B814C815D81F1
:10174000821B930BA40BB50BB7FD21C02E813F81EB
:10175000A8016D857E858F8598890F942B3A20E0AE
:1017600030E040EC5FE30F945C3387FD35C0D70178
:10177000C601805A9541AF4FBF4F8A839B83AC838C
:10178000BD839E819D87AF81AE870F87188BBC89F3
:10179000BB2339F08091B8091092B80981111092D9
:1017A0003302809133028823B9F081149104A1049B
:1017B000B10461F020EDC21A27E0D20AE108F10875
:1017C000C818D908EA08FB08F7FE06C01886F1CE4B
:1017D0000F945C3387FF26C0209133022983222394
:1017E00021F0109233020E9405F339893093850766
:1017F000898166960FB6F894DEBF0FBECDBFDF912C
:10180000CF911F910F91FF90EF90DF90CF90BF90FD
:10181000AF909F908F907F906F905F904F903F9090
:101820002F9008953E2C2F2C0D8B1E8B1982ECCE01
:101830008FE30E942A2E23CF20E030E040E450E4E2
:10184000C301B2010F948C3C18160CF068CF46010E
:10185000570165CF809128028F37E8F18F5790911B
:1018600064139093B7099923A1F12C9A20914D13F9
:101870002093B60990910201211190959072909356
:1018800000018F5F809328028091B50991E089273C
:101890008093B50980912702980F85300CF090E075
:1018A000823009F470C01CF58823B9F1813009F445
:1018B0005EC0909327020E949DC28091A10A9091E0
:1018C000A20A009729F001979093A20A8093A10A97
:1018D00008952C98CBCF9091B709891708F02C98D0
:1018E0009091B609891768F290910201C7CF8430B0
:1018F00009F461C00CF45AC08530D9F62091B409BE
:10190000211102C08093B4098091B4098150809361
:10191000B409882371F295E0CCCF809126028F5FC5
:1019200080311CF480932602C4CF1092260280914D
:10193000B309811113C020915A1330915B13309376
:101940005D1320935C132091431330914413309323
:1019500046132093451381E08093B30910925B13E3
:1019600010925A131092441310924313A2CF88E09E
:1019700080937B0085E480937C0080917A00806472
:1019800080937A0096CF80917A0086FD27C040919F
:1019900078005091790020915A1330915B13240FF5
:1019A000351F30935B1320935A1383CF88E08093C5
:1019B0007B0086E4E0CF80917A0086FD11C04091E3
:1019C0007800509179002091431330914413240FF3
:1019D000351F30934413209343136BCF92E069CFAC
:1019E00094E067CF0F930FB70F9300916E000D7FB8
:1019F00000936E0078940F930BB70F930CB70F9270
:101A00001F922F933F934F935F936F937F938F9387
:101A10009F93AF93BF93EF93FF9311240E942A8C5F
:101A2000FF91EF91BF91AF919F918F917F916F91B6
:101A30005F914F913F912F911F900F900CBF0F918D
:101A40000BBF0F910260F89400936E000F910FBFCF
:101A50000F9118952091621330916313263531054B
:101A60003CF420914B1330914C132630310524F077
:101A7000882349F00C94A22B662329F081E00E9470
:101A8000E1CF0C9405F30895CF93DF93109285076F
:101A9000EAE5F3E111861086109281071092820721
:101AA000109283071092840712862C98C3E4D3E126
:101AB000198618860E94D4271A86809102018072A6
:101AC00080930001DF91CF910895CF92DF92EF9242
:101AD000FF920F931F93CF93DF93CDB7DEB72C9771
:101AE0000FB6F894DEBF0FBECDBF182F6B017A0181
:101AF00080915C08833090F00E942836C6010E94D5
:101B0000312E8BE49FE10E94312E1F3F89F587E43F
:101B10009FE10E94312E8AE00E942A2E0E94448D6D
:101B2000A89580918809811155C081E0809388092A
:101B300082E080935C080E94448D05E10150409A48
:101B400049F169E170E080E090E00E94A577A895F6
:101B5000409868E270E080E090E00E94A577A89548
:101B600068E270E080E090E00E94A577A895E6CF5B
:101B700017FDD1CF85E49FE10E94312E612F012E08
:101B8000000C770B880B990B0E94F7F08AE00E94FB
:101B90002A2EC1CF87E00E946FDE811111C08CE038
:101BA000E1EBF2E0DE01119601900D928A95E1F7EA
:101BB000BE016F5F7F4F80E00E949AC50E94A8B669
:101BC0006EE37FE11F3F11F062E47FE140E0C70177
:101BD0000E94A73A2C960FB6F894DEBF0FBECDBF79
:101BE000DF91CF911F910F91FF90EF90DF90CF90F9
:101BF00008952F923F924F925F926F927F928F92B1
:101C00009F92AF92BF92CF92DF92EF92FF920F938B
